:0200000460009A
:10040000464346420004015600000000010102007C
:1004100000000000000000000000000000000000DC
:1004200000000000000000000000000000000000CC
:1004300000000000000000000000000000000000BC
:1004400000000000010403000000000000000000A4
:10045000000080000000000000000000000000001C
:10046000000000000000000000000000000000008C
:10047000000000000000000000000000000000007C
:10048000EB04180A063204260000000000000000F9
:10049000050404240000000000000000000000002B
:1004A000000000000000000000000000000000004C
:1004B0000604000000000000000000000000000032
:1004C000000000000000000000000000000000002C
:1004D00020041808000000000000000000000000D8
:1004E000000000000000000000000000000000000C
:1004F00000000000000000000000000000000000FC
:10050000D8041808000000000000000000000000EF
:100510000204180804200000000000000000000091
:1005200000000000000000000000000000000000CB
:100530006004000000000000000000000000000057
:1005400000000000000000000000000000000000AB
:10055000000000000000000000000000000000009B
:10056000000000000000000000000000000000008B
:10057000000000000000000000000000000000007B
:10058000000000000000000000000000000000006B
:10059000000000000000000000000000000000005B
:1005A000000000000000000000000000000000004B
:1005B000000000000000000000000000000000003B
:1005C0000001000000100000010000000000000019
:1005D000000001000000000000000000000000001A
:1005E000000000000000000000000000000000000B
:1005F00000000000000000000000000000000000FB
:10100000D100204100C0006000000000000000008E
:1010100020100060001000600000000000000000D0
:10102000000000600000800000000000FFFFFFFFE4
:10C00000008000205932026045D703602D3602605F
:10C0100015360260213602602736026000000000FB
:10C020000000000000000000000000004DD7036089
:10C0300041D703600000000051D70360B5D402600F
:10C0400055D7036059D703605DD7036061D703609C
:10C0500065D7036069D703606DD7036071D703604C
:10C0600075D7036079D703607DD7036081D70360FC
:10C0700085D7036089D703608DD7036091D70360AC
:10C0800095D7036041D7036041D7036041D7036070
:10C0900099D703609DD70360A1D70360A5D703603C
:10C0A00041D7036059910260A9D7036041D703606B
:10C0B000ADD70360B1D7036041D7036041D70360B8
:10C0C000B5D70360B9D7036041D7036041D7036098
:10C0D00041D7036041D7036041D7036041D7036074
:10C0E00041D7036041D7036041D7036041D7036064
:10C0F00041D7036041D7036041D7036041D7036054
:10C1000041D7036041D7036041D7036041D7036043
:10C1100041D7036041D7036041D7036041D7036033
:10C12000BDD7036041D70360C1D70360C5D70360A3
:10C13000C9D7036041D7036041D7036041D703608B
:10C1400041D7036041D7036041D7036041D7036003
:10C15000CDD7036041D7036041D7036041D7036067
:10C1600041D7036041D7036041D7036041D70360E3
:10C1700041D7036041D7036041D7036041D70360D3
:10C1800041D7036041D7036041D7036041D70360C3
:10C1900041D7036041D7036041D7036041D70360B3
:10C3F00041D7036041D7036041D70360FFFFFFFFD0
:10C40000024B1A6902601861002070470004002086
:10C41000024B1A6912681A61704700BF00040020BD
:10C42000C460056146618761C0F81C80C0F8209037
:10C43000C0F824A0C0F828B0C0F82CD080ED0C8B38
:10C4400080ED0E9B80ED10ABC0F808E0FFF7D8BF81
:10C45000104908B50B690BB916F0F8FE1A68586058
:10C460000A611846C468056946698769D0F81C8066
:10C47000D0F82090D0F824A0D0F828B0D0F82CD054
:10C4800090ED0C8B90ED0E9B90ED10ABD0F808E08A
:10C49000012070470004002010B50A460021044620
:10C4A00000F018FB18B914B1204608F07BFC10BD51
:10C4B0000A46002100F00EBB10B5002201210446FF
:10C4C00000F008FB18B914B1204608F06BFC10BD51
:10C4D000FFF7E2BF10B501220C4600F041FE18B98B
:10C4E00014B1204608F05EFC10BD00F039BE00F02B
:10C4F00031BC00002DE9F04300252B4C0326D4F875
:10C50000E0700021013143189A0803F00303BA5C7C
:10C510005B0042FA03F303F00303022BF2D009019C
:10C52000D4F8EC308A0803EB001011B300EB820260
:10C53000036819071AD1D4F8EC10994216D8D4F828
:10C54000F0709F4212D95B1AD4F8E0C048BF0F3395
:10C550001B114FEA930E03F003011CF80E804900F3
:10C5600048FA01F707F00307012F09D00430904281
:10C57000DED1B5B1013D04EB8503D3F8FC00BEE785
:10C5800006FA01F13F2D04EB850941EA08010CF898
:10C590000E1003D80135C9F8FC30E7E7C4F8F8708D
:10C5A000E4E7BDE8F08300BF000400200B461E4A0C
:10C5B000002123F00F0370B51C1A1C4D0646E40041
:10C5C000C5F8F030C5F8E000A2FB0424640AA3EB30
:10C5D000841326442246C5F8EC30C5E939463AF0C2
:10C5E000E7FA0021A200D5F8E80001240732D208BA
:10C5F0003AF0DEFA2022002105F500703AF0D8FA70
:10C60000D5F8E410D5F8EC300022481E85F8FE413C
:10C6100003EB8113A5F8FC21C5F82002C5F8F4301E
:10C62000C5F8242270BD00BFF32C23FA00040020BB
:10C63000034AB2F8FC310133A2F8FC31704700BF65
:10C6400000040020034AB2F8FC31013BA2F8FC319F
:10C65000704700BF00040020034BB3F8FC01003812
:10C6600018BF0120704700BF00040020F8B52F4C10
:10C6700000220327B4F8FC31251D04F1CC06C4F8D0
:10C68000F8200133A4F8FC3155F8040F02071AD141
:10C69000D4F8EC30984216D3D4F8F020904212D25D
:10C6A000C01AD4F8E01048BF0F3000114FEA900CC8
:10C6B00000F0030311F80CE05B004EFA03F202F005
:10C6C0000302012A1FD0AE42DED1D4F824020307B0
:10C6D00018D1D4F8EC30984214D3D4F8F02090421A
:10C6E00010D2C01AD4F8E04048BF0F3000118108C2
:10C6F00000F00303655C5B0045FA03F202F00302FD
:10C70000012A09D0F8BD07FA03F343EA0E0301F842
:10C710000C30FFF7EFFED6E7032202FA03F31D43C6
:10C720006554BDE8F840FFF7E5BE00BF00040020F7
:10C73000030730B419D1124BD3F8EC20904214D334
:10C74000D3F8F010884210D2801AD3F8E04048BFE6
:10C750000F300011810800F00303655C5B0045FAAF
:10C7600003F202F00302012A01D030BC7047032219
:10C7700002FA03F31D43655430BCFFF7BBBE00BF94
:10C7800000040020F8B529B3041F174E032704EB5B
:10C79000810554F8040F03071AD1D6F8EC309842FB
:10C7A00016D3D6F8F020904212D2C01AD6F8E01074
:10C7B00048BF0F3000114FEA900C00F0030311F84E
:10C7C0000CE05B004EFA03F202F00302012A02D0F1
:10C7D000A542DED1F8BD07FA03F343EA0E0301F8E0
:10C7E0000C30FFF787FEF3E7000400202DE9F04F3F
:10C7F0005D4E83B0D6F8F830D6F8E470002B00F028
:10C80000B0800025B900C6F8F850002943D00024B4
:10C81000A208D6F8E00004F00303825C5B0042FA51
:10C8200003F303F00303032B45D001348C42EFD311
:10C83000D6F8F830002BE6D169B34FF0000E4FF078
:10C8400003094FF0020A754604E0012B50D0013570
:10C850008D4220D2D6F8E0C04FEA950805F00304D7
:10C860001CF808200CEB9500640042FA04F303F076
:10C870000303022B2FD0032BE7D10AFA04F401356E
:10C880004FF0000E22EA04020CF80820D6F8E470FB
:10C89000B9008D42DED3202200213448013F3AF016
:10C8A00087F9B6F8FC31C6F82072013BA6F8FC31D6
:10C8B00003B0BDE8F08F20460134FFF71BFED6F829
:10C8C000E470B4EB870F4FEA8701A1D3D6F8F830B4
:10C8D000002B98D1B0E7BEF1000FB8D009FA04F4EC
:10C8E00022EA04020CF80820D6F8E470B900AEE79A
:10C8F000D6F8E830EF0805F0070BD95D03EBD50358
:10C9000041FA0BFC1CF0010F20D0D6F8EC002A01F4
:10C91000825800EB051062B16A460C2108F014FC45
:10C92000009810B1019909F0FFF8D6F8E820D31962
:10C93000D15D012202FA0BFB21EA0B0B83F800B058
:10C94000D6F8E03003EB080013F8082009FA04F4E5
:10C950004FF0010E22EA04020270D6F8E470B9002A
:10C9600075E7B90068E700BF00040020000600205A
:10C9700038B5074C0025B4F8FC31C4F8F850013341
:10C98000A4F8FC31FFF732FFC4F8EC5038BD00BF0B
:10C99000000400202DE9F04F4D4C0023D4E93B1258
:10C9A00043601E46521A036143619C4602601D4665
:10C9B000836199461F4619469E46C0E90233D4F862
:10C9C000E02092F800A04FEA4E0E4AFA0EFE0EF05A
:10C9D000030EBEF1010F65D0BEF1020F5ED0BEF1B5
:10C9E000000F54D0D4F8E420013392009A420CBFD7
:10C9F0004FF001084FF000082FD0D4F8E0204FEAA4
:10CA0000930A03F0030E12F80AA04FEA4E024AFA04
:10CA100002F212F0030214BFC3464FF0010BBBF148
:10CA2000000F43D1012ACED1D846964601291CD009
:10CA3000022902D1426901324261614501D98C4625
:10CA40008161BEF1000F14D14FEA9308D4F8E020C1
:10CA500003F0030E12F808A0B5E7BEF1010F14BFF2
:10CA6000C64648F0010E0129E2D102690132026195
:10CA7000E3E7B74201D93E46C760B8F1000F1BD0CB
:10CA80002D014FEA0913C0E90153BDE8F08F09F108
:10CA9000010901377146C0F80890A3E7013501315B
:10CAA00045609FE70135714645609BE7012A14BF49
:10CAB000C64648F0010EB9E74FEA930AD4F8E020E1
:10CAC000474603F0030ED04612F80AA07BE700BFEA
:10CAD000000400200F302DE9F04F070989B00791BD
:10CAE000059260D0DFF868B2DBF8EC30002B00F084
:10CAF0009B80BBF8FC31002B55D1DBF8EC204FF0CC
:10CB0000FF38DBF8F4309BF8FE119B1A059A81F090
:10CB1000010148BF0F33002A019115BF444601248B
:10CB20004FF0030A4FF0000A082F4FEA23193B4643
:10CB300028BF08237F330693069B059A5BF82330B2
:10CB40000493AABBDBF820229C461146DBF8E030B8
:10CB50000022CDF80C80032688460293C4454FD8A6
:10CB6000029B4FEA8C0E13F80C50019B002B4AD10C
:10CB70000AEB0E0053465900013206FA01F1294230
:10CB80001CD048454FF000021FD3012C1DD1DDF809
:10CB90000C80002297424BD9019B23B916F03AFB37
:10CBA00001230193C8E70023184609B0BDE8F08FC0
:10CBB000DBF820C26345EFD86146C7E797424FF0E4
:10CBC00001010CD803EB0E08E4E748452CBF002117
:10CBD0000121B4F1FF3F18BF002181F001011B19B1
:10CBE000204400F1AA80002900F0A780042BC2D1C4
:10CBF000A444049B63458CBF002101210029ADD1D1
:10CC0000DDF80C80C6E7534606E09742DAD91B19D7
:10CC100000F19280042BEBD05900013206FA01F1A9
:10CC20002942F2D00022F2E7082017F099FA60E7D3
:10CC3000059B9BBB08F10104072FA4EB020437D826
:10CC400007EB080307F17F0007F180014FEA930328
:10CC50004BF820304BF821302AD007F18101062F04
:10CC60004BF8213024D007F18201052F4BF82130F9
:10CC70001ED007F18301042F4BF8213018D007F1A3
:10CC80008401032F4BF8213012D007F18501012FC9
:10CC90004BF821300CD1CBF81C3209E008F1FF33FE
:10CCA00002EB080144469B0801F1FF38CBF8203223
:10CCB000012304F00300A508029E9840E118834078
:10CCC0002846755D884543EA050333540FD3022691
:10CCD00001F003038808DBF8E05001315B002F5CB2
:10CCE000884506FA03F343EA07032B54F0D2DBF836
:10CCF000EC502601059905EB041329B1DBF8F4107B
:10CD0000994288BFCBF8F43012011846002139F05F
:10CD10004FFF079A0346002A3FF446AF0022E1087E
:10CD200004F00704AA510122DBF8E80002FA04F437
:10CD3000425C2243425437E70199A444049B634573
:10CD40008CBF002101F0010100297FF407AF57E7F4
:10CD5000000400202DE9F0412B4C0746B4F8FC31CB
:10CD6000002B49D1002847D0D4F8EC10002945D039
:10CD70007F1A4FF0030CD4F8E8804FF0010248BF4F
:10CD80000F373F1127FA0CF007F00705BE083946A8
:10CD900018F80030AA4007EA0C0E354623EA0203D1
:10CDA00008F80030D4F8E000825D4FEA4E0301310C
:10CDB0000CFA03F301F0030E22EA03024FEA4E03DA
:10CDC00042558D08D4F8E000425D42FA03F303F0C7
:10CDD0000303022BE9D0C91B082928BF08217F3192
:10CDE00054F82130B342D4F8203288BF44F821608F
:10CDF000B34238BFC4F82062BDE8F081082017F0C4
:10CE0000AFF9D4F8EC10B3E70004002010F00F02E3
:10CE100010B41CD11849D1F8EC30984213D3D1F892
:10CE2000F040A0420FD2C31AD1F8E04048BF0F3300
:10CE30001B11990803F00300615C4000014101F0FF
:10CE40000301012908D010465DF8044B7047002209
:10CE50005DF8044B1046704701329918880801F0BC
:10CE60000301205C490040FA01F101F003010229AD
:10CE7000F2D01201E7E700BF000400202DE9F04FD7
:10CE8000B64E87B00546D6F8F43083421ED9030764
:10CE90001CD1D6F8EC10884218D3D6F8F03098425E
:10CEA00014D2431AD6F8E040002B9946B8BF03F1DC
:10CEB0000F094FEA29194FEA990209F00300A25C11
:10CEC0004000024102F00302012A03D0284607B0C5
:10CED000BDE8F08F4FF0000808F1010809EB0802E7
:10CEE000900802F00302205C520040FA02F202F0C5
:10CEF0000302022AF0D05FEA0818E7D0002BD6F828
:10CF0000E8204FEA1817B8BF7F33DB11D35C0193D9
:10CF1000B8F1000FDAD0002900F01A81B6F8FC3120
:10CF2000002BD3D1D6F8EC204FF0FF34D6F8F430F4
:10CF3000D6F820B29B1A3A4696F8FEC148BF0F3386
:10CF4000082F8CF0010C28BF08224FEA231A02F1A7
:10CF50007F03013A56F8233003929B4502931CD37A
:10CF6000D6F8E0300BF1010005940022DE461844AB
:10CF70006446049310F8013D4FEA8E01002C7ED1E7
:10CF800013F0C00F40F08A800132974200F28A808D
:10CF9000A44603235C18974210D9BCF1000F95D129
:10CFA00016F038F9039BD6F820B24FF0010C80330D
:10CFB00056F823309B450293D2D287E74FF0010EFB
:10CFC00004F1FF3C04F00300A7084FEA9C0C049B0B
:10CFD00000FA0EF02244C6F820C204EB0E0113F84A
:10CFE00007C0013A0EFA00F304988A4243EA0C03A0
:10CFF000C35511D34FF0020C01F003038808D6F893
:10D00000E07001315B0017F800E08A420CFA03F38C
:10D0100043EA0E033B54EFD2D6F8ECA02701D6F832
:10D02000F4100AEB04138B4201D2C6F8F430C4F1B9
:10D03000010C1846002109F007096244120139F079
:10D04000B7FD019A034642FA09F919F0010F0DD014
:10D050000022E10804F007044AF807200122D6F86C
:10D06000E80002FA04F4425C224342549D426BD829
:10D070002946424618461D4639F072FD26E713F050
:10D08000C00F53D10132974282D913F0300F18D11B
:10D090000132974216D8A44602237BE7CA1C924568
:10D0A0005AD8224613F0300F3BD101329742F2D9C1
:10D0B00013F00C0F27D10132974228D8A446012340
:10D0C00068E7002213F00C0F32D101329742F5D9F4
:10D0D00013F0030331D10132974212D92146029B4A
:10D0E0000EF1FF3E9C46F34534BF00230123F44577
:10D0F00088BF002313B100297FF43CAFA446059CF0
:10D1000049E7A44646E74A1C924525D8002213F079
:10D11000030314D08A454FF000028CBF0021012187
:10D12000DDE78A1C924517D80022C1E70022ACE750
:10D1300013F003034FF00002CDD00022CEE70132FE
:10D140009742DED90121CAE71846FFF703FEBDE684
:10D15000082017F005F8E1E6059C21E7000400200F
:10D160002DE9F04F064685B0002800F0E681002941
:10D1700000F0D282D24DB5F8FC31002B40F0928005
:10D18000D5F8ECC00F31D5F8E430B0EB0C084FEA1D
:10D1900011144FEA830948BF08F10F084FEA281815
:10D1A00008F10100B0EB830F80F0C282D5F8E0E017
:10D1B000012700234FEA900A00F003011EF80AA09D
:10D1C00049004AFA01F101F0030102294FD019B9CF
:10D1D0000133D919A1424BD3BC4200F0928066D3EF
:10D1E0003B44A34280F08681002A5BD04FEAD801FD
:10D1F000D5F8E8305B5C0393BCF1000F00F09B8234
:10D20000D5F8F430214695F8FEE1AA46B3EB0C03BD
:10D2100000928EF0010E48BF0F33082C754628BFD0
:10D2200008211B117F3199460191019B0021DAF8F9
:10D2300020B25AF823E0DAF8E0300EF1FF3C1A464B
:10D240000293734694449B45C0F033811CF8012F30
:10D2500090075BD0002D40F03581B9EB830F4FEA8A
:10D26000830100F23D8115F0D5FF009DDDE7013718
:10D27000013081459ED8AFE7002E40F053829900DF
:10D2800003310022894594BF002101210133BB42B3
:10D2900002D3002940F08081944240F26282002E45
:10D2A00000F00F820024204605B0BDE8F08F08EBA7
:10D2B000040E3C1B47444FF003097146BC4601F085
:10D2C00003038808D5F8E07001315B003A5C6145E2
:10D2D00009FA03F322EA03033B54F0D1082C4FEA86
:10D2E0009E0328BF08247F3455F82420B2EB9E0FFC
:10D2F000D5F8202288BF45F824309A4238BFC5F8B7
:10D3000020323446204605B0BDE8F08F481C8442E8
:10D3100000F2898055469B008346A3EB0B01072C46
:10D3200001F101092CD8E21804F17F0C04F180000E
:10D33000072C4FEA920245F82C2045F820201FD0F8
:10D3400004F18100062C45F8202019D004F1820058
:10D35000052C45F8202013D004F18300042C45F857
:10D3600020200DD004F18400032C45F8202007D0A4
:10D3700004F18500012C45F8202001D1C5F81C22BC
:10D38000012209F0030C4FEA9900029C0CFA02FCFE
:10D390000231245C02FA0CF2994242EA0402029C35
:10D3A000225411D84FF0020C01F003028808D5F87E
:10D3B000E0400131520014F800E099420CFA02F208
:10D3C00042EA0E022254EFD9D5F8ECA04FEA0B1234
:10D3D00000214FEA091B0AEB0914204639F0E8FB4B
:10D3E00008F00703039A1A411346DB070FD5002301
:10D3F0004FEAD90209F007094AF80B300123D5F8A2
:10D40000E81003FA09F98B5C49EA03038B543A01EB
:10D410003146204639F0A4FB3046FFF79BFC2046FE
:10D4200005B0BDE8F08F12F00C0F1BD1881C8442B0
:10D4300003D89B00554601336EE712F0300F1CD124
:10D440000130844203D89B005546023364E712F052
:10D45000C00F20D1411C8C421BD89B00554608466A
:10D46000033359E79DBB9900481C81457FF6FBAE0D
:10D4700012F0300F03D10120E3E75DBB9900881C57
:10D4800081457FF6F0AE12F0C00F06D101218C422B
:10D49000E3D9009A07E03DBB9900CA1C00219145E1
:10D4A00094BF002201220133734502D3002A7FF486
:10D4B000CAAE8C4240F25081002D7FF4F3AED2E62A
:10D4C0000004002012F00C0F01D10120AFE712F090
:10D4D000300FD0D012F0C00FD8D0009A0021E2E770
:10D4E00012F00C0FF1D0BFE701337345FFF4DAAE51
:10D4F0000021A8E608EB0702A044424511D24FF0F4
:10D50000020E02F003039108D5F8E00001325B003F
:10D5100010F801C042450EFA03F343EA0C034354EA
:10D52000EFD1E21B344606EB07100021120139F05F
:10D530003FFB204605B0BDE8F08F0F310C093FF4EA
:10D54000B1AE894DD5F8EC30002B00F00181B5F873
:10D55000FC31002B7FF4A6AED5F8F470A046D5F8C8
:10D56000EC3095F8FE61FF1A86F0010648BF0F37D0
:10D57000082C4FEA271728BF4FF00808B94608F1D2
:10D580007F0855F828700022D5F8E0C007F1FF3E6B
:10D590003B46D5F820A2E6449A45FFF47DAE1EF83E
:10D5A000010F81077ED0002E00F09D8010F00C0F3F
:10D5B00040F0A38001218C4260D89B0001330A46D1
:10D5C000981A072C00F101062CD8E11804F17F0EFF
:10D5D00004F18007072C4FEA910145F82E1045F819
:10D5E00027101FD004F18107062C45F8271019D009
:10D5F00004F18207052C45F8271013D004F18307A6
:10D60000042C45F827100DD004F18407032C45F8AD
:10D61000271007D004F18507012C45F8271001D108
:10D62000C5F81C12012106F00304B70802308C4033
:10D630001CF807E0984201FA04F141EA0E010CF8E7
:10D64000071011D84FF0020E00F003018408D5F83E
:10D65000E0700130490017F804C098420EFA01F159
:10D6600041EA0C013955EFD9D5F8EC4012010021FF
:10D6700004EB0614204639F09BFA14E610F0300F44
:10D6800023D101318C4202D89B00023397E710F07E
:10D69000C00F7FF4F1AD4A1C944222D89B00114682
:10D6A00003338CE7511C8C4201D89B0087E710F0B4
:10D6B0000C0F01D1911C7EE7FEB999004A1C9145DF
:10D6C00026D8012615F0A6FD5BE7DEB999008A1C75
:10D6D0009145F6D910F0C00F7FF4D2AD01229442EB
:10D6E000DCD90121D2E5B9EB830F4FEA8301E8D9F8
:10D6F00010F00C0F3FF45EAFE0E710F0300F01D1F7
:10D700000121BFE710F0C00FE8D001210022BDE5E4
:10D7100010F0300FDBD1F3E70091FFF71BFB00990E
:10D720000C46C0E50133BB42FFF4BCAD002233E739
:10D730000127002350E50820009216F011FDB5F8EE
:10D74000FC31009A002B7FF4ADADD5F8ECC057E565
:10D75000082016F005FDFAE68B4655464FF0FF33DC
:10D76000DBE54FF0FF332BE7000400202DE9F84FF5
:10D7700010F00F06044604D17E4DD5F8EC10884217
:10D7800002D20020BDE8F88FD5F8F0309842F8D2E8
:10D79000401AD5F8E0E048BF0F300011830800F0D0
:10D7A00003071EF803207F003A4102F00307012F10
:10D7B000E7D14FF0000C0CF1010C00EB0C039A08C0
:10D7C00003F003031EF802205B0042FA03F303F0A8
:10D7D0000303022BEFD05FEA0C13D2D0D5F824322A
:10D7E00033B911E09A685AB1DA685AB11B685BB173
:10D7F0005A68002AF6D1043301201C60BDE8F88F76
:10D800000833F9E70C33F7E7002900F09580B5F805
:10D81000FC31002BB5D1D5F8F430D5F8EC20D5F893
:10D8200000A29B1AD5F8209295F8FE0148BF0F334D
:10D83000D14580F001004FEA231870D3D5F8E0C03D
:10D8400009F101014FEA8902614401F1FF3E11F83B
:10D85000013CD0BB13F0C00F35D002F1030BD8450B
:10D8600060D813F0300F3ED002F1020BD84559D8E2
:10D8700013F00C0F07D002F1010BD84552D813F06A
:10D88000030F32D107463A440123501E02F0030130
:10D890009708994080088B40C5F820021CF80710B3
:10D8A0000B430CF80730531C4AD1022306F0030245
:10D8B000B108D5F8E00001365200445C03FA02F2E8
:10D8C00022434254F2E70327DDE713F0C00FFAD0FA
:10D8D00013F0300F07D013F00C0FD4D013F0030364
:10D8E0001BD11F46CFE70227CDE790458CBF002311
:10D8F00001230239043AA1EB0C01894534BF4FF0F2
:10D90000000B4FF0010B8A4588BF4FF0000BBBF1B5
:10D91000000F04D01BB1714697E70346E9E70028E2
:10D920007FF42FAF15F076FCD5F800A2D5F8209241
:10D930000120D14582D224E7082016F011FC66E7C9
:10D94000D5F8EC101001D5F8F43001EB02129A4230
:10D9500001D2C5F8F42000230B5053609360D360CC
:10D96000D5F8241209B11A60FFDEC5F8242201207F
:10D97000546007E70004002010B58AB00B4C03A8E0
:10D98000FFF708F8059A049B204600920849039A7D
:10D9900000F030FF069A099B20460649CDE9003287
:10D9A000DDE9072300F026FF0AB010BD3C9F0460AC
:10D9B000A86C0460CC6C046010B50446C068FFF726
:10D9C0005DFAE0602046BDE81040FFF757BA00005E
:10D9D000034610B470B304072CD1184AD2F8EC40B7
:10D9E000844227D8D2F8F020824223D982071CD162
:10D9F0000268134CA24203D15DF8044B00F07AB8E0
:10DA0000104CA24203D15DF8044B00F023B80E493C
:10DA10008A4202D00D498A4204D118465DF8044B6F
:10DA2000FFF7CABF0A498A4204D018465DF8044B82
:10DA3000FFF724BA18465DF8044B70470004002035
:10DA400088BF0460F0C7046018D404607CD104600F
:10DA5000F8D9046013B50446B1B101394068C9B2C0
:10DA60000191FFF7B5FF01996060A068FFF7B0FF73
:10DA70000199A060E068FFF7ABFFE060204602B0CC
:10DA8000BDE81040FFF7FAB902B010BDF8B50D4679
:10DA90000446D8B1D1B1164B984217D0037913F090
:10DAA0000A0613D1013D43F00803EDB20371C068CB
:10DAB000FFF7E4F9E060A3689E4209D32046FFF730
:10DAC000DDF9037904466FF3C30303712046F8BD03
:10DAD000E36803EBC60753F8363033B1042B04D0A8
:10DAE00029467868FFF774FF78600136E3E700BFE6
:10DAF0005C0400202DE9F8430D460446002861D05F
:10DB0000324B98425ED000295CD0013D80680026EF
:10DB1000FFF7B4F9EDB2A06060682946FFF7B6FFE1
:10DB20006060E068FFF772F9B6EB900F15D3E0681C
:10DB300004F11007FFF7A2F9E06020464FF000085B
:10DB4000FFF764F9DFF888908008061FB04527D3F7
:10DB50002046BDE8F843FFF791B9E3684FEA86082D
:10DB600053F82600FFF752F9C0B1E36853F8267066
:10DB70003B7803F00703022B07D17868FFF77EF9A3
:10DB80007860B868FFF77AF9B860E368294653F817
:10DB90000800FFF71DFFE36843F808000136C0E7FF
:10DBA000386840B18307294609D103684B4506D13F
:10DBB000FFF76CFF386008F101080437C6E7FFF78C
:10DBC00007FFF7E72046BDE8F88300BF74C804608C
:10DBD00084B70460054B5B695A68824204D8801A96
:10DBE000043053F8200070471B68F5E7000400205C
:10DBF000014441F20553884204D3D8B2012838BF0A
:10DC00000120704703EB431310F8012B5340F2E758
:10DC1000034B044A5A610022C3F8D020704700BF6A
:10DC2000000400202C5E05602DE9F84F80460D466B
:10DC3000FFF7DEFF134B07465C690CB920461EE078
:10DC400004F1100BE3685E460BEB83094E45B246C8
:10DC500001D32468F1E756F8040B0378BB42F5D1F1
:10DC60004378AB42F2D12A464146023038F06AFF8F
:10DC70000028EBD1AAEB0B0A606800EBAA00BDE814
:10DC8000F88F00BF000400202DE9F04780460E46C3
:10DC9000FFF7CAFF0246002875D1404CF51CD4F8A6
:10DCA000D00090B1D4E935132B448B422ED92944AE
:10DCB000FEF71BFC074600BB0246D4F8D810D4F888
:10DCC000D000FEF712FCC4F8D070802D2F464FF024
:10DCD000010138BF80273846FEF7EAFBC4F8D000C0
:10DCE000002854D101212846FEF7E2FBC4F8D000F9
:10DCF00000284BD1284607F055F8D4F8D4302B44EF
:10DD0000C4F8D430D4F8D030002BDED0D4F8D8907A
:10DD10003146D4F8D0A040464D440AEB0907C4F878
:10DD2000D850FFF765FF32460AF8090041467E7079
:10DD3000B81C38F015FFB91900268E706369D3E955
:10DD40000253AB4213D36D000121402D28BF402563
:10DD5000281D8000FEF7ACFB0028CBD06269026072
:10DD60005368D268C6601344C0E9013560616269D6
:10DD7000D368591C0433D16042F8237063695A6830
:10DD8000D8680244013A1046BDE8F0872F460023C8
:10DD9000C4F8D470C4F8D830B8E700BF000400203D
:10DDA00010B5044638F023FF01462046BDE8104078
:10DDB000FFF76ABF08B5FFF70DFF407808BD08B54B
:10DDC000FFF708FF023008BD08B5FFF703FF4378EF
:10DDD00002300B6008BD00002DE9F8431D4600230A
:10DDE00007468846036016460B6013602B60164B8F
:10DDF000DFF858905C690CB14C4505D12B6832684E
:10DE000013442B60BDE8F8833B6801333B60E26854
:10DE1000D8F800301344C8F8003004F11003E26869
:10DE200003EB8202934207D32046FEF7EFFF2B68F5
:10DE3000184428602468DEE753F8041B48783168EA
:10DE4000033101443160EDE7000400202C5E0560E1
:10DE500038B54468054603682144994211D9037BCB
:10DE6000DB0703D50021074806F089FF01F1100404
:10DE7000806824F0070408342146FEF72BFB2C6051
:10DE8000A86038BDDCBC046070B504460E4611467F
:10DE90001546FFF7DDFF31462A46D4E90130184424
:10DEA00038F06CFE62682A44626070BD70B54668E6
:10DEB0000446B14228BF31460D460121FFF7C8FF95
:10DEC000A368681C721B5919184438F057FE636820
:10DED000A06801332844636070BD012938B538BF9C
:10DEE0000121044600250846216065602946FEF7A9
:10DEF000D3FA237BA06065F30003237338BD38B5E4
:10DF00004B1C05460C4602D1084606F04BFF01317A
:10DF1000FFF7E3FF6C6038BD00230160C0E9013208
:10DF2000037B43F0010303737047000038B51446C8
:10DF30000546FFF7D2FF024B2560636038BD00BF86
:10DF400089DE006010B5037B0446DB0702D48068DD
:10DF5000FEF7CDFA0023A36010BD38B500210546B9
:10DF60001020FEF799FA04462946FFF7B6FF20462F
:10DF700038BD10B5044650B1037BDB0702D480687E
:10DF8000FEF7B5FA2046BDE81040FEF7B0BA10BD66
:10DF900038B5037B04460D46DB0703D5002107484F
:10DFA00006F0EDFE016880682944FEF793FA2368C5
:10DFB000A0601D441844256038BD00BFDCBC04606F
:10DFC00038B504460D46FFF743FFD4E901301D4440
:10DFD0001844656038BD10B5D0E9002304469A4264
:10DFE00002D10121FFF7D4FF0021D4E90132D1543D
:10DFF000A06810BD10B50C460121FFF7E1FF0470C9
:10E0000010BD7F29F8B50C46CEB204D80121FFF728
:10E01000D7FF0670F8BD06F03F06B1F5006FC1F3FB
:10E02000871546F0800607D265F03F050221FFF70D
:10E03000C7FF46700570EDE705F03F05B1F5803F7D
:10E04000C1F3073745F0800508D267F01F070321A9
:10E05000FFF7B6FF457007708670DBE7A40C07F08A
:10E060003F07042164F00F0467F07F07FFF7A8FF64
:10E07000857004704770C670CCE713B50446084637
:10E08000019138F0B4FD01990246204602B0BDE886
:10E090001040FFF7F9BE10B51446FFF707FF0470F4
:10E0A00010BD10B51446FFF701FF047010BD4368A2
:10E0B0008B422CBF591A00214160704738B5044685
:10E0C0001546084662688A4203D929448A4201D823
:10E0D000606038BDA368521A1844194438F04EFDE8
:10E0E0006268521B6260F4E7084611461EF0F2BBFC
:10E0F00037B505460846019138F079FD044620B150
:10E1000002466B68019928689847204603B030BDE5
:10E110002DE9F74F89469DF8301017460D9A11F0FA
:10E12000DF0F0646A2EB07023DD030290CA8254997
:10E1300013BF80464FF0100A88464FF0010A13F0D3
:10E14000800535D002EBD2746510A2EB6404002D7B
:10E1500035DDAB46DA45524673684146A8BF5A469C
:10E16000306801929847019AABEB020BBBF1000FAC
:10E17000F0DC2FB13D4473683A4649463068984711
:10E18000002C0CDD2544A245574673684146A8BFC4
:10E1900027463068E41B3A469847002CF3DC2846B3
:10E1A00003B0BDE8F08FDFF820804FF0100AC6E71B
:10E1B00013F0010401D11546C9E71446D9E700253B
:10E1C000D7E700BF559F0460449F04602DE9F043EA
:10E1D000064689B00020119D9DF84880139F8DF858
:10E1E0000F000AB381421ADA2D2249428DF80F201E
:10E1F000109A08AC0DF11009A2F10A008E46B1FB8D
:10E20000F3FC03FB1C126146092A8CBF1218303242
:10E2100004F8012D4C450ED07345EFD90BE0A8074B
:10E2200027D52B228DF80F200029E1D130230DF1C5
:10E230001F048DF81F3015F040099DF80F301CD0D9
:10E2400023B301222B460DF10F013046013FCDE9EA
:10E250000082FFF75DFF814608AA2B462146304623
:10E26000121BCDE90087FFF753FF484409B0BDE812
:10E27000F0836A07D8D52022D4E7002BECD004AA7B
:10E280009442E9D904F8013C013CE5E79946E3E70B
:10E290002DE9F04F93B081461D46C8079DF87430B4
:10E2A0000C4690461C9E0693DDE91E7A0BD4A1070E
:10E2B00003D122687A4B9A4205D0204607F0BEFF70
:10E2C000400040F0010416F0810306D1069A302A7E
:10E2D00003D15745B8BF57469A4620460DF1280B43
:10E2E0000AF042FE002818DBB20712D52B230DF1ED
:10E2F00029028DF82830F006EDB21DD5B8F1020FD5
:10E300000DD13021134603F8021B691C51701A46C7
:10E3100012E0730701D52023E9E75A46EBE7B8F18D
:10E32000080F61D1B1054FF03003137049BF05F1FB
:10E330000E03013253700232A2EB0B03002116F0E0
:10E34000200F11700EAA05930CBF0B462C23BAF1B7
:10E35000010F0B924FF01002C8BF46F040068DF837
:10E360002710CDE90C2116F04002CDE902530792A7
:10E3700044D023460DAA0BA8CDE900810CA90AF0D0
:10E38000E9FB037880462D2B06D18DF8273000F16C
:10E3900001080D9B013B0D93BAF1010F3CDD0D9D72
:10E3A000079B5545B8BF55462BB19DF8273003B1A3
:10E3B0000135059B1D44AF422BDD16F00103A7EB91
:10E3C000050527D12C461D4626F001064CB1202319
:10E3D000019434494846009300231A46FFF798FEFB
:10E3E00004463023069319E0B8F1100FA4D1302170
:10E3F000134603F8021B05F1170187E70AAB0DAAC4
:10E400000CA90BA8CDE9008323460AF0A3FB8046A4
:10E41000C2E700250024D7E700252C46079BDBB187
:10E420009DF8273053B1002301220DF12701484602
:10E43000013FCDE90032FFF76BFE0444059B5BB161
:10E440000023012259464846CDE90032059AFFF7DC
:10E450005FFE059B0444FF1A069BBAF1010FC8BF7B
:10E4600057460D9A41460093484633460197FFF7B9
:10E470004FFE04444DB120230A49484601950093BC
:10E4800000231A46FFF744FE04440B980EAB984253
:10E4900001D0FEF72CF8204613B0BDE8F08F00BF86
:10E4A0006CC30460F5C405602DE9F04316468BB0DB
:10E4B00007469846B207DDF848903DD416F0040FA1
:10E4C0000CBF002320230A4600932021139B02A89F
:10E4D00005F0A4FDF30504460DD5431C1F2B0AD8F7
:10E4E0000AAA00211444252204F8202C0AAA1C465A
:10E4F0001A4402F8201C16F040051FD09DF8083081
:10E500002F2B4FF000031BD8012202A9384609F136
:10E51000FF39013CCDE90032FFF7FAFD0DF10901A9
:10E520000546334622463846CDE90089FFF7F0FD1F
:10E5300028440BB0BDE8F0832B23C4E702A9F0E721
:10E5400002A91D46EDE700002DE9F04F814689B094
:10E55000144600260B461D4613F8012B82B9A9422A
:10E5600011D30B78002B00F03C81013120234FF0B8
:10E5700000080A4612F8015B7DB94FF00A0C2AE048
:10E58000252AE8D1EBE76F1AD9F80430D9F8000052
:10E590003A463E4498472946E3E72D2D03D148F0FB
:10E5A00001081146E5E72B2D02D148F00208F8E7F3
:10E5B000202D02D148F00408F3E7212D02D148F0C4
:10E5C0000808EEE7302D21D148F040082B46E8E757
:10E5D0000CFB0525303D0F4611F8012BA2F1300050
:10E5E0000928F5D92E2A41D17A782A2A10D000207C
:10E5F0004FF00A0C0F4611F801BBABF13002092AAB
:10E6000009D80CFB00BBABF13000F3E70025B4E701
:10E61000023754F8040B20EAE07B3A786C2A08BFF2
:10E62000013797F800A0BAF1000F00F0DA80BAF1D4
:10E63000780F6AD8BAF1570F1BD8BAF1470F61D8D3
:10E64000BAF1440F61D90734049324F00704F4E8C5
:10E65000020138F0ABF8049B00EE100A4246514626
:10E660004846CDE9005BFFF71FFF62E04FF0FF3B3C
:10E67000D3E7AAF15802202A47D801A151F822F085
:10E68000C1E700600BE700600BE700600BE700608C
:10E690000BE700600BE700600BE700600BE7006032
:10E6A0000BE700600BE700601DE700603FE70060DC
:10E6B000A5E7006047E6006047E6006047E60060C7
:10E6C0000BE700600BE700600BE700600BE7006002
:10E6D0000BE700600BE700600BE700600BE70060F2
:10E6E000D7E7006053E700600BE7006077E7006062
:10E6F0000BE7006093E700600BE700600BE700604A
:10E70000C1E70060BAF1500F65D0D9F8043001229A
:10E710003946D9F80000013698470BE054F8042B2D
:10E72000CDE9003543463AB1042230494846FFF767
:10E73000EFFC0644791C0DE705222D49F6E754F855
:10E74000042B07A98DF81C200122CDE90035434692
:10E75000ECE707A954F8040B0493FFF735FBBBF172
:10E76000FF3F0146049B01D1DDF81CB05A46CDE9BC
:10E7700000354346DAE7BBF1FF3F54F8041BF5D1FF
:10E7800008460593049138F032FA8346DDE9041314
:10E79000ECE7CDE902356123CDF8048000930A232C
:10E7A000002207E0CDE9023561230122CDF8048083
:10E7B00000930A2354F8041B4846FFF707FDB8E707
:10E7C000AAF1170ACDF80480CDE902355FFA8AF381
:10E7D00000931023E4E7CDE90235CDF804806123EE
:10E7E000F6E7304609B0BDE8F08F00BF309F046007
:10E7F000359F04600EB403B503AA52F8041B0192BE
:10E80000FFF7A2FE02B05DF804EB03B0704790F989
:10E81000001002460378002901DB1846704703F018
:10E820007F004023184206D112F8013F03F0C001D7
:10E83000802904D0704720EA03005B08F2E703F068
:10E840003F0343EA8010EFE7431C18460133027888
:10E8500002F0C002802AF8D0704703460020994297
:10E8600000D8704711F8012D02F0C002802A18BFAD
:10E870000130F4E701440346002099421A4600D8CB
:10E8800070471278013302F0C002802A18BF0130AD
:10E89000F3E700007F289DBF024B185CC0F34000E7
:10E8A00000207047669F04607F289DBF024B185C64
:10E8B000C0F3C00000207047669F04607F289DBFA2
:10E8C000024B185CC0F3800000207047669F046014
:10E8D0007F289DBF024B185CC0F38010002070475A
:10E8E000669F04607F2809D8064B1B5C13F00C0F51
:10E8F00006D1A0F15F03584258417047002070478D
:10E9000001207047669F04607F289DBF024B185C02
:10E91000C0F3001000207047669F04607F289DBFF1
:10E92000024B185CC0F3401000207047669F0460E3
:10E9300008B50246FFF7E8FF00B12032104608BDD7
:10E9400008B50246FFF7EAFF00B1203A104608BDBD
:10E950003038092884BF20F0200007387047014470
:10E960000246002010B5E524914203D8B0FA80F0A9
:10E97000400915E012F8013B20B11B0611D5431EDA
:10E98000D8B2F1E7BF2B09D9F72B09D8DB0803F080
:10E99000060344FA03F303F00300E5E71B06E3D59F
:10E9A00010BD0020FCE7023981420B4603D202333E
:10E9B000181A401070471A880239002AF4D0F6E776
:10E9C000B2EB131F70B54FEA131416D9121B03F0E4
:10E9D0000F0301EB440115460E46012D31F8024BA1
:10E9E00018BF3468013D24FA03F4A4B220F8024BA6
:10E9F000F2D104B9013A104670BD0022FBE7F0B530
:10EA0000059F0024D21B2646A74210D100EB470CDD
:10EA1000002401EB4701A24214D10CEB42031EB1CA
:10EA2000012102332CF81210181A4010F0BD31F8F1
:10EA3000145033F814C06544354420F814502E0C9B
:10EA40000134E1E731F8145035442CF814502E0C01
:10EA50000134E0E7F0B4049F0025D21B2C46AF42FE
:10EA60000BD100EB4706002301EB47059A420FD17B
:10EA700006EB4201F0BCFFF796BF31F81560344455
:10EA800033F81560A41B20F8154024140135E6E77F
:10EA900035F813100C4426F8134024140133E5E72D
:10EAA000022938B538BF0221044680680D4618B1E6
:10EAB0002368B1EB930F07D96900FDF70BFD2368BD
:10EAC000A06065F39F03236038BD38B5054600217B
:10EAD0000C20FDF7E1FC2A780378044602F00102DD
:10EAE000002123F003031343037028682368C0F355
:10EAF0009D0060F39F03400023606B686360FDF737
:10EB0000CBFCA0602A68A968C2F39D02520038F0CD
:10EB100027F8204638BD00EB410002EB410210B55A
:10EB200009B9084610BD30F8023D32F8024D1B1BF2
:10EB3000002B02DB04D10139F2E74FF0FF30F1E79F
:10EB40000120EFE710B5044638B18068FDF7CFFC2F
:10EB50002046BDE81040FDF7CABC10BD38B50C46D4
:10EB600002210546FFF79CFF002C2B78B5BF012240
:10EB700000226142214662F300032B7000236B6088
:10EB8000D5E90132581C686022F81310090CF7D13E
:10EB900038BD0023C0E900338360704728B1037893
:10EBA0009B0702D48068FDF7A2BC704738B50446C5
:10EBB0000D464968FFF774FF2A782378A06862F34E
:10EBC000000323706A6862605200A968BDE838409B
:10EBD00037F0C6BF09B941607047FFF7BFBF08B53E
:10EBE000FFF7D7FFBDE80840FFF7F4BF920042F0FF
:10EBF00002020260002210B4C0E901215DF8044B5A
:10EC00001946FFF7E7BFF8B59DF8187004210646CE
:10EC100014461D46FFF744FF87B1002C75F1000331
:10EC20000CDA624265EB4503317867F3000131701D
:10EC30000021716052EA030104D1F8BD22462B463F
:10EC40000027F1E7D6E901104C1C746020F8112070
:10EC5000110C180C41EA034103460A46EAE72DE984
:10EC6000F3418DED010A0746019C0378E20F62F340
:10EC700000030370C4F30F4313F4FF4304D10023D4
:10EC80007B6002B0BDE8F081B3F5FF4FF7D0C4F36D
:10EC9000C753A3F17F05002DF1DB05D1012102B09F
:10ECA000BDE8F041FFF75ABFB3F16F08C4F3160493
:10ECB00048BFA3F16008162D44F400044FEA281859
:10ECC00021DCC5F11705EC4000252E4641463846AB
:10ECD000FFF7E6FEC7F8048026B172000021B8688D
:10ECE00037F066FF45B104FA05F2C5F11005BB68BF
:10ECF000EC4023F816200136B045C2D0BB6823F89B
:10ED00001640240CF7E7B3F1960605F1090548BF54
:10ED1000A3F1870605F00F053611D7E72DE9F84373
:10ED20008F18C2F35B0204460D46511C9846089E9C
:10ED3000FFF7B6FE237829461FFA86FC68F3000326
:10ED4000237000236360B942084602D3401BBDE82C
:10ED5000F88302780131A2F13003092B05D9A2F121
:10ED60004103192B14D8A2F13703B342EED2D4E9F0
:10ED700001E0F0468146B8F1000F10D100EB4E02E1
:10ED800013B1023220F81E30121A52106260DAE714
:10ED9000A2F16103192BD9D8A2F15703E5E7B9F81D
:10EDA000002008F1FF3802FB0C3329F8023B1B0C52
:10EDB000E1E7F8B5044615461E46C1B1531E4FF0B3
:10EDC000FF371E44E90020460F310909FFF768FEAE
:10EDD000237800216FF30003616023704DB9D4E9FB
:10EDE000011000EB4101FFF7DEFD6060F8BD012777
:10EDF000E8E700230F290ADC3278013D3E4402FA9D
:10EE000001F201F1080143EA02039BB2F2D1626808
:10EE10001039501C6060A06820F81230DEE770B531
:10EE2000456804460DB9486898B10B78267803F018
:10EE3000010306F00100181A0BD14B689D4209D35B
:10EE40000BD88A682946A068FFF765FEF30748BF1C
:10EE5000404270BD4FF0FF30F8E70120F6E78842EE
:10EE600010B5044601D0FFF7A1FE23786FF300032D
:10EE7000237010BD884210B5044601D0FFF796FEFE
:10EE80002378C3F30002C2F1010262F3000323708E
:10EE900010BD88421FB5044601D0FFF787FE6268A7
:10EEA00062B901212046FFF7FBFD0123A268138010
:10EEB0006360237843F00103237010E02378D907BF
:10EEC0000FD56FF30003A168237001230846ADF846
:10EED0000E3000930DF10E03FFF7BCFD606004B02F
:10EEE00010BD511C2046FFF7DBFD0123D4E90121B1
:10EEF000ADF80E30009308460DF10E03FFF77FFDCD
:10EF00006060D6E72DE9F8434B6805460E46144687
:10EF100003B12AB931462846BDE8F843FFF746BE9B
:10EF200002F10F014FEA111803EB1111FFF7B8FDC1
:10EF300014F00F04AB6808BF1024D6E90102C4F135
:10EF4000100408EB000702EB400E002207F100411D
:10EF5000013903EB41030146994601BB6FF0010CF7
:10EF600022FA04F408F1FF320CFB00FC520003EB20
:10EF70000C0023F80C40C8F1010300EB43031846D2
:10EF800037F016FE831E17B133F8172092B12B7895
:10EF90006F60327862F300032B70BDE8F8833EF8AF
:10EFA00002CD01394CEA020222FA04FC120429F8CB
:10EFB00002C9D2E7013FE6E7F0B50E46496885B0E1
:10EFC0000546144601B12AB931462846FFF7EEFD41
:10EFD00005B0F0BDFFF764FD2346A868D6E901211E
:10EFE000FFF7EEFC2B786860327862F300032B7039
:10EFF000DB07EDD5002322097168ADF80E30994288
:10F0000001D093420FD19142E2D9B36804F00F04CA
:10F0100033F81220012303FA04F4013C224213D0F6
:10F02000ADF80E3008E0B76837F8137057B1012318
:10F030009142ADF80E30E8D8A968012348B90B8099
:10F040006B60C5E70133DAE7BDF80E30002BBFD0A7
:10F05000F2E70246009308460DF10E03FFF7CFFCDE
:10F060006860B5E773B50C465368496806461546AF
:10F07000994206D308D89268A068FFF74CFD002893
:10F0800002DA23462C461D4623782A7861685340CD
:10F09000DB0713D401313046FFF702FD6B68B0681F
:10F0A0000093AB68D4E90121FFF7A9FC33787060C5
:10F0B000227862F30003337002B070BD3046FFF770
:10F0C000EFFC6B68B0680093AB68D4E90121FFF7EF
:10F0D000C1FCEBE7F7B50C46536849680646154690
:10F0E000994206D328D89268A068FFF714FD00283B
:10F0F00022DA234601272C461D4623782A786168A8
:10F100005340DB071AD501313046FFF7C9FC6B6865
:10F11000B0680093AB68D4E90121FFF770FC706020
:10F12000237803F001030FB183F00103327863F316
:10F130000002327003B0F0BD0027DEE73046FFF773
:10F14000AFFC6B68B0680093AB68D4E90121FFF7AE
:10F1500081FCE4E72DE9F04F15464A680C4685B07E
:10F160006B6806469A423EBF2C460B461D462378E6
:10F170006168DB0756BF2B78012303F001031944B4
:10F18000FFF78EFCAB6894F8009000932B78B06882
:10F1900089EA030C696803F0010E43F300031CF0D5
:10F1A000010F09F0010C9BB20CBF09F0010B4FF0ED
:10F1B000000B49F30009CBF1000A1FFA8AF28246DC
:10F1C000D4E9018701921FFA89F2A7F102094746A3
:10F1D0000292A1EB08020392CFB900EB4801BBF108
:10F1E000000F03D00123023120F81830FFF7DBFBBA
:10F1F000706023782A78C3F30003C2F3000213403F
:10F20000327863F30002327005B0BDE8F08F39F850
:10F21000021F013F029A5140039A8C44D1198F4238
:10F2200029BF009A194632F8021B594028BF0092A4
:10F23000019A8E440CEA0E014FEA1E4E4FEA1C4C16
:10F2400051401BFA81F14FEA114B2AF8021BC3E728
:10F250002DE9F04F14464A680D4685B063680646AE
:10F260009A423EBF25460B461C462B786968DB0751
:10F2700056BF2378012303F001031944FFF710FC64
:10F2800095F80080A36818F0010F2278009308F029
:10F29000010C0CBF2378012348F30008B06808BFB5
:10F2A00003F00103D4F804B002F0010E42F30002AF
:10F2B000C3F1000A92B21FFA8AF78246D5E901919A
:10F2C00001971FFA88F7A1F1020849460297ABEBB4
:10F2D0000907039791B900EB4901FFF764FB7060E0
:10F2E0002B782278C3F30003C2F300021343327871
:10F2F00063F30002327005B0BDE8F08F38F802BF4A
:10F300000139029F8BEA070B039FDC4407EB010BDB
:10F31000594529BF009F934637F802BB8BEA020B81
:10F3200028BF0097019FDE444CEA0E0B4FEA1E4EA9
:10F330004FEA1C4C8BEA070B13FA8BF32AF8023BBB
:10F340001B0CC7E72DE9F74F15464A680C460646E1
:10F350006B684FF6FF7B9A423EBF2C460B461D461C
:10F3600023786168DB0756BF2B78012303F0010384
:10F370001944FFF795FB23782A78A16883EA020CE9
:10F38000D4F80480B068DB43D243A1F1020A696873
:10F390000CF0010CAF6803F00103A1EB080102F0CF
:10F3A0000102C64681460191BEF1000F19D100EB62
:10F3B0004801BCF1000F03D00123023120F81830BE
:10F3C000FFF7F1FA706023782A78C3F30003C2F3E1
:10F3D00000025340327863F30002327003B0BDE89C
:10F3E000F08F3AF8021F0EF1FF3E59440B44019989
:10F3F00071448E452ABF37F8021B4FF6FF715944FE
:10F400000A4483EA0201120C1B0C1CFA81FC29F845
:10F4100002CB4FEA1C4CC7E72DE9F04F4B6885B093
:10F4200006460D4614460BB1536823B9002373609A
:10F4300005B0BDE8F08F81422ED1FFF746FBB44204
:10F440000546074600D1044663683046696819449A
:10F45000FFF726FB32680021B068C2F39D0252001C
:10F4600037F0A6FBAB68D6F808E00022D5F804A078
:10F470000193F446A3680EEB4A08114602936368B1
:10F480000393039B934231D0ACF10200DDF804B04A
:10F490000023CDF800A018E0824204D1FFF715FB4D
:10F4A00004460746D0E70027CEE730F8029F99448C
:10F4B0003BF8023B1946029B33F8123003FB0193E1
:10F4C0000099038001391B0C009100990029ECD1AF
:10F4D0004146881C13B10146A8F80030A1EB0E018B
:10F4E0000CF1020C013280464910CAE771603846BF
:10F4F00022782B785340327863F30002327005B0E3
:10F50000BDE8F04FFFF71EBB70B54B6806461446CA
:10F5100013B11378DA0702D50023736070BD6368F6
:10F5200023B90121BDE87040FFF718BB0846FFF77B
:10F53000CCFA05462046FFF7C8FA012104463046BA
:10F54000FFF70CFB636883B1A3681B88DB0704D556
:10F550002A4631463046FFF75FFF0123D4E90121F7
:10F560000846FFF72DFA606038B92846FFF7EAFA37
:10F570002046BDE87040FFF7E5BA2A4629462846EE
:10F58000FFF74AFFDEE72DE9F04F0C4651681746BA
:10F590008DB0013198460546FFF782FA7A6800215E
:10F5A000A8680132520037F003FB002320466B604D
:10F5B00079680131FFF774FA39462046FFF7F6FA09
:10F5C000D8F80430D4F804A00093534530D8AB6881
:10F5D000A668D8F8089001932CD34A465146304685
:10F5E000FFF799FA10BB0123019A606013806B60EA
:10F5F0003B7898F800205340DB0714D52B7843F074
:10F6000001032B70636873B14FF0FF3109A8FFF756
:10F61000E6FA09AA29462846FFF724FD4246214674
:10F620002046FFF71FFD0DB0BDE8F08F013001D17E
:10F630000023DCE7009B002103F10043013B4FEA7C
:10F64000430E39F8132012F4004F01F1010051D09C
:10F65000002289B2B44626F81A20C1F1100A606867
:10F6600001306060606806EB400BDC4546D339F83A
:10F6700013308B400293009B012B09D909EB0E0339
:10F68000C1F1100233F8023CD340029A1A430292AD
:10F690006FF0004C009B00EB0C02C01A019B6860ED
:10F6A000604406EB420203EB400303930EF10203B6
:10F6B0000793A9F10203069363680098984229D33F
:10F6C00003F100434FF0000CC1F1100E013B06EBBB
:10F6D00043039E4240F283806FF000416B6833B178
:10F6E0005A18019830F81220002A00F084806FF038
:10F6F000004185E05200014692B2A4E7BCF8000048
:10F7000000FA01FB4BEA02022CF8022B20FA0AF263
:10F7100092B2A7E7138832F802BC4BEA034B029B74
:10F72000BBFBF3FB079BD31A0493069BDDF81090F9
:10F73000059300239A464A450CD810881B1A002BC3
:10F7400046D1039B023A23F802B903936368013B55
:10F750006360B1E70598B9F800E030F802CF059092
:10F760000CFA01F040EA1A4A1FFA8AF00BFB00F08B
:10F77000704503D2AEEB000C9C450FD81844A0EBAB
:10F780000E03AEEB00001FFA80FC98B2003818BFE1
:10F79000012000EB134329F802CBCCE7ACEB030CC0
:10F7A00000231FFA8CFCF6E73AF802EF0EFA01FE8E
:10F7B0004EEA1949BCF800E010FA89F070442CF8C0
:10F7C000020B000C6245EFD81B1A0BF1FF3BB6E7AA
:10F7D0000020DDF818A0DDF810C08146F2E71A8895
:10F7E00042FA01F002FA0EF240EA0C001FFA82FC23
:10F7F00023F802096DE7013B6B606FE7013B636033
:10F800006368002B3FF4F4AE5A1836F81220002A31
:10F81000F4D0EDE610B5D0E901210346002001EB5C
:10F820004202914204D31B78DB0748BF404210BD1F
:10F8300032F8024D44EA0040F3E730B5D0E9012444
:10F84000002304EB4202944206D302780120D2073F
:10F8500048BF5B420B6030BDB3F5004F04D232F8B5
:10F86000025D45EA0343EEE70020F4E72DE9F043AB
:10F8700071B19F1800254FF0010E1A44AC46D0E933
:10F880000194A4F10208B9F1000F03D1BDE8F0839F
:10F890001F46EFE738F8024F0CF1100C44EA05451B
:10F8A000BCF1070F02DC09F1FF39ECE70678ACB2D6
:10F8B000F60741BFE4435EFA84FE1FFA8EF4CEF3EE
:10F8C000072EE4B249B17E1E07F8014CB342DDD0E9
:10F8D000ACF1080C2D0A3746E2E73E4606F8014B2C
:10F8E0009642F4E7D0E901329FED0C0A02EB4303A4
:10F8F0009FED0B7A9A4205D30378DB0748BFB1EE40
:10F90000400A704733F8021D07EE901AF8EEE77AC6
:10F91000E0EE077AB0EE670AECE700BF00000000F7
:10F92000000080472DE9F84F446881468A46154615
:10F930001E469DF828B00B9F9CB982B1551E3B46D0
:10F9400015F8011F184639B930230370002300F859
:10F95000013FC01BBDE8F88F03F8011BF0E73846F4
:10F96000F2E7640000212046FCF796FD804622461F
:10F97000D9F8081037F0F4F83846394608EB040295
:10F98000A6F13A03A2F1020C0026E045644639D9FB
:10F9900030360C46392E88BFF61804F8016B4646FF
:10F9A000B242B44638D8BBF1000F0AD00126A4EB0E
:10F9B000000CBCF1030F02BF8C1C81F801B0204683
:10F9C000F6B14046FCF793FD5DB1284637F00FF9DC
:10F9D0002A18611E1346AB4229D8954288BF0020E1
:10F9E000044499F80030DB0744BF2D2304F8013BA1
:10F9F0003B46621E9A421FD80023E01B2370A9E7F2
:10FA00002146BFE7248844EA0646B6FBFAF40AFB1F
:10FA100014662CF80249B8E7BCF800C00236BCF105
:10FA2000000FBDD0BBF1000FEAD00026BFE713F8EE
:10FA3000016D01F8016FCEE71978107803F8010B1A
:10FA400002F80119D6E7D0E9023293423DBF5A1CB1
:10FA5000826018784FF0FF30704710B50368044695
:10FA600013B14068FCF743FD2046BDE81040FCF7A9
:10FA70003EBD0000F8B50C461F461646054600215F
:10FA80001020FCF709FD054B8460C0E90074344484
:10FA9000C4606B60024B2860AB60F8BD47FA006041
:10FAA0005BFA00600369272B2BD0222B29D0A3F10E
:10FAB000620113291ED8174ACA40D2071AD54269D3
:10FAC000272A1ED0222A1CD0722B1CD1662A06D1CE
:10FAD0008269272A15D0222A13D0722B15D14369A7
:10FAE000622B0CD1806927280BD0A0F12203584249
:10FAF00058417047662BF0D14269722AE8D0002045
:10FB0000704701207047662BF6D0622BF7D143690E
:10FB1000722BE6E71100090010B5026904460A2AB3
:10FB200040D1836A013383620123E3626369236105
:10FB3000A369636194F87030002B3BD0B4F8723045
:10FB4000626E93421BBF591CA26E0023A4F8721070
:10FB500018BFD35CA36163690D2B08D10A22A36986
:10FB60009342626103D1D4E901039847A061A3697C
:10FB7000013306D163695A1C03D00A2B1CBF0A2328
:10FB8000A36194F8703063B1236953B9E26984F8D2
:10FB900070302261226A63666261626AA4F8723020
:10FBA000A26110BDC36A092A04BF073323F007030B
:10FBB0000133BAE7D4E901039847A061CBE770B5F8
:10FBC00004460D4600262069431C01D1304670BD15
:10FBD0000A2808D115B1636B002BF7D02046012607
:10FBE000FFF79AFFEFE7FEF755FE18B12046FFF743
:10FBF00093FFE8E72369232B08D12046FFF78CFF0A
:10FC000023695A1CDFD00A2BF7D1DCE75C2BDDD14E
:10FC100063690A2BDAD12046FFF77EFFE6E7000092
:10FC20002DE9F04F436E87B00446CBB190F87030A9
:10FC3000B3B929216030FEF7E4F9012384F870306C
:10FC40002369E36163692362A3696362A36E1A781F
:10FC500022615A7862619B78A3610323A4F8723011
:10FC6000002120466165FFF7AAFFA36A256B636444
:10FC7000002DE36AA36407DA0C23013584F84C30C5
:10FC8000256307B0BDE8F08F04D00B23013D84F855
:10FC90004C30F5E7002834D0626B92BB0A225D1E1F
:10FCA0006FF0004384F84C20D4E90F20D11830F8CD
:10FCB00011108D42E5D019D9A16B8A4207D30831C2
:10FCC0004900FCF707FCA36B20640833A363D4E965
:10FCD0000F32591CE16322F81350236B0133236365
:10FCE000CFE7013AE263226B013A2263E26BD1185B
:10FCF00030F811108D42F4D3C3D0022384F84C3075
:10FD0000BFE72669721C01D10023F7E72046FFF701
:10FD1000C9FE0746002800F0BA81002384F84C3061
:10FD2000CDE900332369752B00F0CB82622B0DD116
:10FD30006369722B0DBFB9464FF0000901260226F8
:10FD40001123009A002A9CD1019717E0722B08D149
:10FD50006369622B00F0BA82662B40F0BA820923F5
:10FD6000CCE7662B40F0B9826369722BF7D0019B18
:10FD7000002B86D1994601261023009794F84C2039
:10FD8000002A3AD184F84C303EB12046FFF7C4FE39
:10FD9000022E02D12046FFF7BFFE23692046222B08
:10FDA00014BF4FF0270B4FF0220BFFF7B5FE23696E
:10FDB0005B4525D163699B4522D120464FF0030A5C
:10FDC000FFF7AAFE2046FFF7A7FE4FF0000804F158
:10FDD0005006029743462169481C00F05281BAF14F
:10FDE000010F02D10A2900F04C8153450BD319466B
:10FDF00004F15000FEF75BF947E09A42C4D040E7B7
:10FE00004FF0010AE1E78B450DD1013359463046E9
:10FE1000CDE90333FEF7F5F8039B20460393FFF784
:10FE20007BFE039BD7E7009B3BB37B2912D1304677
:10FE300088F00108FEF7E5F8636E23B9B84904F1CC
:10FE40006000FEF71AF92046FFF766FECDF808803D
:10FE50000023C0E77D2910D13046FEF7D2F8B8F173
:10FE6000000F04D02C2104F16000FEF7CAF82046F0
:10FE70004FF00008FFF750FEEAE7B8F1000F25D079
:10FE800023290DD1052384F84C3001212046FFF7AA
:10FE900096FE2046FFF706FE00287FF443AFF0E60B
:10FEA0005C2901D10423EEE73A2909D0029B3BB13A
:10FEB00004F16000FEF7A5F82046FFF72DFEC7E726
:10FEC0003046FEF79EF800230293F5E75C2940F0E8
:10FED000D38020460391FFF71FFE23690399B9F1F0
:10FEE000000F06D003933046FEF78BF8039B1946AC
:10FEF0009DE0782B06D85B2B0BD8222B76D053D8DD
:10FF00000A2B4FD0A3F13001072900F2AE80032362
:10FF1000A4E0A3F15C021C2AF4D801A151F822F05C
:10FF2000EDFF006005FF006005FF006005FF006059
:10FF300005FF006095FF0060C5FF006005FF0060E1
:10FF400005FF006005FF0060D5FF006005FF006051
:10FF500005FF006005FF006005FF006005FF006011
:10FF600005FF006005FF0060CDFF006005FF006039
:10FF700005FF006005FF0060C1FF006005FF006035
:10FF8000C9FF0060D9FF0060D1FF006005FF00607D
:10FF900043000160072194F84C30102B68D13046A3
:10FFA000FEF72FF8002338E7552B15D0AAD8272BBA
:10FFB0001CD04E2BA6D15B4814F066FA05F08EFDDE
:10FFC0000D21E8E70821E6E70921E4E70A21E2E755
:10FFD0000B21E0E70C21DEE794F84C20112A07D131
:10FFE0005C2130460393FEF70CF8039B1946D2E7D9
:10FFF000752B0CBF04230823002116E0204605932F
:02000004600199
:100000000391FFF789FD226910460492FEF760FC18
:10001000002800F050810399049A090110460391C9
:10002000FEF796FC0399059B0144013BE6D24B1C6D
:10003000B8D0B1F5881FAED34FF0010384F84C302F
:10004000B0E70223D8E72046CDE90313FFF764FDAC
:1000500022690399303A049B02EBC1016269303A8C
:10006000072AE4D8013BEED1E1E75C2103933AE7AC
:10007000FF29E1D8112BDFD1C9B23046FDF7BAFF15
:1000800090E753453CBF032284F84C20AFE630464E
:10009000FEF70AFC064620691EB95F2801D07F28BA
:1000A00046D90D2304F15005C1B284F84C302846DE
:1000B000FDF7A0FF2046FFF72FFD2069421C1BD152
:1000C0002846194FFDF787FF0025064657F8041B01
:1000D000304636F082FD00281CD11335EDB2162DC6
:1000E00084F84C507FF4CDAD104BD3F8DC30002BAE
:1000F0000CBF1523132301E6FEF7D6FB40B9206998
:100100005F2805D07F2803D8FEF7D8FB0028D7D07A
:10011000217CCCE7FFF6B5AD0135222DD6D1B0E577
:1001200027A0046030A00460E8A004600004002060
:10013000FEF7C4FB68B321692E2935D10F2384F85B
:100140004C3004F150050F272846FDF75AFF204692
:10015000FFF7E2FC2069431C3FF493AD002E35D13C
:1001600020F02003452B31D16521284684F84C70BE
:10017000FDF747FF2046FFF7CFFC21692B2901D06F
:100180002D29E7D12846FDF73CFF2046FFF7C4FCA8
:10019000E0E723692E2B04D16069FEF78FFB00286E
:1001A000C9D100264E4D31E00E23302984F84C3061
:1001B000C7D1636943F02003623B162B9EBF494DB4
:1001C000DD4005F0010505F00106BAE7FEF76CFB1E
:1001D00028B121692E290DD184F84C70D2E720690D
:1001E000FEF76CFB0028F4D123692E2BF1D05F2B96
:1001F000CBD046E521F020034A2BC3D1ECE7652F95
:1002000001D0632F00D10135013601352F7817B1A8
:100210002369BB42F3D12046FFF77EFC0FB90123CF
:100220006CE5212F07D123693D2BF8D12046FFF73C
:1002300073FC472362E52E2F0FD123692E2B02D1A9
:1002400063692E2B01D0502358E52046FFF764FC4C
:100250002046FFF761FC122350E50335334615F8BD
:10026000027C632F0FD0652F0DD01F4AD35C03F0A3
:10027000FD0284F84C30482A01D04C2B13D1636B1B
:1002800001336363FDE415F8012C013621699142C5
:1002900007D12046FFF740FC3346652FE5D00235F5
:1002A000DDE7632FFAE7492A02D04D2B7FF4E9AC52
:1002B000636B013BE5E74FF00103014684F84C30E6
:1002C00069E6012610234FF000093AE5B9460226F7
:1002D00036E5B9460126102333E52E46F2E700BF86
:1002E000E69F046001204000BCA004607FB501AD22
:1002F0000646742085E80E000021FCF7CDF8044680
:10030000034695E8070043F8046B002583E80700DF
:1003100001236FF0010229461420C4E90A320A229F
:10032000C4E90C55C4E90E23FCF7B6F8202120647B
:1003300004F15000FDF7D1FD294604F16000FDF7FE
:10034000CCFD236C20461D802561C4E90555FFF7CF
:10035000E3FB2046FFF7E0FB2046FFF7DDFB2046EE
:10036000FFF75EFCA36C2046012B1CBF0B2384F817
:100370004C3004B070BD30B585B0054601AC2046A8
:10038000FFF778FB284694E80E00FFF7AFFF05B0B3
:1003900030BD30B585B00546014601AC204611F0B0
:1003A00055FF2846FDF7FCFC94E80E00FFF79EFF82
:1003B00005B030BD10B5044670B1C36840689847B9
:1003C00004F15000FDF7BEFD206CFCF790F82046CC
:1003D000BDE81040FCF78BB810BDD0E90432013BFA
:1003E000036152F8230070470369C9431944436904
:1003F00053F82100704738B5D0E9033204460D4662
:100400009A4208D3103340699900FCF763F8E36817
:1004100060611033E360D4E90432591C216142F871
:10042000235038BDF8B504461D460F461646D0E9A0
:100430000003834208D31030C100A068FCF74AF8DB
:100440002368A06010332360D4E90103421C62607A
:1004500003EBC00253F8301067F3170143F8301074
:10046000D6705560F8BD10B48469CAB20023616CBF
:100470005DF8044BFFF7D6BFF8B5446A06460D4653
:10048000B4B1D4E900030B44834224D908310022DB
:1004900001442046FCF729F80246C8B961682046A5
:1004A0000831FCF722F863682360336A63603462C2
:1004B000102D2F464FF0000138BF102707F108001C
:1004C000FBF7EAFF0023076004464360706202E026
:1004D00023682B44236060680834054444F8045CB6
:1004E0002044F8BDF7B5866905460F4696F84C30AE
:1004F0000D2B27D1716DFF2906D9354813F0C4FFA4
:100500000146344804F03BFCB06DFDF7BDFB8A2F7B
:1005100004460ED1C100002205F1280041F0060179
:1005200036F086FB28B14468E3071FD544F001018B
:1005300002E0210141F00201284603B0BDE8F0408D
:10054000FFF759BF0E2B07D133460022D6E915100D
:1005500003F0C4FF0446E7E70F2B13D100960023F6
:100560000122D6E9151004F03BF804460C21284678
:10057000766CFFF781FF40F2371301460660C0E951
:100580000134D9E7A3F11002012A1CD8D6E91510CD
:100590000A290BD8FDF778FB96F84C3048B1102BA0
:1005A0000CBF06230A2343EA0011C5E7FDF73CFB15
:1005B000F2E7094C0948D6E91521102B08BF20465F
:1005C0000AF0D7FCD1E7190141F00E01B4E700BFF2
:1005D00070A1046054BD046018D404607CD1046030
:1005E000B0F59F7F07D010F0010306D043080CBF81
:1005F0000120002070470120704718467047B0F571
:10060000AF7F07D010F0010306D0430814BF0120CC
:1006100000207047012070471846704710F0010213
:1006200004D040F00100086001207047A8B110F02C
:1006300003030FD10279372A0ED1836813F001002A
:100640000B60F1D19A0708D11868044BC31A5842BD
:100650005841704710467047184670476CC3046095
:100660002A2A2DE9F04F044685B0884616461D46D5
:100670000BD10021FFF7B8FE98B3810702D10379AF
:100680008C2B2ED005B0BDE8F08FA2F11C03012BFE
:1006900056D8A9462F460AE01C2E44D1FFF7AFFFDB
:1006A000C8B91046FFF79CFF002808BF574607F15E
:1006B000FF3AB9F1000F0ED009F1FF392046494643
:1006C000FFF792FE236961690246DB1B41F82300B4
:1006D000B9F1000FE0D1002151452CD16D1A012D47
:1006E000D0D0A6F12103022B57D8691E2046FFF770
:1006F0007BFE01A9FFF792FF00287BD0212E39D085
:10070000222E0CBF4FF016094FF01709AF1E002F15
:1007100033DA002D40F06081019EF30740F16181E2
:1007200046F001011FE0FFF75BFF0028D3D1104620
:10073000FFF765FFB8E72046FFF74FFE0131CBE733
:100740001E2ACED10021FFF74FFE0246FFF748FFD9
:1007500068B91046FFF753FF0028C2D04FF49F71CD
:100760002046FFF73AFE2046FFF745FE8AE74FF4A2
:10077000AF71F5E74FF01509C8E739462046FFF796
:1007800033FE02A9FFF74AFFA0B34846013FDDE967
:10079000011236F05DFA0190B9E7A6F12403022BAD
:1007A0004BD8691E2046FFF71FFE01A9FFF736FF51
:1007B00000B3AF1EDFF85092002FAADD791E20464D
:1007C000FFF712FE02A9FFF729FF98B1394620462C
:1007D000FFF70AFEC0F30710484410F835ACBAF131
:1007E000FF0F07D0029808F0BFFBBAF1190F17D816
:1007F00000281ADAA91C46EA052620468900FFF7D8
:100800003BFE4660014600F10806C0F80080002D5E
:10081000A9D0013D2046FFF7E0FD46F82500F6E7A8
:10082000BAF11C0F01D90028E4D05046023FDDE99F
:10083000011236F00DFA0190BEE7272E1BD10021E0
:100840002046FFF7D1FD01A9FFF7E8FE0028D1D02F
:1008500001212046FFF7C8FDC0F30710352808D056
:1008600036280CBF01200220019904F0F9FA01900A
:100870004FE70020F8E7052E6CD100212046FFF756
:10088000B3FD07460028B5D010F0030A03D1037961
:10089000533B012BAED901212046FFF7A5FD00F007
:1008A0000F03022BA6D1BAF1000FA3D13B79292B5C
:1008B000A0D1BB6803F00F02022A9BD140F2711253
:1008C000B2EB131F96D1FB68002B93D09A0791D1FE
:1008D0001A792D2A8ED1D3F808B04FEA101902A93F
:1008E0005846FFF79BFE80B9434813F0CDFD014603
:1008F000424807F0EEFAA169054653463A6809688E
:1009000007F028FB2846FBF7A3FD4FEAC9010122A7
:1009100004F1280041F0060136F08AF9029B436099
:100920004846FDF74CFA037820465F2B0BD1FFF7C2
:1009300054FD2046FFF751FD0023082220461946AA
:10094000FFF78EFE9EE6FFF748FD59462046FFF76B
:1009500052FD4FE7292E7FF44DAF01212046FFF7CE
:1009600043FD00F00F030746022B7FF443AF002145
:100970002046FFF739FD00283FF43CAF10F003029A
:100980007FF438AF03792F2B7FF434AF3909D0F8D7
:1009900008901B48C90041F0060136F049F90028CB
:1009A0003FF428AF02AA4FEA1911406804F0CCFBCB
:1009B000029B002B3FF41EAFD90707D49A077FF4A0
:1009C00019AF19680F4A91427FF414AF039A002AB5
:1009D0007FF410AF01939CE62046013DFFF7FDFC3C
:1009E00097E60C212046FFF747FD40F237130146FA
:1009F0000560C0E90136B6E67EA1046054BD04601E
:100A000018A204606CC30460E3A6046010B5036818
:100A100013B91846136010BD9C0702D01060012066
:100A2000F9E71C798C42F9D103F10801116058688B
:100A3000000AF0E72DE9F04F002393B00D46402166
:100A4000019000920793CDE905130598012805D977
:100A50000021C000FBF72CFD0790B0B1002320223D
:100A60000A93CDE908230898012805D900218000C0
:100A7000FBF71EFD0A9060B1079B73B9B34813F0F2
:100A800003FD0146B24804F07AF9059B5B08059323
:100A9000DBE7089B5B080893E5E70A9B002BEDD09A
:100AA00000210FA80B95CDE90D1105F021F9009B50
:100AB000002B49D0022B0CBF3A2200220027DFF87E
:100AC000ACA20023696C05A8FFF7ACFC069C002CC7
:100AD00000F07B81013C07999E4E01EBC403069414
:100AE00051F83410DA78C1F317099B49662A5B681C
:100AF00011F802B099490BF00F08895C88BF41F4E6
:100B0000807106EB41060BF0300110291ED0202920
:100B10004BD0002F00F02C81B8F1020F40F009817A
:100B2000012B18D000211BF0010F03F1FF3006D07C
:100B300074880AEA0404B4F5805F08BF58080128E5
:100B400000D161B10346BFE03822B7E72BB906EB0D
:100B50004306984505D80127B8E7002FF7D10027AD
:100B6000B4E7374636F8021B01EA0A00B0F5805FA9
:100B70000DD195F84C00C1F30B01884213D105A8A3
:100B80001146FFF7AFFC2846FFF74AF8E7E70133C5
:100B9000434503D2494605A8FFF744FC398805A818
:100BA000FFF761FCDBE70133D3E78FB103F10041CD
:100BB000013936F811100AEA0101B1F5405F1ED182
:100BC000002105A8CDE90232FFF715FCDDE902326C
:100BD00006EB4304984532D8009B002B55D10024E6
:100BE00006EB48082746B04573D1012F40F09580A9
:100BF0001BF0400F00F091800026314687E0012B6A
:100C0000A9D995F84C30092B07D8032B00F20F8196
:100C1000022B00F00A8152480AE10B2BFBD151480C
:100C200013F032FC0146504807F053F90446002304
:100C30006A6C296807F08EF92046FBF709FC274605
:100C400034F8021B01EA0A00B0F5805F1BD1C9B27B
:100C500095F84C00884212D10D2807D1114605A8FD
:100C600003930292FFF73EFCDDE902232846CDE91B
:100C70000232FEF7D5FF029B039A0133AAE7002B4D
:100C80003FF469AFBDE7013384E7052AA7D100210E
:100C900005A80292FFF7A8FB029A00289FD1012124
:100CA00005A8FFF7A1FB10F0030F029A00F0C58022
:100CB00000F00F00022892D005A8FFF78EFB05A8D0
:100CC000FFF78BFB00230822494605A8FFF7C8FC65
:100CD00045E738F8023D03EA0A01B1F5805F06D125
:100CE000DBB20D2B7FF47FAF013401377BE7214668
:100CF00005A80292FFF778FB029A00B10137013490
:100D000071E7FFF76AFB0136002818BF0146A642CB
:100D100005A8F6D1FFF76FFB21E71BF0800F06D087
:100D2000002105A802920134FFF765FB029A2346D1
:100D3000CAE7012B3FF40FAF13F001013FF4F3AE0C
:100D4000B8F1030F7FF45DAF0121ECE69AA10460D6
:100D500038BB0460D8A204602CA2046038A60460EA
:100D600009A20460B0A104600CBA046000F0FFFFA7
:100D700008EA030101F0010136F8114004EA0A0013
:100D8000B0F5805F17D1C4F30B0495F84C00A04276
:100D900003F101040DD129B9114605A80292FFF70C
:100DA000A1FB029A28460292FEF73AFF2346029AD6
:100DB000DEE72346B0E6494605A80133FFF732FBDC
:100DC000214605A8FFF74FFB80E60FA804F0ADFF12
:100DD0000E9860B1416822460831FBF786FB0E9BF6
:100DE0005A681A60DDE90D235A600E9B0D9395F841
:100DF0004C30002B7FF405AF099B002B3FF401AF73
:100E00000A9B07981B680C93FBF771FB0A98FBF78A
:100E10006EFB2846FFF7CEFA019BDDE90C0183E863
:100E20000300184613B0BDE8F08F0848F8E60848FC
:100E300013F02AFB01460748F6E600283FF4CFAE40
:100E40000379372B3FF438AFC9E600BFC2A1046075
:100E5000F6A1046054BD046010B5406800B910BD2F
:100E60004468FBF744FB2046F8E700002DE9F04119
:100E700005460E463020002190461F46FBF728FB12
:100E8000072D04460570C660A0F8108001D0012D22
:100E900011D1B268C2F30F12628203F0F1FC042395
:100EA0006061002167762020E384FBF7F5FAE062B9
:100EB0002046BDE8F081014B5A5DEDE7EEA60460E7
:100EC00010B50446C06AFBF712FB2046BDE810408F
:100ED000FBF70DBB30B500220446058D954201D8C5
:100EE000002030BDE36A03EBC20043688B42F8D0B8
:100EF0000132F3E770B504460E461546FFF7EAFFE8
:100F000010B100232B7070BDE38C228D9A4208D360
:100F10000633E06AD900FBF7DDFAE38CE0620633C2
:100F2000E384238DE26A591C02EBC3002185002172
:100F300042F8331001234660E4E7034618465B6835
:100F4000002BFBD1FFF7C6BFF7B5446806460D4638
:100F500017464CB900232B7004E00378022B01D113
:100F60000323037003B0F0BD20466468002CF1D069
:100F70003946FFF7AFFF0028F6D00378023B022B7B
:100F8000E8D804232B701C4675680DF1070239461A
:100F90002846FFF7AFFF9DF80730002BDDD0047027
:100FA0006D68F2E7838B426A01339BB28383918C35
:100FB000994238BF93847047F7B51E4659B111F076
:100FC000030511D14F68FCB294420DD13F0A01F1E3
:100FD0000804BD4201DB03B0F0BD54F8041B013529
:100FE0000190B0470198F4E7334603B0BDE8F04004
:100FF00018470000024B97228968FFF7DDBF00BF4A
:10100000DD1B0160024B67228968FFF7D5BF00BF77
:101010003B32016010B50446084611462268FFF7CE
:1010200025FF636A436000238360236A0BB9206253
:1010300010BD1A469B68002BFBD19060F8E78968C9
:101040000022806A090902F0E4BD8968806A02F022
:101050008EBD2DE9F74F05460C46174698461BB145
:101060000B7E43F008030B76E7836B6A1B78002B3B
:101070003FD143463A462146A86A03B0BDE8F04F47
:1010800002F053BFDB6A03EBC60B13F83630033BA9
:10109000012B1BD84FF0000915E0E36A03EBC902EE
:1010A00013F83930042B0CD1DBF804105368994243
:1010B00007D10AF1010A0023BBF80220A86A02F056
:1010C000F3FB09F10109238D4B45E6DC01366B6A20
:1010D0001A8DB242D6DCBAF1000FCAD03B46524656
:1010E0002146A86ACDF8008002F035FF03B0BDE8C4
:1010F000F08F0026B246EAE7F8B50E4611461A46CA
:101100000023044685794769837143610D4BFFF7DE
:1011100053FFA368A3B9E18A39B1A28A2AB9A06AA8
:1011200002F0B7FEA06A02F02CFDA38A3146E28AE3
:101130002046FFF78EFF003D676118BF0125A571AE
:10114000F8BD00BFC922016070B5437905460C4661
:10115000012B06D1436A0A4602215B7EFFF75AFF44
:101160002061A268284621694823BDE87040FFF746
:10117000C3BF70B51346427905460C46012A04D117
:101180000A460721FFF746FFA061A66928464023CB
:10119000E2683146FFF7B0FF708A70BD31B101F0EF
:1011A00003030268134304BF0B6803607047000029
:1011B00038B583680D460446114653B9054806F014
:1011C00088FE2946A06004F10C00BDE83840FFF716
:1011D000E5BF38BD54BD046013B504460548019110
:1011E00013F052F901990246204602B0BDE81040C2
:1011F000FFF7DEBFF5A6046070B50B7904460D4617
:10120000092B0BBF068B0B480B48668B13F03CF980
:101210004FF6FF739E4204D1024629462046FFF74F
:10122000C7FFA28B3146E38BA06AD21ABDE870409B
:1012300002F062BD27A7046012A7046073B5446A78
:1012400006460D46207E810709D5274813F01CF974
:10125000294602463046FFF7ABFF02B070BD05F0ED
:101260000F01022916D12909B3791BB1A38B0133D0
:10127000A38302E0638B0133638301240029ECD054
:101280000DF10702706AFFF735FE9DF807303BBB92
:101290001648DBE72979914202D1A9680909E3E7F9
:1012A000994216D1B379002BCFD10123B371AA682B
:1012B000002AD2D0237E02F00F0243F00103022A5B
:1012C00023764FF0030416BFAB68A9689968090933
:1012D000D4E7A96840F00200090920760524CDE78B
:1012E000022344700370B8E709A204603FA70460BA
:1012F0004B234A22FFF7A2BF43234222FFF79EBFA0
:1013000010B40446426A40790B46012804D11046C5
:101310005DF8044B02F0DBB8A06A02495DF8044BAB
:1013200002F0FEB8B0AA046010B40446426A4079E4
:101330000B46012804D110465DF8044B02F0D8B8E2
:10134000A06A02495DF8044B02F0EAB8B8AA04604A
:1013500010B5436A04465A7EFFF70BFF014620464C
:10136000BDE81040FFF7E0BF10B40446426A407980
:101370000B46012804D110465DF8044B02F0B8B8C2
:10138000A06A02495DF8044B02F0CAB8A8AA04603A
:1013900037B505460C4629B1CA0705D54910806AFC
:1013A00002F096FB03B030BD8B072BD001F00F0489
:1013B0000B09062C07D00A2C0AD0022C1BD1194687
:1013C000FFF79EFFEEE71946806A02F0C4FBE9E7EB
:1013D0004279042A04D01149806A02F0C8FBE1E78F
:1013E00001A91846FCF7F0FCAC6A019909F036FE39
:1013F00001462046F1E70A2BD4D0D9B2806A02F028
:1014000049FBCFE70968806A02F0C8FA2279044BE9
:101410002146284653F822309847C3E774C8046031
:10142000C8A904602DE9F14F0D4604461646A907E8
:1014300011D005F00F03022B16D1F2074FEA151158
:1014400004D401B0BDE8F04FFFF76EBF01B0BDE8B6
:10145000F04FFFF755BF6968CBB22A2B75D00ED875
:10146000062B10D0292B15D0514813F00DF8294622
:101470000246204601B0BDE8F04FFFF799BE2B2B86
:1014800074D0972BF0D1002EEED105F108030A0A93
:1014900000217EE0022A02D0A968FFF779FFEF68F9
:1014A000002FE1D017F00309DED17B68B846DAB22D
:1014B000882A0DD1022E4FEA132805D007F1080A19
:1014C00008F1FF3BD9450EDB08F1010857F82880E9
:1014D00098F804302E2B1FD1022E0CD1A06A02F0F6
:1014E000B5FB012112E05AF8041B204609F101095D
:1014F000FFF74EFFE6E7D8F808102046FFF748FF51
:10150000012EEED1A06A02F068FB0021A06A01B0B2
:10151000BDE8F04F02F0A3BB2F2BA5D1012EA06A8E
:101520000BD102F051FBD8F8081000220909A06A7B
:1015300001B0BDE8F04F02F06CBB022E01D102F009
:101540005FFBD8F808100122F0E7A86800288BD0CC
:10155000002A89D1C16839B311F0030324D14A6844
:10156000D6B28F2E17D11A46816812E0002A7FF476
:101570007BAFA96829B90B4601B0BDE8F04F00F078
:1015800019B88B0703D10B7908468C2BE2D00023C6
:101590001A462046F0E7902E03D101F10803120A03
:1015A000E2E7A72E3FF460AF00F1080302226FE7E5
:1015B00058A704602DE9F74F0E1E054617469846BA
:1015C00014BF4FF001094FF000091ED016F00304BC
:1015D0001BD13379202B18D12146806A02F098FC68
:1015E0004FF0000A7B1EBA4512D1631C36D109EBBD
:1015F0000701A86A02F081FC002E38D108EB8707AA
:10160000B84537D103B0BDE8F08F4FF0FF34E7E7BE
:1016100058F82AB0BBF1000F12D01BF0030F0FD106
:101620009BF80420202A0BD101340CD10AEB0904C9
:10163000A3EB0A02A86A2146019302F069FC019B10
:101640000AF1010ACFE7124812F01EFF594602467E
:10165000284603B0BDE8F04FFFF7AABD002ECDD05D
:101660002CB92246B1682846FFF7DCFEC6E7002207
:101670003146F8E7A14558F8041B4FF00002284610
:1016800008BF896809F10109FFF7CCFEB8E700BF80
:1016900073A704602DE9F74F06460C4615461F4612
:1016A0002046FEF79DFF08B1E5B904E02046FEF7AD
:1016B000A6FF38B1B5B13946B06A03B0BDE8F04F06
:1016C00002F0E8BA002C54D0A30752D163684FEA65
:1016D000132BDBB21C2B1BD1F5B1083404EB8B0BA5
:1016E0005C450DD103B0BDE8F08F43465AF8041BAA
:1016F0003046019209F10109FFF7CCFF019A19E088
:101700003B462A4654F8041B3046FFF7C3FFE7E781
:101710001D2B22D1002DE0D0D6F8108004F1080A4C
:101720004FF0000985F0010208F1010333610BF16C
:10173000FF330093009B4B45D7DC0BF10101304692
:101740003B462A4654F82110FFF7A4FF4146B06AF1
:1017500003B0BDE8F04F02F071B91E2B03D1A468AD
:1017600085F001059CE72A2B03D1A368002BA1D1AA
:101770009AE721463046FFF70BFE3A462946B06A03
:1017800003B0BDE8F04F02F091BA2DE9F8430769C4
:101790001E4604460D46BB1C07F10109394690461A
:1017A0000361806A02F04AF94946A06A02F003FB2D
:1017B000A96800222046FFF735FE2D690DBB414682
:1017C0002046FFF7E5FD636A1978062913D1A06A60
:1017D000294602F00BFCA06A02F008FA3946A06A1A
:1017E00002F058FAA06A494602F028F9A06ABDE85A
:1017F000F84302F0ECBAB200A06A053202F065FBD1
:10180000ECE72B79A82B07D1A9683B46002220469C
:10181000FFF740FFED68D1E7E9682046FFF7B8FD24
:10182000A06A012102F0B8FA731C424629462046FC
:10183000FFF7ABFFD2E700002DE9F3410D4600268C
:10184000044642710661114645622A46806A01F0EB
:101850005FFF6379012B04BF6E84AE84EE6866B1CE
:10186000B2070AD133793A2B07D1B1682046FFF786
:101870008FFDA06A02F0A2FB20E02B7843B931462D
:101880002046FFF785FD1421A06A02F003F9F0E776
:10189000072B677918D1012F07D10023402220465A
:1018A000A3714D4BF168FFF787FB20467169FFF785
:1018B0006FFDA06A01F0E5FF0028E4D0A06A01F006
:1018C000B1FF02B0BDE8F081022B14D1012F07D186
:1018D000002348222046A371404BB168FFF76CFB00
:1018E000F1682046FFF754FD2B7E5B07C1D5A06A47
:1018F00002F07CF9C7E7033B032B3FD8012FD6F852
:101900000C8008D10DF107023946606AFFF7F2FA40
:10191000022303706F832B78032B1ED10122002139
:10192000A06A02F0B6FA2B78062B1ED1A06A02F04C
:1019300028F901212046FFF7E3FCA06A02F021F913
:10194000A06A02F01EF90023B26841462046FFF764
:101950001CFF2B78062B8CD195E7042B01D1032299
:10196000DDE7052BDFD10622D9E720460121FFF76D
:10197000C7FC0121A06A02F00FFAE4E7012F07D1AA
:101980000DF107020A212846FFF7B4FA022303707B
:101990002A212046FFF7B4FC28212046FFF7C4FC8B
:1019A000B168A06A090902F0D6F832212046FFF793
:1019B000BBFC31692046FFF7EBFC0A212846FFF704
:1019C00089FA0378022B3FF45EAF428800230A2194
:1019D000A06A01F069FF4CE7F9120160F1120160A1
:1019E00070B5436A04460D461B78072B0BD0022BBB
:1019F00009D0174812F048FD294602462046BDE8A6
:101A00007040FFF7D5BBAD682DB91421A06A02F074
:101A100041F8002112E015F0030614D12B79AA2B0E
:101A200011D1A9682046FFF7B3FC3146A06A02F045
:101A3000B3F91421A06A02F02DF80121A06ABDE8D3
:101A4000704002F0D3BA29462046FFF7A1FCE0E738
:101A50008DA7046038B505460C46C968FFF798FCA9
:101A6000A1682846BDE83840FFF792BC38B50B792D
:101A700004460D46312B0CD18968FFF789FCED68CF
:101A8000AD685DB91421A06A02F004F808220221B1
:101A900015E01421806A01F0FDFFF1E7AB071CD1CE
:101AA0002B79942B10D11421A06A01F0F3FFA968BF
:101AB0000029EBD02046FFF76BFC08220321A06A27
:101AC000BDE8384002F0E5B9952B06D1A96820465B
:101AD000FFF75EFCEB689968EAE729462046FFF7C6
:101AE00057FCD3E710B504468968FFF751FC002185
:101AF000A06ABDE8104002F0B2B82DE9F0410646F8
:101B000015460C4611B10124FFF742FC3DB16F6848
:101B10004FF0000808353F0AB84507DB3C44214632
:101B2000B06A0022BDE8F04102F0B3B955F8041BD9
:101B3000304608F10108FFF72BFCEDE70A460021CB
:101B4000FFF7DBBF2DE9F04706690446D0F818A07F
:101B50000D46B31C06F10108B0F81E900361838B9B
:101B60000683A0F81A80C3838868FEF739FDE0B9C0
:101B700027697B1C2361A868FEF741FD18B941461F
:101B8000A06A02F087F83946A06A01F057FFE968B9
:101B90002046FFF7FDFB4146A06A01F04FFF3B46A0
:101BA0000122A9682046FFF775FD2046C4F818A059
:101BB000A4F81E902969FFF7EBFB3146A06ABDE847
:101BC000F04701F03BBF10B504468968FFF7E0FB22
:101BD000A06ABDE8104002F009B800002DE9F04706
:101BE00005460C4604F00F03022B05D121092846B7
:101BF000BDE8F047FFF7B8BB002C66D0A20764D160
:101C00002379292B37D1A1682846FFF7C1FBE66865
:101C1000002E5AD016F0030857D177683346FAB22F
:101C2000882A09D13F0A06F1080907F1FF3AC2459F
:101C30000FDC013756F827301A792E2A11D12846A1
:101C40009968FFF7A5FBA86A0221BDE8F04702F0FA
:101C500006B859F8041B284608F10108FFF798FB5D
:101C6000E5E72F2A31D199680222A86A0909BDE85F
:101C7000F04701F0CEBF2A2B27D1A4682CB3E66829
:101C8000EEB1B3071BD17768FAB28F2A01D1A468ED
:101C9000A8E7902A11D1A1683F0A083600242846F7
:101CA000FFF79CFFBC4201DBBDE8F08756F8041B40
:101CB00028460134FFF792FFF4E7A72A05D0A16870
:101CC0002846FFF78BFFE4688CE7054812F0DCFB41
:101CD000214602462846BDE8F047FFF769BA00BF33
:101CE000A6A704602DE9F0414B6805460E4601F1B8
:101CF00008081F0A0024BC4201DBBDE8F08158F847
:101D0000041B2846FFF744FBAB6843B1023405F1DE
:101D10000C0056F82410BDE8F041FFF73FBA01343B
:101D2000E9E710B50446FFF7DDFF2021A06ABDE812
:101D3000104002F088B82DE9F347066904460D46C5
:101D4000731C03618868FEF74BFC0246F8B92769EB
:101D500020467B1C23613B46A968FFF79BFC20467D
:101D6000E968FFF715FBA868FEF749FCE8B92B699D
:101D70000BB96B693BB1A06A01F083FD18B931461C
:101D8000A06A01F087FF3946A06A01F057FE01AA58
:101D90006C2105F110000027FEF738FE81464F4503
:101DA0000ADB69692046FFF7F3FA3146A06A01F0C1
:101DB00045FE02B0BDE8F087019B53F82780D8F8B4
:101DC0000800FEF70DFC024608BBD4F810A0204620
:101DD0000AF1010323615346D8F80810FFF75AFCB3
:101DE0002046D8F80C10FFF7D3FAD8F80800FEF711
:101DF00006FC0028D9D1A06A01F043FD18B931468C
:101E0000A06A01F047FF5146A06A01F017FE0137B2
:101E1000C5E770B5437904461546CE68012B06D157
:101E2000436A0A4629465B7EFFF7F4F87061002397
:101E3000716920461A46FFF70CF9F1682046FFF752
:101E4000A7FA062D03D10021A06A01F0A5FF002307
:101E5000A06A01211A46BDE8704002F098B870B53A
:101E60008D68044635B901222946A06ABDE8704054
:101E700002F00FB8AA0730D12B798C2B2DD1EE6848
:101E800006B3B3071ED133798F2B05D1A968FFF7AD
:101E90007FFA01221146E8E7902B0BD1A968FFF7E2
:101EA00077FA31462046FFF71DFF71680122090AC3
:101EB0001144DAE7A72B05D129460322BDE870407B
:101EC000FFF7A7BFA9682046FFF762FAE968204636
:101ED000FFF75EFA01220221C7E729462046D6E72E
:101EE0002DE9F04F4FF0000B87B004461F46D9464E
:101EF000DA465E46D84603A8CDE9022105AA9F210D
:101F0000FEF784FD0190019B9B4516DB5EB1BAF1A3
:101F1000000F6AD1A06A01F034FEB9F1000F6AD156
:101F2000A06A01F02EFE029BA06A002B69D0334606
:101F30004246394602F036F813E0059A52F82B5023
:101F4000002D43D0A80741D12A79A12A12D1F10747
:101F50000AD52F4812F098FA294602462046FFF784
:101F600027F907B0BDE8F08F46F00106AA460BF14D
:101F7000010BC8E7A22A07D1B20701D52548E9E736
:101F800046F00206A946F2E7A32A1FD1EA6822B169
:101F9000930702D11279A72A11D0A96801F00F0284
:101FA000022A01D01C48D5E70909A06A01F0D3FD37
:101FB000E968204608F10108FFF7EAF9D7E70622A9
:101FC000294620460137FFF724FFD0E70EB113481A
:101FD000C0E7B8F1000F01D01148BBE72946204601
:101FE00001374646FFF7D4F9C1E7DAF80810204672
:101FF000FFF7CEF991E7D9F808102046FFF7C8F9A6
:1020000091E733464246394601F0C1FFA9E700BFD8
:10201000BEA70460D5A70460EDA704600EA8046005
:1020200029A8046070B50D4641790446134601297C
:1020300003D12A46FEF7EEFF6861A06A01F0BBFDFE
:102040006E690023204631461A46FFF702F8718A6E
:10205000A06A01F080FDE96829B18B0703D10B79F3
:102060009E2B08BF0021204602230022FFF738FFE5
:10207000708A70BD10B5436A04465A7EFFF7D2FFDE
:1020800001462046BDE81040FFF74EB9002389689D
:102090001A46FFF725BF00002DE9F04F0E4685B028
:1020A00004463D2102AA06F10800FEF7AFFC002518
:1020B000636A8346A846DFF8E4A093F819905D456B
:1020C00014DBF1684A4620460B79032B5AD1FFF7FF
:1020D00050F805460026ABEB0808B04555DC29460C
:1020E0002046FFF721F905B0BDE8F08F029B03AA57
:1020F000682153F8253003F108000093FEF786FCB1
:10210000039B40F2472207461968B2EB111F0CD01F
:102110002046FFF73DF90123BB4227DB009BD9682E
:1021200081B12046FFF734F90CE002280CD050466C
:10213000009112F0A9F9009902462046FFF738F8FD
:1021400008F101080135BAE75F683B09B3F5A97FDB
:1021500009D040F259229342F2D0504612F094F93D
:1021600039460246E9E74FF00109E9E7039AA06A18
:1021700052F8231000220193090901F04AFD019B46
:102180000133C9E7FFF74EFFA3E700230121A06A4F
:1021900001361A4601F0FBFE9FE700BF4BA8046022
:1021A0002DE9F7438D6804462DB903222946A06A1C
:1021B00001F06FFE10E0AA077AD12B79342B0ED1F3
:1021C00003220121806A01F064FE20462946FFF7C0
:1021D000DFF8A06A01F06FFE03B0BDE8F083992B31
:1021E00066D1EB681A799C2A52D19D2101AA03F18C
:1021F0000800FEF70BFCA9680746E1B18B071AD16E
:102200000B79342B17D10322411CA06A4FF001092E
:1022100001F03FFEA9682046FFF7BAF8A06A01F076
:102220004AFE4FF00008B8450BDBB9F1000FD3D1DF
:102230000622791CBBE720464FF00009FFF7A8F8FB
:10224000EFE7019B53F82810B1B18E0714D10E7936
:10225000A6F13400464246412046FFF799F8B9F10D
:10226000000F11D056B9164812F00EF92946024651
:102270002046FEF79DFFAFE70026EDE7A06A01F0DC
:102280001AFE08F10108CEE7002EFAD00D48EBE760
:10229000AB684BB19A0707D11B79342B04D10422C8
:1022A0002946FFF7B6FD97E7052229462046F8E7BD
:1022B00029462046FFF76CF80622012177E700BF88
:1022C00069A8046086A8046001F00F03022B70B5B2
:1022D00004460D460ED04B6803F0F702432A02D1A4
:1022E0000123837170BD442AFCD0DBB2422B11D193
:1022F0002E698EB9A379002BF4D1E38A002BF1D09B
:102300001C4812F0C1F8294602462046BDE870403C
:10231000FEF74EBFEE68ECE7A3790BB3A38AAD6876
:1023200001339BB2012BA3820AD1E18AA06AA1B139
:10233000002201F0AEFD03220021A06A01F0A9FDF8
:1023400031462046FFF724F8A06A290901F003FC72
:10235000A06ABDE8704001F0AEBD01F012FCEAE7F2
:10236000E38A314620460133E382BDE87040FFF73F
:102370000FB800BFA5A804602DE9F7430D46896892
:102380000446FFF705F8EE68002E5DD07768FBB2D3
:10239000882B636A1B7819BF05F10C0601273F0AD9
:1023A0000836072B53D1AB6803F00F02022A4ED137
:1023B00040F20B32B2EB131F49D133681A792D2A40
:1023C00045D19B68002B42D10A212046FEF798FF99
:1023D000626AD36A128D62B931683148019112F094
:1023E00053F801990246204603B0BDE8F043FEF7DA
:1023F000DFBE5978C9070DD559682046FEF780FF22
:10240000022F0AD800230221A06A01251A4601F0F2
:10241000BEFD17E0013A0833DDE773681A792F2A09
:10242000F0D1B5682A792D2AECD199680122A06AE9
:10243000090901F0AFFBA96803250023012220460A
:10244000FFF74EFDAF4204D803B0BDE8F08300258E
:10245000F8E705F10108AB0056F82510B84519D288
:102460000A792F2A16D13344D3F8049099F804300E
:102470002D2B0FD189680022A06A090901F08AFB7F
:1024800000230122D9F808102046FFF729FD08F1A2
:102490000105D7E72046A846FEF77AFFF7E700BF19
:1024A000D3A804602DE9F0414F680226DFF83C8094
:1024B0000C463F0A89680546FEF76AFFB74201DC11
:1024C000BDE8F08121692846FEF762FFE368A86A4B
:1024D0000236C3F307130834353B082B94BF18F8B2
:1024E0000310192101F0AFFCE8E700BFA6A90460C2
:1024F0002DE9F0414D680C4601278968A5F10C08CB
:102500000C342D0A06465FFA88F8FEF741FFAF4209
:1025100001DBBDE8F08154F8041B3046FEF738FFBC
:102520004146B06A013701F08EFCF0E7F8B5CD689E
:1025300004460E461DBB0379A3B1436A1D788DB9CD
:102540003521FEF7DDFEB1682046FEF721FF2B4660
:102550002A460121A06A01F01AFDA06ABDE8F840F0
:1025600001F044BBB1688B0700F0848001F00F03D9
:10257000022B40F086802046FEF70AFFEDE7AF070A
:1025800072D16B68DAB2532A15D101228968FEF73D
:1025900049FFE9682046FEF7FBFEAB68A06A1B090D
:1025A000543B0A2B96BF374A1421D15C01F04BFCF7
:1025B0000222B16853E0542A21D11B0A5F1E013365
:1025C00055F82310FEF7E4FE002F02DDA06A01F0AB
:1025D000FBFAB1680835002600222046FEF722FFEC
:1025E000BE424EDA0136BE4202DAA06A01F0ECFACF
:1025F000002255F8041B2046FEF714FFF0E7062AD8
:1026000032D18F6887B3B8072ED17A68D1B2062944
:102610002AD11B0AB3EB122F26D1022B24D1BB687F
:1026200023B1990702D11B79202B1DD0FB6823B160
:102630009A0702D11B79202B16D0A9682046FEF7F5
:10264000A7FEE9682046FEF7A3FEA06A01F0D8FACB
:102650000022B9682046FEF7E5FE0022F968204610
:10266000BDE8F840FEF7DEBE29462046FEF790FEA4
:1026700000229EE700293FF47EAF0B79372B7FF4D1
:102680007AAFF8BDAFA9046038B50C46C9680546F5
:10269000FEF77EFEA368C3F30713352B08D0362B55
:1026A00014BF02210121A86ABDE8384001F0BFBB78
:1026B0000021F8E710B504468968FEF769FE03219A
:1026C000A06ABDE8104001F0B2BB2DE9F84391F8D3
:1026D00004900546D0F8108001F10804A9F11C030C
:1026E0000027D3F1000949EB030908F10103036155
:1026F0004E68360AB74205DB4146A86ABDE8F84392
:1027000001F09CB9013754F8041B2846FEF740FE3F
:10271000B742F1DA42464946A86A01F0DAFAE9E737
:102720002DE9F8434E680D4689680446360A0127AC
:10273000FEF72EFEDFF8B890032E89BFD4F8108084
:102740004FF0000808F1010323617B1CB3421CDB3E
:10275000032E4ADD2569A06A6B1C2946236101F01E
:1027600099FA4146A06A01F069F90121A06A01F0D5
:102770008DF8A06A01F044FAA06A01F037FA294600
:10278000A06ABDE8F84301F059B90237296920462B
:10279000FEF7FEFDB74205DAA06A01F015FAA06A5D
:1027A00001F054FAEB68A06A03F00F020E2A11D16F
:1027B0001B093C3B0B2B94BF19F80310062101F0B9
:1027C00042FBB74204DA42460021A06A01F081FAD6
:1027D0000835BAE71A797F2A01D13021EFE79B68E3
:1027E0000BB90721EBE73121E9E7BDE8F88300BF2A
:1027F000BAA904602DE9F04105690446D1F80C80BE
:102800000E46AB1C00226F1C03612B46D8F8081043
:10281000FEF740FFB1682046FEF7BAFD3946A06AD0
:1028200001F038FA2946A06A01F008F9A06A4FF0D1
:10283000FF3101F02BF8D8F80C102046FEF7A8FD68
:102840003946A06ABDE8F04101F0F8B82DE9F04F33
:102850002DED028B8B6887B004460E4603F00F0304
:10286000022B40F0F280CB68002B00F0EE8098073E
:1028700040F0EB801A79292A40F0E7809A6802F04C
:102880000F01022940F0E18040F29521B1EB121FC7
:1028900040F0DB80DB681A792D2A40F0D6809B68F7
:1028A00005AA9F2104A80493FEF7B0F8431E022B4B
:1028B00000F2CB80059901280A6800F0B98002284F
:1028C000D1F804A000F004818D68E90740F1BD80D3
:1028D0006B0800F0BA8032B1930704D11179A139A5
:1028E000022940F2B280BAF1000F08D01AF0030FAB
:1028F00005D19AF80410A139022940F2A680B368E4
:102900001AF0010B776908EE103A3369A18B08EED3
:10291000903AA36926690293E38B06F10208E183EA
:1029200006F10401019306F1010306F10309268370
:1029300003936383216105D1514620460392FEF73C
:1029400027FD039A11462046FEF722FD4946A06A5C
:1029500001F0A0F94146A06A01F070F8A06A01F008
:1029600033F9002218EE101A2046FEF75BFD18EE30
:10297000901A2046FEF70CFD711CA06A01F05EF86B
:1029800029462046FEF704FD0E21A06A01F05BFAFD
:10299000A06A494601F052F8A06ABBF1000F4BD182
:1029A00001F01BF9A06A01F02BF9002DA06AACBF61
:1029B0000021012101F047FA42460121A06A01F0FD
:1029C00075F9029BA361019BE383002F3BD0A06AB2
:1029D00001F00CF9BBF1000F02D1A06A01F006F979
:1029E00039462046FEF7D4FC2569A06A6B1C2946AF
:1029F000236101F04FF98BF00101A06A013100F071
:102A000045FFA06A314601F019F8A06A01F0EEF81E
:102A1000BBF1000F02D1A06A01F0E8F81FB129460E
:102A2000A06A01F00BF807B0BDEC028BBDE8F08F97
:102A300092460325024656E701F0C6F85146204665
:102A4000FEF7A6FCB1E73D46DBE725692046A38BF0
:102A5000B4F81E906F1CE3836FEA4543D4F818A0C6
:102A600005F102086FEA534367832383EB1C23615C
:102A7000F168FEF78DFC0121A06A01F08DF939465D
:102A8000A06A00F0DBFF4146A06A01F094F9002241
:102A9000B1682046FEF7C6FC20463169FEF778FC97
:102AA000A06A00F0EEFE18B93946A06A01F0F2F80B
:102AB0004146A06A00F0C2FFA06A01F088F9C4F89C
:102AC00018A0A4F81E9020467169FEF761FCA6E7E5
:102AD000032500E72DE9F7430446904699460F4643
:102AE00029B9194603B0BDE8F043FEF751BC0669A9
:102AF000731C036115684DB315F0030226D12B79C1
:102B0000762B23D1A9680192FEF742FC019A314647
:102B1000A06A01F025F9019AE9682046FEF782FCD7
:102B20002046FEF73FFA4B4608F10402791EFFF7F4
:102B3000D1FFA06A314601F057F9A38BA06A013B8F
:102B4000A38303B0BDE8F04301F01CB92946204639
:102B5000FEF71EFCA06A0022314601F001F9A06ACE
:102B600001F044F8DCE737B50C46054601AA7521AB
:102B700004F10800FDF74AFFE3680146019A284680
:102B8000FFF7A8FF03B030BD2DE9F04F2DED028B0C
:102B900083B005699B4604460E9B0F460192294669
:102BA00008EE103AAB1C022205F1010A036100266F
:102BB000806A01F0D5F82046FEF7F4F93946FEF7B1
:102BC000E7FBA06A01F007F95146A06A01F062F83C
:102BD0002946A06A00F032FFA06A01F018FAD4F882
:102BE000108008F101032361019B9E421ADBA38B35
:102BF000A06A013BA38301F0C5F8A06A01F00AFABC
:102C00005146A06A00F01AFF18EE101A2046FEF78F
:102C1000BFFB4146A06A03B0BDEC028BBDE8F04F9C
:102C200000F00CBF5B46D4F810900BF1040B01369A
:102C30001A68009209F101022261009A9768002F38
:102C40004DD1019AB24238D10025A06A00F0CEFFE2
:102C50002F46009B2046D968FEF79AFB15B1A06A63
:102C600001F0B9F8A06A01F0D9F8CDB11421A06A39
:102C700000F010FF3946A06A00F0E0FE1421A06ABF
:102C800000F008FF29462046FEF74EFB2046294665
:102C9000FEF76AFBA38BA06A013BA38301F072F8E5
:102CA0004146A06A00F0F6FF4946A06A00F0C6FE61
:102CB0000121A06A00F0EAFD96E719681F4800911B
:102CC00011F0E2FB009902462046FEF771FAA38B51
:102CD000013BA38303B0BDEC028BBDE8F08F17F07E
:102CE000030528D13A793B46712A02D1DD68BF68D5
:102CF0002D09A06A00F068FF39462046FEF748FB20
:102D00000821A06A01F09FF84A460021A06A00F05D
:102D1000CDFF002D98D029462046FEF705FB2769F8
:102D2000A06A03227B1C3946236101F019F8204672
:102D3000FEF738F98DE70025DBE700BFEBA804605C
:102D40002DE9F0430769164685B004467A1C0D4606
:102D50003946039302610322806ADDE90C9800F092
:102D6000FFFF2046FEF71EF9039B26BB0321A06A46
:102D700000F08CFD29462046FEF70AFB6FF00201A9
:102D8000A06A00F083FDA06A01F025F8A06A142172
:102D900000F080FE3946A06A00F050FE2046414611
:102DA000FEF7F6FAA38BA06A013BA38305B0BDE84A
:102DB000F04300F0E7BF32462946CDF80090FFF718
:102DC000E3FEE0E77FB5CD6806460C462B79732B12
:102DD00009D1AB680193002300931A468968FFF775
:102DE000AFFF04B070BD6F2B03AA4FF0720116D174
:102DF00005F10800FDF70AFE2B6902463BB9EB68B6
:102E000000933046039BA168FFF7BEFEE9E79B688D
:102E10003046A1680193EB680093039BDFE704F160
:102E20000C00FDF7F3FD00230246E9E738B5436ADD
:102E300004460D461B78072B09D00C4811F024FBE3
:102E4000294602462046BDE83840FEF7B1B98968F8
:102E500041B91421806A00F01DFEA06ABDE8384027
:102E600001F0ACB8FEF794FAF7E700BF09A90460D7
:102E700030B48968044619B90A4630BCFEF73DBE35
:102E8000CB688BB113F003020ED11D798F2D01D1C8
:102E90008968F2E7902D01D11A46F9E7A72D03D1F1
:102EA000062230BCFEF7B5BF0A4620460021E4E703
:102EB000F8B5144B04460D46D3F8DC700FBB066919
:102EC0000122731C036133468968FEF7E3FB682126
:102ED0000122A06A00F002FDE96841B12046FEF738
:102EE00057FA3B463A460121A06A01F050F8A06A21
:102EF000012101F06FF83146A06ABDE8F84000F00A
:102F00009DBDF8BD0004002038B58D6804462DB97C
:102F10002946A06ABDE8384001F05CB8AB070BD188
:102F20002B795A2B08D1A968FEF732FAE9682046B6
:102F3000FEF72EFA0221ECE729462046FEF728FA92
:102F40000121E6E72DE9F04F437985B004460D46AF
:102F5000012B0FD191F80480B8F1100F0DD0436A06
:102F60001B7853B92A4811F08FFA294602462046A9
:102F7000FEF71EF905B0BDE8F08F03AA692105F13F
:102F800008000026FDF742FDDFF888900746DFF8CD
:102F900088A0DFF888B0B742ECDD039B0DF10B028F
:102FA000606A53F8261009090191FDF7A3FFB8F1F3
:102FB000100F03469DF80B20019916D15AB90278DB
:102FC000012A08D0584611F05FFA294602462046E9
:102FD000FEF7EEF807E001221A70606AFDF7ADFF18
:102FE00008B1012202700136D5E75AB10A460190B4
:102FF0000146606AFDF7A8FF019B1B78002BF2D108
:103000005046E0E70378042BEDD04846DBE700BFED
:1030100023A9046085A9046067A9046048A9046025
:103020002DE9F04F87B081460C4600AF11B9012160
:10303000116013E011F0030619D10B79642B06D14E
:10304000CB681B0913608C68002CF0D0012604F0BB
:103050000F03022B0DD12109002EE9D00022D9F84F
:10306000000000F0FAFC1C37BD46BDE8F08F0026DA
:10307000EDE716B9A3681B091360636800254FEAE2
:10308000132804F1080308F1FF3A9B46FB60A845AA
:1030900025DC0AF107034FF0000B23F00703ADEB2B
:1030A000030D6B461D46D84521DC51461846FAF7FC
:1030B000EBFD00220146D9F8000000F0CEFC002E06
:1030C000D1D00C340125A845CDDD54F8041B0022D5
:1030D000D9F800000135090900F09BFDF3E75BF822
:1030E000040B01350009FAF765FE8244CFE7BBF116
:1030F000000F03D04FF02E0205F8012B7B6007F183
:103100001401FB680BF1010B53F8040B0009FB6081
:10311000FAF75AFE7A6901462846BA6033F020FD74
:10312000BA687B681544BEE72DE9FF418C68054607
:103130000E4604F00F030E2B06D0002C40D0A30740
:103140003ED12379612B2DD10294002403AA612161
:1031500002A8FDF75BFC0023039A40F20E5C1946BF
:10316000834225DBF26840F27E332F469A4257F8BD
:10317000280F27D100F0ACFC4B21A86A00F0EBFC33
:1031800000220121A86A00F084FE03AA21463846E5
:10319000FFF746FF02220021A86A00F05EFC04B09F
:1031A000BDE8F0815E2B0BD1A3680293E468CDE704
:1031B00052F82370013367450CBF01310331CFE76B
:1031C0000021CFE700F084FC06F10C0002AA662182
:1031D000FDF71CFC4FF000080646B045A86A0FDB5F
:1031E0000022314600F055FE2146002403AA38464D
:1031F000FFF716FFB442A86A0CDB00F0F7FCCEE73D
:10320000029B53F8283008F101089968090900F079
:10321000A2FCE2E7029B012253F82470B968090975
:10322000019100F01AFCFB682BB901992846013482
:10323000FEF77AF8DEE71909F8E773B504460E469B
:10324000806A0021254600F043FC142155F8280F20
:1032500000F020FC01AA31462846FFF7E1FE019963
:103260002046FEF761F802B070BD2DE9F04F8DB039
:103270000F46144606462822002102A81D4633F0B8
:1032800097FC4FF0FF3332680021079301A82346D3
:1032900001978DF808500027FDF7BCFE044600F0AA
:1032A0001FFADDF8248005460B90B8F1000F01D01D
:1032B000039B03B3099B4FF0000C4FF0010E0BB1C1
:1032C000039A22B33946284600F00EFA099F039B61
:1032D000002F00F0E080002B00F0C6800A9B04A8BD
:1032E000D968FDF75BFF0A9B049A5B8A01990398F2
:1032F00004F030FED2E04146012201A8FEF79CFA1C
:10330000059BD8F808809F4238BF1F46CDE7197E3D
:10331000C90713D5198D013910D3D86A00EBC1083C
:1033200098F8010010F0020F17D03AB1D2E900A9C5
:1033300098E8030082E80300C8E900A90022A3F886
:1033400020C0198D8A420EDB0022198D8A422DDBA6
:103350005A68002A64D19B68B1E7002ADBD10128B2
:1033600008BF4246D7E719784FEAC209D86A01294F
:1033700000EBC20805D1D8F804100A290CD101329B
:10338000DFE710F8321007D931B900F809E098F8F2
:103390000110C80704D4F2E710F809100229F6D189
:1033A000198C481C1884A8F80210E8E7D96A01EBC8
:1033B000C20011F83210032906D14178C9075FBF56
:1033C000198C4180013119840132BEE7C96A01EBD1
:1033D000C80A11F838100339012917D84FF000092D
:1033E00011E0D96A01EBC90B11F83910042908D191
:1033F000DAF80400DBF80410884204BFABF80220BE
:10340000013209F10109198D8945EADB08F101084A
:103410005968088D8045D9DB002A9CD0002117E02F
:103420004FF000084246F3E7D3F82C8008EBC100C8
:1034300018F83180B8F1040F04D190F8018018F029
:10344000010F04D0B0F802809044A0F8028001314E
:10345000188D8142E8DB598B11FA82F15983198C5E
:1034600011FA82F21A8476E70222394601A80B95F6
:10347000FEF7E2F9039B63B90322394601A8FEF780
:10348000DBF9039B2BB9042239460DEB0200FEF752
:10349000D3F9BF681BE7002B7FF420AF284600F06C
:1034A0002DF93046FDF7D8FC65692046A468FDF784
:1034B00007FD002CF9D1039808B1F8F7C9FF22469F
:1034C0002146284601F0F8F90DB0BDE8F08F37B578
:1034D0000DF107020D460446FDF70CFD9DF807307F
:1034E00001461BB12A462046FDF72EFD03B030BD34
:1034F00013B50DF107020446FDF7FCFC9DF807200B
:10350000237832B1012B01D9022300E0002303709C
:1035100004E0012B02D90378002BF5D002B010BDD6
:1035200037B504460D46104619460193FDF7D2FC07
:10353000037801993BB96D681A4620462B4603B0C3
:10354000BDE830401847012BF5D0022B2D6842888A
:1035500020460CBF00230123AC4603B0BDE8304039
:10356000604737B50DF105040B46214602F07F0593
:10357000D20904F8015DF9D1091B01AD9847234632
:103580000146AB4205D19DF804201B1BC25403B079
:1035900030BD13F8012B62F07F0201F8012BF0E738
:1035A0004379026A032B11448CBF036B034601620B
:1035B00088BF9B181846704710B50C460121FFF7CD
:1035C000EFFF047010BD4279836A032A19448CBF4F
:1035D000426A0346816282BFD218036B9B18184669
:1035E000704710B50C460121FFF7EDFF047010BDC8
:1035F00013B504460192FFF7F4FF019A03492046F0
:1036000002B0BDE81040FFF7ACBF00BFC735016096
:10361000C36830B415465C8B9A8B038F1444C28EFA
:1036200014445A1C02871A194379042B04BFC36B34
:1036300043F8225030BCFFF7DBBF2833D9B2FFF785
:10364000D7BF38B514460D460321FFF7BCFF4470C1
:10365000240A0570847038BD38B543790D460321BE
:10366000032B89BF846A0024C369C4F1FF2481BF8E
:1036700053F8223004F57F04FD34E418FFF7A3FF6C
:1036800005704470240A847038BD38B543790D46FE
:103690000321032B89BF846A0024C369C4F5FF4456
:1036A00082BF53F822307D34E418FFF78CFF057099
:1036B00044702412847038BDC36810B45A8B9B8B3D
:1036C0001344828E541C1A4443798486042B04BF0D
:1036D000C36B43F8221017215DF8044BFFF788BF36
:1036E00000214020F8F7F4BE10B504460846A16159
:1036F00080000021F8F7D0FEE06110BD10B504464F
:10370000C069F8F7F4FE2046BDE81040F8F7EFBEB8
:10371000F8B5002315464171044683600E46837157
:10372000836203623E49C0E90323012242616B8C3C
:103730002A8C1A44012A38BF0122FFF712FFAA8CF3
:1037400037492046FFF70DFFE3682046197EFFF753
:1037500033FFE3682046997EFFF72EFFE36820469B
:10376000197FFFF729FFE3682046997FFFF724FFC1
:10377000042E2BD12A492046D4E90832D21AFFF769
:10378000F0FE6F8A02212046FFF70AFF07703F0A0A
:103790000221477020462F8AFFF702FF07703F0A79
:1037A000477000272B8DBB4215DCFF212046FFF719
:1037B00018FF0023042EA386238730D16A8BA98BA0
:1037C0000A449A422BDD288D002124E00221204664
:1037D000FFF7E6FED5E7EB6A03EBC70213F83730D5
:1037E000032B03D191782046FFF7FBFE0137D9E781
:1037F000EA6A02EBC1025678F6070BD556889E425C
:1038000008D15268D200E16B42F0060241F8232051
:103810000133D3E701318842EADC4B22F2E7F8BDFD
:10382000A135016010B543790446012B1DD000215C
:10383000FFF7C2FEA38EE3866379032B16D1A36A3A
:103840000021206AE36260621844F8F741FEE368F1
:1038500020630021588B9B8B1844A38E1844238F20
:1038600018448000F8F734FEE06310BD042BFCD14F
:10387000E068E26B037E216B4069BDE8104001F017
:103880000AB88079003818BF012070474379012BAE
:1038900009D083681944C36881605A8C9142C8BFBB
:1038A000598400238371704770B51D460121064677
:1038B0001446FFF7EBFF45B90F2C06D8A4F15001D1
:1038C000BDE87040C9B2FFF78CBE05F11901224670
:1038D0003046C9B2BDE87040FFF78ABE70B51446E5
:1038E0000E4601211B34FFF7D1FF3246E1B2BDE89D
:1038F0007040FFF7A6BE70B51D464FF0FF3106467B
:103900001446FFF7C3FF45B90F2C06D8A4F14001B8
:10391000BDE87040C9B2FFF764BE05F1220122463E
:103920003046C9B2BDE87040FFF762BE70B51446BC
:103930000E464FF0FF312434FFF7A8FF3246E1B2C4
:10394000BDE87040FFF77DBE70B514460E460021FD
:103950002A34FFF79BFF3246E1B2BDE87040FFF723
:1039600070BEF7B5DDE90876C91AD4B243EA07227A
:103970000546A1EB470101925EB10239FFF786FFD0
:10398000611C019AC9B2284603B0BDE8F040FFF7B8
:103990002FBEFFF77BFF019A2146F4E7264B2DE966
:1039A000F047D3F8DC3004468946022B0ED846692E
:1039B0008E420BD2856A8E1B036940F2FF77ED1AA7
:1039C00056EA050304D1A36AC4E90439BDE8F087C7
:1039D000062E01D90F2D1AD91F2DAA4628BF4FF048
:1039E0001F0A554510D8032EB04628BF4FF00308D4
:1039F00001212046FFF7D4FD4AEA48130370A5EBE6
:103A00000A05A6EB0806DBE74FF00008F0E7BE4228
:103A1000B0464FF00201204628BFB846FFF7C0FD70
:103A2000AA464FEA181380F8018003F070032B4375
:103A300063F07F030370E2E70004002038B50D4611
:103A40000021FFF723FF4379012B05D0032B9EBFF5
:103A5000826AC36943F8252038BD012A70B505463E
:103A60000E4614460AD11146FFF710FF683432465D
:103A70002846E1B2BDE87040FFF7E3BD4FF0FF31EB
:103A8000FFF704FF022CF1D16A21BDE87040FFF777
:103A9000A8BD000038B50D4601210446FFF7F6FE2B
:103AA000142D09D0152D09D0132D09D11021204630
:103AB000BDE83840FFF795BD1121F8E71221F6E780
:103AC0000249BDE83840FFF7F7BD00BF20CC0460D5
:103AD00073B50C4601210646FFF7D8FE04F110032A
:103AE0003F2B06D8A4F18001C9B2FFF77AFD02B0DE
:103AF00070BD0DF105051421FFF773FD294604F093
:103B00007F00E3B2E4112A4605F8010D601C01288C
:103B1000F5D8013403F0400312D11BB97F2305F817
:103B2000013C951E491B3046FFF74DFD01AC014697
:103B30002B46A34208D19DF804205D1B4255D6E7D1
:103B4000002BEFD00023EAE713F8012B62F07F028D
:103B500001F8012BEDE713B501910121FFF796FE66
:103B6000019A162102B0BDE81040FFF76ABD38B5D2
:103B70000D460121FFF78AFE2946BDE83840FFF7D0
:103B80009BBD012110B5FFF781FE1821BDE8104053
:103B9000FFF727BD70B50E4651001446C1F1010173
:103BA000FFF774FE002C324614BF1F211E21BDE812
:103BB0007040FFF746BD012110B5FFF767FE2021D9
:103BC000BDE81040FFF70DBD012110B5FFF75EFE07
:103BD0003021BDE81040FFF704BD022110B5FFF70A
:103BE00055FE3121BDE81040FFF7FBBC4FF0FF311F
:103BF00010B5FFF74BFE3221BDE81040FFF7F1BCD6
:103C0000002110B5FFF742FE3321BDE81040FFF759
:103C1000E8BC38B50D460446114642B9FFF736FEFA
:103C20002A461D212046BDE83840FFF70ABD022A7A
:103C300004D1FFF7A6FF2046FFF7E2FF6FF0010176
:103C40002046FFF723FE2A462621EBE7002110B588
:103C5000FFF71CFE3421BDE81040FFF7C2BC10B5D1
:103C6000044649B94FF0FF31FFF710FE21212046ED
:103C7000BDE81040FFF7B5BC022904D1FFF781FF72
:103C80002046FFF7E3FF6FF002012046FFF7FEFD3D
:103C90002721ECE713B501910021FFF7F7FD019A09
:103CA000352102B0BDE81040FFF7EFBC37B50D4637
:103CB0004FF0FF3101920446FFF7E8FD019A35B15C
:103CC0003621204603B0BDE83040FFF7DEBC372187
:103CD000F7E737B50D464FF0FF3101920446FFF785
:103CE000D5FD019A35B13821204603B0BDE83040FA
:103CF000FFF7CBBC3921F7E773B5164605460C46EE
:103D000021F40042F6B931460192FFF7BFFD14F4E9
:103D1000004F019A0FD03221FFF763FC3221284671
:103D2000FFF75FFC32212846FFF75BFC3221284673
:103D3000FFF757FC019A3521284602B0BDE87040D4
:103D4000FFF7A3BC4621FFF7A0FC2846210A21F07B
:103D50007F013143C9B202B0BDE87040FFF741BCFA
:103D600070B505460E46144652B902213D34FFF7A0
:103D70008DFD32462846E1B2BDE87040FFF76CBCCD
:103D80000021F3E74FF0FF3110B5FFF77FFD412130
:103D9000BDE81040FFF725BC38B50C1E14BF032149
:103DA0000021FFF773FD002CBDE8384014BF472108
:103DB0004221FFF716BC13B501910121FFF766FD03
:103DC000019A432102B0BDE81040FFF745BC6FF0F7
:103DD0000301FFF75BBD002110B5FFF757FD44213C
:103DE000BDE81040FFF7FDBB38B504460D46FFF7B0
:103DF000F2FF14212046FFF74DFE20462946FFF72B
:103E00001DFE0221FFF742FD3E21FFF7EAFB20469F
:103E10006FF00301BDE83840FFF738BD002110B551
:103E2000FFF734FD4521BDE81040FFF7DABB38B598
:103E30000C460021FFF72AFDA4F13001BDE838400F
:103E4000C9B2FFF7CEBB302937B50C461AD031299D
:103E50001BD1012507244FF0FF310190FFF716FD1C
:103E6000A4F129010198C9B2FFF7BBFB019875B114
:103E70000021FFF70BFDD321019803B0BDE83040CE
:103E8000FFF7AFBB01250624E5E70025E3E703B014
:103E900030BD70B514460D46032A04F1500414BF1A
:103EA000C5F101010121FFF7F1FC2A46E1B2BDE8AD
:103EB0007040FFF79DBB6FF0010110B5FFF7E6FC06
:103EC0005421BDE81040FFF78CBB032970B516469E
:103ED0000ED004290FD000240225E143FFF7D6FCC1
:103EE000A219572145EA8202BDE87040FFF780BB66
:103EF00000242546F1E70124FBE738B50C460139DB
:103F0000FFF7C4FC59212246BDE83840FFF770BBDB
:103F100070B50C4615461144FFF7B8FC5A2144EA27
:103F20000522BDE87040FFF763BB38B51343044674
:103F30000D4609D10121FFF7A9FC6A6960212046DD
:103F4000BDE83840FFF764BB4FF0FF31FFF79EFC40
:103F50006A696121F3E770B50D4604990446D6B24B
:103F60000B430ED1C2F10101FFF790FC6A69622197
:103F70002046FFF74DFB31462046BDE87040FFF775
:103F800030BBD143FFF782FC6A696321F0E707B5D4
:103F9000CDE900230B4664220021FFF7E2FC03B0C9
:103FA0005DF804FB07B5CDE900230B4666224FF010
:103FB000FF31FFF7D6FC03B05DF804FB4FF0FF3193
:103FC00010B5FFF763FC01235B218371BDE810404E
:103FD000FFF707BB38B50C464942FFF757FC0221F3
:103FE000FFF7F1FA5C234470037038BD38B50C4616
:103FF0004942FFF74BFCC26804F15D01137EC9B270
:1040000043F004031376BDE83840FFF7EABA042111
:10401000FFF73CBC6FF00201FFF738BC06292DE921
:10402000F74F9DF8305010D8012905D93F2300F8EB
:10403000013B0023037001E00029FAD1012994BF5C
:104040000020012003B0BDE8F08F10EE104A002CD4
:10405000044622DAB4EE400AF1EE10FA1DD6B1EEB3
:10406000400A2D2504F8015BF0EEC07A9FEDC37A7B
:1040700002F0200EF4EE477AF1EE10FA12DD8EF027
:1040800049038EF04605E11C23708EF04E03A570A7
:1040900063700023081A0B70D4E7002DE4D004F8F5
:1040A000015BE1E7B4EE400AF1EE10FA08D74EF0FA
:1040B0004E038EF04105E11C23706570A370E8E7A4
:1040C000002B42F02002B8BF0623672A02D1002B42
:1040D00008BF0123251A10EE106A491B002E01F1BA
:1040E000FF3549D1662A39D15E1C0027AE42BC4655
:1040F0003E46A8BFCB1E66215D1C652923EAE378F6
:1041000040F00D8108F10105B2EE047A00234FF072
:104110002E0B0193019B9D4200F30A81662A40F019
:104120003781AE4240F38881A7B10A214EF0450E97
:104130006770043404F804EC96FBF1F393FBF1F29E
:1041400001FB136601FB12323036303204F8016C89
:1041500004F8022C0023201A237073E75E1DAE4280
:104160004FF00005A8BFCB1F652A114640F0D18053
:104170002B27AC462E46C0E7B6F17E5F70D2DFED4E
:10418000807A0027DFF800824FF0200CB4EEE70AB7
:104190003E46DFF8F8A1F1EE10FAACBF4FF031095E
:1041A0004FF03009B8EC017AB4EEC07AF1EE10FAB3
:1041B000C8BF0AEB070B07F10407C8BF66444FEA04
:1041C0006C0CC4BF9BED007A20EE070A182FE9D1D2
:1041D00010EE107AB7F17E5F27D2B4EEE70AF1EE67
:1041E00010FA1DDB002EB7EE000A14BF2D272B2777
:1041F000662A03D0672A29D1042E27DC672A84F88F
:10420000009004BF06F1FF37DB195F1CAF42A8BF67
:10421000CB1E63B901341D461F464FF0FF3C5AE0E8
:10422000F2EE047A013620EE270A2D27E0E72E2150
:104230001D46023404F8011C3021013E6BD00DB93B
:104240002F46EAE7013D04F8011BF6E78D1F9D426A
:1042500002DC672A61D0CB1F11460025AC464CE733
:104260000027DFF828814FF0200CDFF81C913E4634
:10427000F8EC017AF4EEC07AF1EE10FA98BF09EB8F
:10428000070A07F1040798BF66444FEA6C0C9CBF0D
:10429000DAED007A20EE270A182FE9D1FDEEC07A78
:1042A00017EE907A092FC2BFDFED367A013620EE85
:1042B000270A662A11D1AE4217DA99190131A942AB
:1042C00005DBAD1B012DA5F1020308BF0023F51886
:1042D000B4460027013566210FE7652A05D0672A15
:1042E0000CD0114600252B27B8E78D1F9D4200DC1E
:1042F000CB1F00252B276521AC46FEE61F1DAF42D4
:1043000000DB8B1F9E4201DB6721EBE7711C5B1A10
:10431000DDE72F462DE737467FE72B469CE76729E9
:104320007FF4F2AE002BD6BF01254546A846EBE64A
:10433000FDEEC07A04F1010A17EE903A002BA8BFF7
:1043400003F13009019BB4BF4FF030095FFA89F9DE
:104350009C4584F8009006D1B8F1000F03D004F119
:10436000020A84F801B0F8EEE77A019B5446013363
:1043700030EE670A019320EE070ACBE6FFFF7F7F4E
:10438000F8FF7F3FCDCCCC3DC0AA0460D8AA046022
:10439000F1EE047AB4EEE70AF1EE10FA24DB631EC4
:1043A0004FF030091D7803F1FF3C2E2D2ED0A5F1E2
:1043B000300ABAF1090F2BD901331D78302D13D1F2
:1043C00093F801C0BCF12E0F2FD166292DD02D2FCF
:1043D00083F800C05D7026D1013E08BF2B2721461F
:1043E0008B4224D331211970672A7FF49DAEB8F136
:1043F000000F3FF499AE23461C46013B14F8012CF4
:10440000302AF9D02E2A08BF1C468DE66346C9E73C
:10441000392D02D001351D70CFE798428CF80190FC
:10442000F4D10346C9E70136D9E70134D7E711F8DB
:10443000015C01F80159D3E7F1EE047AB4EEE70A22
:10444000F1EE10FAABDA6FE6012910B5146827D93E
:1044500034F01001037814D1302B1DD14178831C26
:1044600041F02001782903D110211160181A10BDE4
:10447000CCB96F2901D10821F7E7622911D10221B6
:10448000F3E7082C11D1302B0DD1437843F02003F2
:104490006F2B08D1831CE9E7082C04D0022C02D032
:1044A0000CB90A2313600346E0E7022CFBD1302B42
:1044B000F9D1437843F02003622BEAE7044608B5BC
:1044C00031B1054B036000234A6C096803F042FDDB
:1044D0002046F7F7BDFF00BF54BD04602DE9FF473C
:1044E0001E464518019212B1023A222A37D80446D4
:1044F000AC4227463ED214F8010BFAF7CBF98046BE
:104500000028F5D13B782B2B2ED12746E91B3846C6
:1045100001AA0024FFF798FF0744B946A9454B4676
:104520002BD3B8F1000F00D06442640044F00104C2
:10453000BB4209D01F46AF423B4646D218780137EE
:10454000FAF7A8F90028F6D122480FF09DFF019A4A
:104550000146214803F0B0FC3146FFF7AFFF1F488A
:104560000FF092FF00F050FC2D2B04BF27464FF0B8
:104570000108CBE74FF00008C8E719F8012BA2F1BA
:10458000300ABAF1090F09D95F2AC7D042F02002D8
:10459000A2F161011929C4D8A2F1570A0199514524
:1045A000BFD920460CF09EFB28B9019B03FB04A455
:1045B00094EA4403B2D5019B4246E91B03A8039742
:1045C00004F05BFD039B0446B2E7BDD1204604B076
:1045D000BDE8F08713AB046080BE0460F0AA0460FD
:1045E0002DE9F04F2DED028B83B00446914646181D
:1045F000DDF838800193B442254680F02A8128787E
:104600000134FAF747F907460028F4D12B782B2B11
:1046100009D125468246B4420CD300279FED908AEB
:10462000384600978CE02D2B03D125464FF0010A28
:10463000F1E782462B7843F02003692B31D1AB1C84
:104640009E4240F2FE806B7843F020036E2B40F0D8
:10465000F880AB7843F02003662B40F0F280EB1D2E
:10466000EC1C9E421AD9EB7843F02003692B15D13C
:104670002B7943F020036E2B10D16B7943F020038C
:10468000692B0BD1AB7943F02003742B06D1EB7966
:1046900043F02003792B01D105F108049FED718AC5
:1046A00014E06E2B2DD1AB1C9E4240F2CA806B7879
:1046B00043F02003612B40F0C480AB7843F020032B
:1046C0006E2B40F0BE80EC1C9FED678ABAF1000FA4
:1046D00001D0B1EE488AAC4209D0B442234680F002
:1046E0008E8018780134FAF7D5F80028F5D15F48A4
:1046F0000FF0CAFE01465E4803F0EBFB4146FFF7B0
:10470000DDFE0022F2EE046AAC469FED558A1046AB
:1047100011469FED587A0092644614F801EBAEF111
:10472000300BBBF1090F37D802291ED1524B9842EA
:1047300002DC0A2303FB00B0A6425CD802B140426F
:10474000009BB2EE040A034413F1250FBEBFDFED58
:104750004B7A253328EE278A07EE903AF8EEE70ADF
:1047600026F04EF828EE008AB0E7B4EEC78AF1EEE4
:1047700010FA0DD507EE90BA0129F8EEE77AE8EEC7
:10478000267AB0EE678A33D1009B013B0093D3E7D2
:1047900031B9009B0133F9E721B9BEF12E0F03D1E6
:1047A0000121C9E7022916D04EF0200BBBF1650F9D
:1047B00011D1A64250D99CF801102B2905D10CF13A
:1047C0000204B44293D00221B6E72D2912D10CF194
:1047D00002040122F5E7B9F1000F04D04EF0200BDE
:1047E000BBF16A0F09D0BEF15F0FA5D06446A5E703
:1047F0000021A1E70221A4468EE74F469EE77FF401
:1048000076AF57B1F0EE480A9FED150A03B0BDEC44
:10481000028BBDE8F04F02F017BD019B23B1B0EE53
:10482000480ADFED0F0AF1E718EE103A23F0030013
:1048300040F00200A0F1FF4003B0BDEC028BBDE8E8
:10484000F08FBAF1000F3FF452AF2C469FED048A6F
:104850003FE74FF0000AE0E63FF449AF6EE700BFE4
:10486000000000000000807F0000C07F3BAB0460C0
:1048700080BE0460EC78AD6064666606EA1C0802DF
:104880000021102008B5F7F723FE0121027861F31B
:104890000202027008BD03F07F0310B50488DB003C
:1048A00024F47F7443F0020324F003042343C0E99B
:1048B0000112038010BD000010B5044608461146E1
:1048C000237803F00703022B0AD1D4E9012303F074
:1048D000BBFE23889B0608D5BDE8104003F034BF1B
:1048E00002480FF0D1FD00F07FFA10BD55AB046017
:1048F00038B5154611F480720C460CBF1146D5E947
:104900000012FFF7D9FF6209E1B202F008022A445F
:10491000BDE8384002F020BC08B502480FF0B4FDF5
:1049200000F062FA66AB046070B505460C468E185E
:10493000B44200D170BDD5E900039847431C01D1B2
:10494000FFF7EAFF04F8010BF2E738B5044600254B
:10495000D4E900039847421C01D1FFF7DDFF00F0C6
:104960007F0343EAC5150306F2D4284638BDB0B527
:1049700000AF0546FFF7E9FFC31D0446024623F0DA
:1049800007032846ADEB030D6946FFF7CDFF21462F
:104990006846F9F779F9BD46B0BD00002DE9F04F42
:1049A0002DED028B8BB00446FFF7CFFF8046002130
:1049B000F7F772FD4246014607462046FFF7B4FF6F
:1049C00004A804970BF0E8FD04A80BF0E5FD049B98
:1049D00005A85A1C04921A4612F8021B0492DA1C0B
:1049E0005E780433049208EE101A13F8025CCDE9E5
:1049F00004330BF0D1FD049B18440490049B5A1C13
:104A000004921B78FF2BF9D12046B844FFF7AFFF83
:104A100081462046FFF7ABFF059B83F800904FEAE5
:104A20001929059B83F80190059B9870000A059B46
:104A3000D870DDF81090C8452AD820462E44FFF7DC
:104A400084FF81462046FFF780FF834648440021CB
:104A500030448000F7F720FD804600EB86060546CF
:104A6000B54226D14FF0000ACA452BD100255D453D
:104A700068D1FFF705FF044618EE103A4246394662
:104A8000FFF709FF20460BB0BDEC028BBDE8F08FAD
:104A900006A948460BF01AFF012807D12046FFF768
:104AA00066FF89F80100000A89F80200069B994414
:104AB000C1E72046FFF75BFFC00040F0060045F865
:104AC000040BCDE7D4E900039847451C01D1FFF75B
:104AD00023FFC5B2652D33D02046FFF736FF0146D0
:104AE000039006A8F9F70BFA039A08992046FFF7F6
:104AF0001BFF732D0AD0622D0AD1164806A906F0B5
:104B00005FFA0AF1010A46F8040BADE71248F5E72F
:104B1000692D06D100230A22DDE90710FFF7DEFC2C
:104B2000EFE7662D01D0632DD1D1A5F163010023FC
:104B30004A4200934A41DDE90710FFF751FDE0E7E3
:104B40000648DEE72046FFF729FF46F82500013535
:104B50008DE700BF7CD1046018D4046020CC0460D1
:104B600037B5042204460DEB0201FFF7DDFE9DF888
:104B700004304D2B0BD19DF80530032B07D19DF848
:104B80000630022B03D19DF807301F2B04D90748AC
:104B90000FF07AFC00F0B8FF2046FFF7FFFE054655
:104BA000A36820689847284603B030BD78AB0460FE
:104BB0001FB5014601A80DF049FB01A8FFF7D0FF82
:104BC00005B05DF804FB000070B5F9F721F8134C4F
:104BD0000025134B134A04F15C06032104F148003D
:104BE000A5652563C4F8DC50C4E90A350E4BC4E959
:104BF0000E256363C4E9105302F0D6FE012130464E
:104C000002F0D2FE4FF49B724FF4AB71304632F09B
:104C100013F8C4F88C50C4E9026670BD000400208B
:104C2000C0BA0460A0BC046098D60460704700005D
:104C300037B5144DC10004460022E86841F0060172
:104C40000430019131F0F4FF019940B9D5F88C306E
:104C500043B10246181D31F0EBFF019910B14068D5
:104C600003B030BD0022084831F0E2FF0028F6D141
:104C700006480FF009FC22460146054803F01CF9DE
:104C8000F7F7E6FB0004002068DF0460DDAB04609A
:104C9000B0BB04600A4B10B50446D3E90203984246
:104CA00009D0E1000022043041F0060131F0C0FFDC
:104CB00008B1406810BD2046BDE81040FFF7B8BFFE
:104CC0000004002008B5074BD3F88C0008B906484B
:104CD00008BD00223E21043031F0AAFF0028F6D0A2
:104CE0004068F5E70004002028DE0460C000034BA4
:104CF00040F00601986802F0D6BE00BF0004002014
:104D0000C000034B40F00601D86802F0CCBE00BFE3
:104D1000000400207FB5C000074B40F00600CDE93D
:104D2000041201A901900520CDE902330AF00CFC20
:104D300007B05DF804FB00BF74C80460F8B505F067
:104D400039F8002502F0DAFE06467368AB4200D857
:104D5000F8BDB368EF0053F8354074B1042C0CD0A3
:104D6000E4082046F9F72BF803785F2B05D0B368E9
:104D700020463B44596831F07BFF0135E5E708B533
:104D800019B903F032F8F7F763FB03F0A2F8FAE77A
:104D90000EB403B503AA52F8041B019203F032F8D3
:104DA000F7F756FB08B50446F7F756FC30B107484D
:104DB0000FF06AFB01460648FFF7E1FF05480FF0D8
:104DC00063FB224601460248FFF7E2FFF6AB0460B0
:104DD00038BB04601FAC04600146024808B5FFF709
:104DE000CEFF00BFA4B804600146024808B5FFF733
:104DF000C6FF00BFDCBC04600146024808B5FFF7EF
:104E0000BEFF00BF48BA04600146024808B5FFF77C
:104E1000B6FF00BF80BE04600FB407B504AA044803
:104E200052F8041B019202F0EDFFF7F711FB00BFEF
:104E300080BE04600146024808B5FFF7A0FF00BF2E
:104E400008BE04600FB407B504AA044852F8041B56
:104E5000019202F0D7FFF7F7FBFA00BF08BE04602B
:104E600003287FB505460C4607D1084631F004FFFC
:104E7000F0B1354C204604B070BDCA072CD549109E
:104E8000072827D801A353F820F000BF754E016012
:104E9000B94E0160D54E0160D54E0160AD4E016046
:104EA000D54E0160754E0160B54E01600029E0D01D
:104EB000264CDFE70029DDDAB1F1404F05D14FF094
:104EC000804004F0B5F80446D4E74C42640044F056
:104ED0000104CFE7CC43F9E706281BD11C4B0B405C
:104EE000062B08D08B0715D10B689A69194B9A428B
:104EF00010D1486802E0C80831F0A6FE30B903A915
:104F0000204606F0EDF80399F8F772FE400040F0F5
:104F10000104AFE7204601F047F8436973B90E4832
:104F20000FF0B2FA0D4B06462046595D019101F093
:104F300072F8019902463046FFF784FF2146284661
:104F400098470028BFD1EAE7F0B30460F8B30460E3
:104F5000070080FFF1C201604DAC046034DA0460E8
:104F600030B585B00446CDE90221019301F01CF86B
:104F7000056945B103992046AC46DDE9013205B02B
:104F8000BDE83040604705480FF07EFA05462046F0
:104F900001F041F801462846FFF754FF6BAC04606E
:104FA00000231A461946FFF7DBBF00002DE9F04148
:104FB000174C98B00F460646E16806A80291A16812
:104FC000C4E902320391F7F72BFA0546C8B9D6F8BF
:104FD00000803A46314604A8FBF72CFD2B462A46B2
:104FE000414604A8FEF741F9FFF7DAFF0190F7F711
:104FF0000FFA029B0198E360039BA36018B0BDE821
:10500000F081029B0798E360039BA360F7F720FA07
:105010000004002007B50022019101AB0121FFF738
:105020009FFF03B05DF804FB30B455681446003DA3
:1050300018BF0125C5F1020302EB83030A462918B4
:10504000206830BCFFF78CBF73B51C4693070E4633
:105050001546019015D113682E4A934203D16B680F
:10506000236002B070BD2C4A934207D110B100F00A
:105070009BFF06466B68C4E90036F2E7274A934275
:1050800001D12560EDE7DA8840F2D5118A4207D0D8
:1050900040F265118A4203D040F2D9118A421DD1F3
:1050A000019AC2B91E498B420BD01E498B4208D0CF
:1050B0001D498B4205D01D498B4202D01C498B42B1
:1050C00009D100210C20F7F7E7F91A4B8560C0E9F8
:1050D00000362060C5E7C4E90052C2E7164A934291
:1050E000CFD1F268154B9A42CBD00028C9D02846C0
:1050F00004F026FF124B0068984204D111480FF0CB
:10510000C3F9FFF769FE01AB00220121FFF728FF79
:10511000DFE700BF80D9046044D90460F8D9046097
:10512000C4BF046000C004603CC0046078C0046078
:10513000B4C0046030AE0460F0C704606DDE01608E
:1051400074C8046087AC046000232DE9F0410D466B
:1051500007461446C2E9003300F026FF0A2D064632
:1051600002D12060BDE8F0812D2D05D1836A1BB1ED
:105170000F4BC4E90037F5E7F3692BB12246294606
:105180003846BDE8F0411847B06B0028EAD0E90086
:105190001A46043041F0060131F04AFD0028E1D002
:1051A0002346426831463846BDE8F041FFF74CBF20
:1051B000F8DE046037B5154604460091FFF7C4FFDA
:1051C0002A68009BE2B9A2070ED121680D4A9142DC
:1051D0000AD10D480FF058F9009B0146E2880B48B0
:1051E00002F06AFEF7F734F9094801930FF04CF921
:1051F0000090204600F00FFF0246DDE90013EEE7C5
:1052000003B030BDF8D904609CAC0460A4B804605D
:10521000C3AC046007B56A46FFF7CCFFDDE90001C7
:1052200011B903B05DF804FB01F030FFF9E70000AD
:1052300030B595B005461C4602A8CDE90021F7F728
:10524000EFF8DDE9002130B92846FFF77DFFF7F7D9
:10525000DFF815B030BD002CFBD1039B0449186862
:1052600008F0F0FF0028F4D10398F7F7F1F800BF39
:10527000A4B804602DE9F0478AB005460C4600AF9B
:1052800007F10C02FFF760FF3B693BB12C480FF0C0
:10529000FBF8224601462B48FFF77AFDF868002804
:1052A0004AD128460AF02CFB0028EFD007F10C0267
:1052B00028462A21FFF748FF07F10801F86806F0A1
:1052C00013FD78602046F8F775FDD7F808907968E7
:1052D00009F101064A468519EB1D23F00703ADEBE2
:1052E000030D6B46E84618464FEAD30A31F038FC06
:1052F0002E234644204609F83A30F8F760FD7860DE
:105300002046F8F757FD79680246304631F028FC10
:1053100029464046F8F7B8FC0B4BC00007F11401D2
:10532000C7E90633094B40F006003B620123786170
:1053300005207B620AF008F92837BD46BDE8F087F2
:10534000E5AC0460D0B9046074C80460F8B30460CC
:1053500073B504461E460D4661B11868019200F00F
:1053600023FE6368019A834204D006480FF08CF84C
:10537000FFF760FD33462946A06802B0BDE87040E3
:10538000FFF7EEBDFBAC04607FB504460E46154644
:1053900000F00AFEC369C3B1042231462046CDE9BC
:1053A000022502AA9847029B002B34D01E480FF01A
:1053B0006BF80190204600F02EFE3346024601991C
:1053C0001A4802F079FDF7F743F8806B0028EDD01A
:1053D000F1001A46043041F0060131F029FC0028A2
:1053E000E4D0406810F003020192DFD10168104B55
:1053F0009942DBD1002CD9D004F0A2FD0D4B019ACB
:10540000CDE902454DB980689842CFD002AB2A461B
:105410000121FFF7A5FD04B070BD40689842C5D0DA
:1054200002AB0221F5E700BF13AD0460A4B804602D
:10543000F0C7046074C8046010B5044602F04CFD67
:1054400038B1002320461A461946BDE81040FFF740
:1054500087BD204602F056FD40B905480FF014F80C
:1054600001460448BDE8104002F033BD204610BD9F
:105470003CAD046008BE0460F0B597B01D4606461A
:105480000C46174600F090FD324B984207D12B4650
:105490003A462146304603F063F917B0F0BD826A00
:1054A0002D4B42B19C422ED13046904728600038A7
:1054B00018BF0120F1E79C4225D101AA2D213046D9
:1054C000FFF742FE019B73B901AA40F2CF2130469B
:1054D000FFF770FE039401AA00210120FFF7A4FD4D
:1054E00028600120D9E704A8F6F79AFF014630B9F1
:1054F00001AAFFF799FD2860F6F78AFFF1E7059BFF
:105500002B600220C9E7002CDED1384600F04CFDAC
:10551000124908F097FE01AA70B14FF4B2713046FB
:10552000FFF712FE019B83B101AA21462046FFF737
:105530007BFD28602046B0E740F21B313046FFF784
:1055400003FE019B0BB10397C5E73846FFF774FFD5
:105550002860D6E700C2046074C8046094B904608F
:1055600073B505460C4600F01FFD164B426A064611
:105570009A4225D024B921461020F6F78DFF044623
:10558000736A8BB96A4619212846FFF7DDFD009B37
:105590008BB90D480EF078FF0446284600F03BFD1D
:1055A00001462046FFF74EFC214628469847002832
:1055B000E8D002B070BD2146684603F0D5F9F8E79F
:1055C0002846F6E71566016066AD046037B5044607
:1055D00000F0EAFC856A1DB12046A84703B030BD43
:1055E0006A462D212046FFF7AFFD009B2BB16A468E
:1055F00029462846FFF718FDF0E705480EF044FF5E
:105600000546204600F007FD01462846FFF71AFC34
:1056100082AD046030B5054695B000F0B7FA284673
:1056200000F0C2FC846A2CB12846A04704462046FC
:1056300015B030BD6A462D212846FFF785FD009B39
:10564000ABB102A8F6F7ECFE014630B96A46FFF7A7
:10565000EBFC0446F6F7DCFEE9E7039B0949186812
:1056600008F0F0FD0028E2D10398F6F7F1FE0648B5
:105670000EF00AFF0446284600F0CDFC0146204605
:10568000FFF7E0FB18BD046082AD04602DE9F04F28
:105690002DED028B13688BB008EE103A002868D10C
:1056A00002F104090446C1F307235FFA81F801936C
:1056B0005B0053FA81F1029359F821B009EB8101A3
:1056C0004F68002F59D017F0030056D13968884A27
:1056D000914202D1384602F0E3F9019B4FEA880A71
:1056E0001E187600BBF1000F49D108F1010259469E
:1056F0001644B000F6F7D0FE05460CB10460012454
:1057000005EB840044445246494631F029FA019B96
:1057100009EB0A0105EB8400DA0031F021FA029B63
:105720002344984697B117F0030940F09E803A68E9
:105730006F4B9A4240F0998038464E4602F0DEF9AF
:10574000DFF8B89107467B689E4273D3A8EB04024A
:1057500021462B4618EE100A5208FFF701FC0446BA
:105760002846F6F7C4FE20460BB0BDEC028BBDE820
:10577000F08F02F10809546895E70020ADE71BF0AF
:10578000030F2BD1DBF800205A498A4202D05A4934
:105790008A4223D106AA05A9584600F055FE059B6A
:1057A0000021013343441E44B000F6F775FE054660
:1057B0000CB1046001245246494605EB840031F0E7
:1057C000CFF908EB0400059A069905EB80009200DA
:1057D00031F0C6F9059B43441C4498E708F10402E4
:1057E00000211644B000F6F757FE05460CB10460E0
:1057F00001245246494605EB8400444431F0B0F997
:1058000006A95846FFF7ACFE80464046FFF702FF68
:10581000034600283FF47BAFA64207D8F100284694
:1058200003937600F6F756FE039B054645F82430B1
:105830000134EAE7BB684FEAC60A53F8360090B174
:10584000042810D000EA0903062B01D006F046FD1B
:1058500045F828004FEA8802BB6808F102082A448C
:1058600053445B68536001366DE706AA4FF4097133
:105870003846DFF888B0FFF79DFC002106AA0846ED
:10588000FFF7D2FB0021FFF76BFE81464846FFF78A
:10589000C1FE824600283FF459AF08F1010296424A
:1058A00008D876002846042E38BF0426B100F6F743
:1058B00011FE05460AEA0B02062A03D0504606F0FE
:1058C0000DFD824606AA19213846FFF773FC06AA89
:1058D00000210120CDF820A0FFF7A6FB4FEA8802A7
:1058E00045F828A008F1020813462B445860CDE77C
:1058F00084B70460A0D60460DCC40460070080FFA5
:10590000830770B50C4686B015461BD103681F4A45
:10591000934202D01E4A934214D102AA01A900F078
:1059200093FD019BA3422AD31AD8029B043D03EBAB
:1059300084049C4201D106B070BD54F8042D45F892
:10594000042FF6E702A9FFF70BFE0023064601939A
:105950003046019BA34208D3FFF75CFE0028EAD043
:105960000C480EF091FD21460DE0FFF753FE30B1DB
:10597000019BDA430133224445F82200E7E7064859
:105980000EF082FD0199FFF747FA00BFA0D6046030
:10599000DCC40460C4AD0460A1AD046083072DE9DC
:1059A000F3411546CFB2C1F3072433D103683A4A15
:1059B000934202D0394A93422CD101AA694600F0A1
:1059C00043FD00983B1983425FD80199002601EB03
:1059D0008003A64214D1C01B01EB8701BC00801BD1
:1059E00005EB860803F0DCFF0199424645F82600E6
:1059F0000B19994202F1040208D102B0BDE8F0810E
:105A000053F8042D45F826200136E2E753F8040D3B
:105A10001060EEE70021FFF7A3FD0023804600930E
:105A2000009BBB421AD30021084603F0B9FF06468B
:105A30004046FFF7EFFD0146D8B9B368A34224D32F
:105A400045F82460034605EB8405B168A342A1EB49
:105A5000040112D1304603F0CFFFCEE74046FFF7F6
:105A6000D9FD90B1009BFA1A0133224445F8220077
:105A7000D5E7304603F0D6FCDAE71944F268013383
:105A800052F8212045F8042DDFE705480EF0FCFC14
:105A90000099FFF7C1F900BFA0D60460DCC4046020
:105AA000A1AD0460400008B540F00101024802F0D9
:105AB000A0F9F6F7CDFC00BF28BC046007B5400094
:105AC0006A4640F00100CDE900010221024802F0DF
:105AD00085F9F6F7BDFC00BF28BC0460014602480A
:105AE00008B5FFF74CF900BFECBB04600FB407B575
:105AF00004AA044852F8041B019202F083F9F6F755
:105B0000A7FC00BF64BC04600146024808B5FFF76B
:105B100036F900BF74BB046008B502480EF0B4FC4F
:105B2000FFF762F99470046010B594B0044602A8BF
:105B30000191F6F775FC48B920460199FFF76AFA1A
:105B40000446F6F765FC204614B010BD0399002406
:105B5000014800F08FFAF6E73C9F046082B0024BE8
:105B600001AA1A6002B070470004002082B0034B03
:105B7000186801ABC01A02B0704700BF00040020D3
:105B8000014B5860704700BF0004002008B5FFF7C4
:105B9000EDFF034B5B68984201D3FFF7BDFF08BDE3
:105BA0000004002070B51E46044615469DF81030CE
:105BB00029B123B910480EF067FCFFF73BF9B54255
:105BC00008D1A54216D00D480EF05EFC22462946AB
:105BD000FFF738F9A54205D909480EF055FC291BF5
:105BE000FFF730F9A64205D206480EF04DFC2246DA
:105BF0003146EDE770BD00BF6CAE046095AE046049
:105C0000CEAE046000AF046010B49DF8044011B142
:105C10000968C1F31B1101945DF8044BFFF7C2BF83
:105C20002DE9F74F002406468B461546A046A146AF
:105C30000193DDE90CA7019B9C4206D1B1453FD2FF
:105C400024480EF021FCFFF7F5F8B44210D2BAF860
:105C500002209205F4D409F101095BF824009AF8B6
:105C60000220012A25D131F007F807F8240018E0B6
:105C7000BAF8001000222846C90041F0060130F0B1
:105C8000D7FF90B9BAF80220D30506D512480EF016
:105C9000FBFBBAF80010FFF7D5F8DAF8042047F854
:105CA000242001340AF1080AC5E708F10108406818
:105CB000D5E7022A01D100F0C1FA47F82400F0E745
:105CC0002B68B8EB131F01D20448BAE703B0BDE854
:105CD000F08F00BF46AF04602FAF046067AF046071
:105CE00008B502480EF0D0FBFFF7F8FE85AF046060
:105CF00010B504460846616039B92368A06003F016
:105D0000080343F00103236010BD0021C000F6F733
:105D1000DFFBF2E703684160090103F008038260DA
:105D200041F0070119430160704710B5037804463C
:105D30009B0702D48068F6F7DAFB0022236862F33F
:105D40001F136260236010BD10B5037804469B07E3
:105D500002D48068F6F7CBFB236803F00C0343F012
:105D6000010323600023C4E9013310BD2DE9F04194
:105D70004668044619490022731C31F8025BAB42A5
:105D800006D90132222AF8D103EB530343F001056F
:105D9000E8000021A768F6F79BFB23684FF0000896
:105DA00065603D1D03F00E03A06043F00103236016
:105DB000B04504D13846BDE8F041F6F798BB55F838
:105DC000041C39B1042905D00122204630F030FFEF
:105DD0002B68436008F101080835E9E7C8AF0460A3
:105DE00010B5044608462160002180006160F6F786
:105DF0006FFBA06010BD2DE9F74F036804460F4606
:105E0000924623B912F0010F60D000F063F83946D2
:105E10000620FFF725F822684FEA600B0AF001031D
:105E2000BBFBF2F902FB19B900934D460026A068AE
:105E3000AA0050F8258000EB8501B8F1000F0BD1C6
:105E40001AF0010F42D0002E08BF0E466368B84614
:105E500001336360376033E0B8F1040F17D1002ECF
:105E600008BF0E4601352268B5FBF2F102FB115561
:105E7000A945DCD1009B4BB3002EE7D1204600F0B2
:105E800029F82268BBFBF2F902FB19B9CDE73946C4
:105E90004046019200F078F9019A0028E2D01AF009
:105EA000020F0DD0013520686368B5FBF0F1013BAE
:105EB00000FB11556360A36853F8251021B9995070
:105EC000404603B0BDE8F08F0421F8E74FF000082A
:105ED000F6E70000F8B505680446866800226B1CEA
:105EE000134931F8020B834206D90132222AF8D134
:105EF00003EB530343F001000021374606EB850511
:105F0000206061608000F6F7E3FAA060AF4204D140
:105F10003046BDE8F840F6F7EABA57F8041B002906
:105F2000F4D00429F2D001222046FFF764FFEDE708
:105F3000C8AF046070B500230168994201D1002206
:105F400014E0846854F8232004EB83060133002A0C
:105F5000F3D0042AF1D04568013D4560B3FBF1F070
:105F600001FB103354F8233013B93360104670BD71
:105F70000423FAE710B504468068F6F7B8FA002360
:105F8000C4E90033A36010BD00F00303022B05D168
:105F9000034B0340981F18BF012070470020704733
:105FA000070080FF7047000008B5C307024608D409
:105FB000074B0340062B06D0FFF7E6FF28B9106811
:105FC00008BD0448FCE70448FAE70448F8E700BFC6
:105FD000070080FF6CC3046018D4046034BF046001
:105FE00038B5816804460846FFF7DEFF4369054679
:105FF00005209847E168B1EB600F0ADA49002B6A87
:106000000422A06841F001019847E3680133E3608E
:1060100038BD0020FCE708B5FFF7C6FFC088BDE823
:106020000840F7F7CCBE000037B50D460446019294
:10603000FFF7ACFD30F024FE2846FFF7B5FF83687C
:1060400033B1019A2946204603B0BDE830401847D5
:10605000C2882046024903B0BDE83040F8F7CABB09
:1060600018B004600A4601460148FFF7DDBF00BFD3
:10607000CCE404602DE9F04F83B0044608460E4698
:1060800000AF01F03FFF00283AD00EF01BF9B8B383
:106090003A1D3946304601F093FF3B6883B32C48E4
:1060A000E9460EF0F1F903880733DB08A9EBC303D7
:1060B0009D4669466D460EF079F926480EF0E4F9E2
:1060C00003880733DB08A5EBC3039D466946EA4610
:1060D0000EF06CF920480EF0D7F903880733DB087F
:1060E000AAEBC3039D466946EB460EF05FF92946CD
:1060F0002046F7F7FDFF3D68033D002D0DDACD4644
:10610000022231462046FFF78FFF14492046F7F759
:10611000EFFF0C37BD46BDE8F08F7A685146204648
:106120004FEA850802EB850352F825205B68F8F7F3
:1061300061FB7B6843449A6822B908492046F7F717
:10614000D7FFD9E759462046F8F754FBD4E700BFFC
:106150001DB0046041B0046056B0046090700460EB
:1061600008B50146FFF720FF064A0069904203D0B8
:10617000003818BF012008BD0846BDE8084007F0F8
:1061800041BF00BFA1DD0160884210B5044608D1BF
:10619000FFF7FAFE28B9A20744D12268224B9A429F
:1061A00040D1224B9C4201D1002010BD9942FBD02E
:1061B000E30704D5C807F7D423460C4619461C4B01
:1061C0002340062B1A4B03EA010305D0A20710D186
:1061D0002068184A90420CD1062B05D08807E3D1DD
:1061E0000A68144B9A42DFD12046BDE8104005F002
:1061F00029BD062BD8D08A0703D10A680D4B9A42D5
:10620000D2D02046FFF7D0FE8369002BCCD00A46BF
:106210000220214698470028C6D0074BC31A58428F
:106220005841C2E70120C0E760B5046074C804604B
:10623000070080FF18D40460F8B3046038B5124B2F
:10624000044698421BD0114B98421AD0C20701D580
:10625000401038BD830707D102680D4B9A4203D125
:10626000BDE8384002F028BF0A480EF00DF9054697
:106270002046FFF7D0FE01462846FEF7E3FD00204A
:10628000E7E70120E5E700BFF0B30460F8B304607E
:106290006CC304605FB00460C20705D4830705D1F6
:1062A0000268034B9A4201D102F0FFBEFFF7C6BF5E
:1062B0006CC304600F4A904210B50C4603D1002312
:1062C0000B60012204E00C4A904203D101220A60D3
:1062D000104610BD10F0010202D043100B60F7E72A
:1062E0008107F5D10168054B9942F1D102F0E4FE36
:1062F0002060E6E7F0B30460F8B304606CC30460A8
:10630000174B0246984210B50C4622D0154B9842C6
:1063100022D0C10708D5431000EE103AB8EEC00AEB
:10632000012084ED000A10BD830706D101680E4BE1
:10633000994202D103F01AF8F2E71046FFF724FE63
:106340000028F0D002F1FF4222F0030300EE103AE1
:10635000E6E79FED060AE3E7B7EE000AE0E700BFD5
:10636000F0B30460F8B304606CC304600000000084
:1063700037B501A90546FFF7C3FF50B907480EF02E
:1063800083F804462846FFF746FE01462046FEF7FE
:1063900059FD9DED010A03B030BD00BF77B0046028
:1063A000244B984270B504460D46164603D100238F
:1063B0000B60336070BD204B984204D14FF07E5388
:1063C0000B600023F5E7C30707D5441007EE904A9A
:1063D000F8EEE77AC1ED007AF3E710F0030208D196
:1063E0000168164B994204D102F0C0FF85ED000A06
:1063F000E7E72046FFF7C8FD28B104F1FF4424F089
:1064000003042C60DDE752B922680D4B9A4206D195
:10641000324629462046BDE8704000F0EBBF0948EF
:106420000EF032F805462046FFF7F5FD01462846F6
:10643000FEF708FDF0B30460F8B304606CC30460B9
:1064400060B5046091B0046038B5830704460ED18E
:1064500003680C4DAB4203D1BDE8384007F026B8C5
:10646000094DAB4203D1BDE8384003F0B7BA074845
:106470000EF00AF805462046FFF7CDFD01462846F6
:10648000FEF7E0FCA0D60460DCC40460ADB004609C
:1064900013B50C4601A9FFF7D7FF019BA34206D015
:1064A00004480DF0F1FF019A2146FEF7B5FC02B059
:1064B00010BD00BFD0B00460F0B51F46D30785B053
:1064C00006460D4614460FD554100394039A002A2D
:1064D000BCBF52190392039AF7B1002A18DA0023BD
:1064E0000393039805B0F0BD03A91046FFF7E2FE41
:1064F0000028EBD10E480DF0C7FFF1880546204675
:106500000191FFF788FD019902462846FEF79AFCA3
:10651000AA42E6D90395E4E7002A01DBAA42E0D3C8
:1065200004480DF0B1FFF28801460348FEF730FC45
:10653000FDB0046021B1046048BA0460820701D054
:1065400002F076BD002803DB400040F001007047F8
:1065500002F089BD8307014610B510D102680D4BCA
:106560009A420CD10C4B0340062B06D1C008F7F71A
:1065700021FC400040F0010010BD8068F9E70846AA
:10658000FFF712FD43691BB10520BDE81040184715
:106590001846F1E77CD10460070080FF38B5054656
:1065A000FFF7D8FF50B906480DF06EFF04462846A5
:1065B000FFF731FD01462046FEF744FC38BD00BF21
:1065C00037B1046070B504461546FFF7EDFC036A69
:1065D00033B12A462046984706460DF083FE8EB911
:1065E00055B909480DF050FF05462046FFF713FD49
:1065F00001462846FEF726FC042D01D10348F1E7A9
:106600000348EFE7304670BD58B1046083B10460C1
:10661000A4B1046070470000044B0B60044BC1E957
:10662000013000230846CB60704700BF94C7046068
:10663000E15F016013B504460192FFF7B5FCC36A40
:106640003BB1019A20469847B0FA80F0400902B069
:1066500010BD1846FBE7000008B5FFF7EBFF20B9B7
:1066600002480DF011FFFEF7E5FB08BDD1B1046053
:10667000062806BF480040F00100002070470000D7
:10668000042803D0052808D0002070478A68054BED
:106690000548002A08BF184670478868400040F047
:1066A00001007047F0B30460F8B30460084BC1E91F
:1066B00000300023C1E90233064B02689A4208BF4A
:1066C0004368084604BFC3F317238B60704700BFBD
:1066D000A0B2046074B3046070B50D46017904463D
:1066E000164601F07F010022402008F005FBE26819
:1066F0002A60A36843436B60237903F07F03AB6098
:10670000094B216899420BD194F90430002B01DB2D
:10671000B30707D46368C3F3172300FB0320286083
:10672000002070BD0120FCE774B30460F8B50022BE
:1067300005460E460146402008F0DEFA00210746D5
:106740001020F5F7A9FE0A4A0A4B044605710021FC
:10675000012D18BF1346036043686FF31F23C0E980
:10676000013606FB07F0F5F797FEE0602046F8BD1E
:10677000FCB2046038B304607FB5044601220846C9
:1067800001A9FFF769FF00222179402008F0B4FA3F
:10679000029D63680646B5FBF0F5B5EB132FC3F316
:1067A000172219D9A16829444143E068F5F792FE00
:1067B0006368E0606FF31F23636005FB06F20199D5
:1067C000D4E9020300FB063030F0CAF9A36804489C
:1067D0001D44A56004B070BD521B62F31F23EBE79C
:1067E00074C80460F7B5466804460B4636F0FF06E9
:1067F0001FD1324601910179402008F07DFA62688C
:106800000821054661F31F22A168083162604143F7
:10681000E068F5F75FFE6268A168C2F31722E060E6
:1068200001FB05573146013A38446A4330F0C0F95C
:10683000019B2079D4E9022108F064FDA368044893
:106840000133A3606368A3F58073636003B0F0BD98
:1068500074C8046030B44268C36891688B420AD23D
:1068600014795D1CD1688268C56004F07F001A4409
:1068700030BC08F01DBB002030BC70472DE9F0474C
:10688000044686B00D4616460AB90025B6E011F05A
:1068900003078068DFF8F89140F0C6800B68754AFE
:1068A000934240F0C1806A4607F024FE20B9724846
:1068B0000DF0EAFDFFF712F92179042E3A464FF068
:1068C000400001F07F0100F0818008F015FA16F019
:1068D000030205464CD133686849186A88423AD1A8
:1068E0003179402001F07F0108F006FAA84204D077
:1068F00063480DF0C9FDFEF787FA33684B45D6E9CA
:10690000028A04D17368C3F3172305FB03AA236823
:10691000E6684B45DDE90007A0EB0707474429D1AE
:1069200094F90430002BB0DA002FE1D16368C3F38F
:10693000172305FB036605FB08F2514605FB0060C3
:1069400030F00EF90199A2680098521A05FB016116
:1069500040446A4331E04B4A934209D1012DC7D1EB
:106960002A4603A93046FFF777FEDDE903A8CEE704
:1069700045489DE7002FDEDD6368B7EB132F0BD989
:10698000A168304639446943F5F7A4FD63680646BB
:10699000E0606FF31F2363600098A2684044019990
:1069A0003A4401FB0561121A05FB00606A4330F0AE
:1069B000E5F805FB08F25146009805FB006030F051
:1069C000DDF8A3681F44A760304D17E008F094F984
:1069D000236806464B4515D139461020F5F75CFD76
:1069E000054694E80F0085E80F00009A02EB11239A
:1069F00063F31F216960019B9B1AAB60284606B0B8
:106A0000BDE8F087DDE900312079C91AFFF78EFE75
:106A1000E1680546C068DDE90032D21A06FB0311C1
:106A2000724330F09DF8E9E700232A4601462068CA
:106A3000FFF742FD236802464B4511D16368042EDF
:106A400000EB13220ED094F90430002BBFF61DAFDB
:106A500020793346E16800F07F0008F053FCB3E78B
:106A6000042EF5D12079E16800F07F0008F020FACB
:106A70000546C3E7D0CC046000B204607D680160C5
:106A800031B204607CD1046052B2046074C8046006
:106A900074B304601A28F0B5064689B00C46154652
:106AA00074D009D80E2800F09A8010282AD0022825
:106AB00000F0B380002453E01C2823D02E28F9D105
:106AC000012205A92846FFF7B5FD002800F09180B6
:106AD000A20740F0A08022685A4B9A4240F09B8067
:106AE000012202A92046FFF7F7FD0123DDE902019B
:106AF0000093DDE9052304F01BFA002800F08B80E9
:106B0000514C2DE015F0010206D115F00303D1D14F
:106B100029684E4A9142CDD12846FFF78FFB0122CA
:106B2000054605A92046FFF7D7FD102E069F1AD16E
:106B300000222179402008F0DFF8A3686B4300FBB6
:106B400003F1E068F5F7C6FCA368E0606B43A3605F
:106B500063686FF31F23636015B1013DC31997B9D3
:106B6000204609B0F0BDA1689DF81C006943FFF7FD
:106B7000DDFD0446C368F2E718463A4605992FF052
:106B8000EFFF03463B44013DF6D2E9E702A90122AB
:106B90002046FFF7A1FD05A928460122FFF75CFD6D
:106BA00000229DF81010402008F0A6F8069EA1686B
:106BB0000546B6FBF0F69DF810003144FFF7B6FD30
:106BC0000446C068DDE902122FF0CAFFE068039BAB
:106BD00006FB05F2059918442FF0C2FFC0E70A68CA
:106BE0001B4B9A423FF466AF29462046FFF7C4FD8F
:106BF000B6E7EB0706D415F0030306D12A68134B5A
:106C00009A4208D10020FEF769FF022B03D1114BF5
:106C10002B40062BF6D1104CA2E7012202A92046F8
:106C2000FFF75AFD012205A92846FFF703FD0028BA
:106C3000F1D0069B30460093059BDDE9021207F078
:106C4000E9FC5AE738B30460F8B304606CC304602D
:106C500074B30460070080FFF0B3046001282DE9DD
:106C6000F043074685B00E4608D08B0724D10B6849
:106C7000254A934202D0254A93421DD1012201A9FF
:106C80003046FFF7D7FCB8B100223946402008F063
:106C900033F8029E0546B6FBF0F638463146FFF75C
:106CA00045FD06FB05F204460199C0682FF058FF28
:106CB000204605B0BDE8F0833046FFF74BFC0546A3
:106CC00000B1451029463846FFF730FD0021044643
:106CD0003046FEF745FC4FF0000806463046FEF70A
:106CE00099FC03460028E3D025B919462046FFF752
:106CF00079FDF3E708F101094246E1683846C846E4
:106D000008F000FBEAE700BF7CD1046038B3046000
:106D100073B50D4600261446194601220223284663
:106D20000096FEF771FF206804F0C6FF012D007881
:106D300005D1314602B0BDE87040FFF7F7BC61688D
:106D400002B0BDE87040FFF789BF0000F7B50B79CE
:106D500005460C46012B10D11B490193F7F7C8F9E2
:106D6000019B2846D4E9022104F03AF81749284645
:106D700003B0BDE8F040F7F7BBB91A461449F7F77E
:106D800039FDA368002BF1D00026124F1249284686
:106D9000F7F7AEF9A368B34204D810492846F7F7CD
:106DA000A7F9E3E71EB139462846F7F7A1F93246BD
:106DB000E1682079013608F07BF801220146284677
:106DC000FFF732F9E6E700BF75B20460E0880560BE
:106DD00081B20460CD0406608CB2046028C00560F6
:106DE00030B50C4685B015460022194620460123D1
:106DF0000092FEF709FF34B92146012005B0BDE835
:106E00003040FFF793BC2968CA070BD48B0703D126
:106E10000A680D4B9A4205D0012005B0BDE830400C
:106E2000FFF71CBF0846FFF709FA0146039001204F
:106E3000FFF77CFC0446039A0021C0682FF0B8FEDF
:106E4000204605B030BD00BF6CC3046070B5064677
:106E50000D46102000211446F5F71EFB044A06716A
:106E600002604268C4606FF31F22C0E9012570BD53
:106E700074B30460F0B5084687B0194600260123B4
:106E8000154600961A46FEF7BFFE012203A92868A0
:106E9000FFF7E2FB9DF81440049F32462146402054
:106EA00007F02AFF039AB7FBF0F12046FFF7CEFF69
:106EB0000322044603A92868FFF7BCFB18B1237915
:106EC00063F07F032371204607B0F0BD37B50D4650
:106ED000019001460120FFF729FC0446019A29464A
:106EE000C0682FF03DFE204603B030BD136870B57A
:106EF0006BB94468A51C50F825509C4207D055F842
:106F00002360B14204D1023350F82330136070BDC6
:106F10000133F2E72DE9F04716460025DFF85490DB
:106F20000F4606F10808DFF850A010490446F7F7AD
:106F3000DFF87368AB4205D820460D49BDE8F0473D
:106F4000F7F7D6B81DB149462046F7F7D1F857F8FC
:106F50002520514620460135F7F74CFC012258F810
:106F6000041B2046FFF760F8E3E700BFB5CC0460E0
:106F7000E0880560CD040660B0B304604B680A4643
:106F8000023351F82310FFF7C5BF0979490041F0DA
:106F900001012FF05DBE052805D00979490041F0B7
:106FA0000101FDF75DBF00207047000037B50C46BA
:106FB000154600221946204601230092FEF724FEC2
:106FC0001CB128682FF058FE10B9024803B030BD3C
:106FD0000148FBE7F0B30460F8B30460032A0B79BF
:106FE00005D113B10449F7F783B80449FBE70BB1A6
:106FF0000349F8E70349F6E7309F0460359F0460D2
:107000004BA0046045A004602DE9F84F984602EBC0
:10701000430300AF81465D1C042B8A4616464FEAA7
:1070200085051FD8EB1D4FF0000B23F00703ADEBD8
:10703000030D6C4620462A1FB96A40F804AB2FF0B6
:107040008FFD23464246711C4846FDF789FF0446E2
:10705000BBF1000F02D05846F5F749FA2046BD466D
:10706000BDE8F88F00212846F5F722FA04460028EB
:10707000D8D08346DEE707B5009313460A46D0E929
:107080000101FFF7C1FF03B05DF804FB38B5054609
:107090000C460C200021F5F7FFF9024A8460C0E994
:1070A000002538BD3CB404604068704741607047BB
:1070B00010B5002104460820F5F7EEF9014AC0E9B1
:1070C000002410BD78B404602DE9F04F86680446B2
:1070D00001EB420987B006EB010B0F4615469846B7
:1070E0000BEB420004F10C0A4FEA8909052816D877
:1070F000B600514601A832462FF032FD01AB4A4698
:10710000414698192FF02CFD606801AB2A4659467C
:10711000FDF726FF0446204607B0BDE8F08F0021AA
:107120008000F5F7B9F9A2685146064692002FF0A3
:1071300017FDA0684A46414606EB80002FF010FD7F
:10714000A16833462A4639446068FDF709FF0446C2
:107150003046F5F7CCF9DEE72DE9F041CD1C80464D
:107160000E460021AD0017462846F5F795F9074B66
:1071700004468660A5F10C023946C0E900380C309F
:107180002FF0EEFC2046BDE8F08100BFB4B40460EF
:10719000136853B9B1F5287F08D1436823F003037E
:1071A00043F00203A3F1FF4313607047B1F5FC7F86
:1071B000FBD18368F2E7000030B591ED010A87B09A
:1071C00000230446B5EE400A0D46009367220623CD
:1071D0001021F1EE10FA02A80AD195ED020AFCF78F
:1071E0001DFF02AA14492046F7F704FB07B030BD83
:1071F000FCF714FF02AA11492046F7F7FBFAD5ED78
:10720000027AF5EEC07AF1EE10FA04DAF4EE677A5B
:10721000F1EE10FA03D70A492046F6F769FF00237A
:107220006722102102A80093062395ED020AFCF7BD
:10723000F5FE02AA0349D6E7F0B40460F4B4046092
:10724000F8B40460FAB4046008B500210C202DEDF8
:10725000028BF0EE408AB0EE608AF5F71DF9044A21
:10726000C0ED018A026080ED028ABDEC028B08BD90
:1072700060B5046008B5072805D8DFE800F0052AE6
:107280000404070419360021084608BDD1ED017A2F
:10729000F5EE407AF1EE10FA3AD1D1ED027A1D48BE
:1072A000F5EE407A1C49F1EE10FA08BF0146EBE713
:1072B000D1ED017A91ED027AFDEEE77ABDEEC77A63
:1072C00017EE903A17EE101A4B40590041F00101A9
:1072D000DAE7D1ED020A91ED010AF1EE600AB1EEB2
:1072E000400ABDE80840FFF7AFBF91ED020AD1EDBB
:1072F000017A20EE000AA7EEA70A24F0E7F810EEC4
:10730000103A23F0030141F00201A1F1FF41BBE774
:107310000149B9E7F0B30460F8B3046030B50C4636
:10732000154600221946204602232DED028B85B01A
:107330000092FEF769FCF4B1012C2B6822D09A0769
:1073400043D11968274A91423FD193ED018AD3ED89
:10735000028A6868830740D10268224B9A423CD176
:10736000D0ED027AD0ED010A38EE678A78EEA00AF5
:10737000B0EE480A03E0DFED1C0AB0EE600AFFF74A
:1073800063FF15E0194A18461A40062A05D09907E6
:1073900015D11A6816498A420ED103A9184604F07D
:1073A000A3FC00230399009301231A46FDF718F963
:1073B00005B0BDEC028B30BD0A498A42F8D01846B0
:1073C000FEF7D6FFDFED080AD9E71846DFED068A9B
:1073D000FEF7CEFFB0EE408ABBE7FEF7C9FF70EEC6
:1073E000280AC5E760B5046000000000070080FFC0
:1073F00018D4046043680B60836813607047000012
:1074000010B52DED048B82B004460846B0EE409ACC
:1074100001AA6946B0EE608AFEF7C2FFA01E1E28D0
:1074200000F2D280DFE800F0BBD0D0D0D0D0D0D0F6
:10743000D0D0D0D0101F5F282DD06CD0D0D0D0D0DD
:10744000101F5F282DD06C00DDED008ADDED017A84
:1074500079EE288A38EE278AF0EE480AB0EE680AFC
:10746000FFF7F2FEACE0DDED008ADDED017A79EEAA
:10747000688A38EE678AEFE755480DF005F8FDF7A2
:10748000D9FCDDED017A9DED007AF5EE407AF1EE62
:1074900010FAB5EE407A0ED1F1EE10FA06D14D4851
:1074A0000CF0F2FF01464C48FDF769FCC9EE078A73
:1074B00088EE078AD0E7F1EE10FA06D1B1EE499ACC
:1074C000C8EE278A89EE278AC6E767EEA76AF1EE3B
:1074D000677AE7EE076A87EE266A87EEA67A8DED71
:1074E000006A8DED017ADDED000ADDED017A68EECE
:1074F000678A20EE888AE0EE898AA7EE898AABE760
:1075000028EE080AA9EE090A23F0E0FFB5EE400ACA
:10751000F1EE10FA1AD1DDED017AF5EE407AF1EED6
:1075200010FA11D1DDED007AF5EEC07AF1EE10FA25
:107530000ADBF5EE407A9FED290AF7EE008AF1EEBC
:1075400010FA48FE808A87E72548A9E723F0B4FDB2
:10755000F0EE490AF0EE408AB0EE480A24F0F6FF59
:10756000B0EE409ADDED007A9DED017A27EE899A22
:1075700020EE470AA7EE289AA7EEA80A23F0F4FB0C
:10758000B0EE408AB0EE490A24F06CFD60EE088A45
:10759000B0EE490A24F024FD20EE088A5CE7DDED18
:1075A000007AF4EE497AF1EE10FA0FD1DDED017AAE
:1075B0000C4BF4EE487A0C48F1EE10FA08BF18466E
:1075C00002B0BDEC048B10BD0020F9E70648F7E7D8
:1075D000FFB404602FB50460BCBE0460000000006E
:1075E00048B50460F8B30460F0B304600B4611467C
:1075F000D3ED020A93ED010AFFF702BF044B0B60C3
:10760000037A0B71436808468B600023CB60704798
:1076100000B70460044B886008460B6001230B71BF
:107620000023CB60704700BF00B7046010B5002195
:1076300004460C20F4F730FF024AC0E9002402227D
:10764000027210BD3CB7046008B503799B0702D5F0
:107650000020FDF7EFFB08BD10B50446FFF7F4FF6F
:10766000201DFEF771FB014810BD00BF74C8046007
:10767000042803D0052809D0002070474B6807482C
:1076800033F00F03064B08BF184670474868C0F335
:107690001B10400040F00100704700BFF8B30460C9
:1076A000F0B30460F8B506460D460F68144612B1F3
:1076B0003846FFF7C9FF22466968381D2FF0B8FA2F
:1076C000034608B1406880B9022E07D1022C0AD1C6
:1076D0006968084800F08DFBF4F7BAFEA868012C31
:1076E00000D15860F8BD0448F9E7022C04BF00221D
:1076F0005A60F7E784BA046074C804600122FFF797
:10770000D1BF0222FFF7CEBF0022FFF7CBBF30B5BB
:107710000B688468A34201D300200BE0C268DD003F
:1077200052F833200133002AF4D0042AF2D00B603F
:10773000C068284430BD13B5044600F10C018068D0
:10774000FFF7E5FF60B12379012B0BD0022B0BD0A3
:1077500003686946009343680220019305F082FDA7
:1077600002B010BD0068FBE74068F9E7F0B5174BC1
:1077700004460A7A85B00D46012653F82210F6F722
:10778000B7FC13492046134FF6F7B2FC124B009397
:107790002B7A8DF804306B680293002303936846BC
:1077A000FFF7C9FF054628B90C492046F6F7A0FCAB
:1077B00005B0F0BD1EB939462046F6F799FC012206
:1077C000294620460026FEF72FFCE8E778B704603C
:1077D0009CB50460CD04066000B704609FB50460EA
:1077E000032A2DE9F3470F461A49154604460CBFF4
:1077F000154601254FF00108F6F77AFCDFF85C909A
:107800000023DFF85CA0019301A93846FFF77FFF52
:10781000064630B910492046F6F76AFC02B0BDE8CA
:10782000F087B8F1000F03D149462046F6F760FC17
:107830002A46316820464FF00008FEF7F5FB514616
:107840002046F6F755FC2A4671682046FEF7ECFB09
:10785000DAE700BFA2B5046032FF0460CD04066021
:10786000D107056030B5044685B00025FFF7ECFE72
:1078700001A920460195FFF74AFF30B90B480CF0EB
:1078800003FE01460A48FDF77AFA636802A9103B35
:10789000636003680293436803930423C0E90035DF
:1078A000022005F0DFFC05B030BD00BFEBB5046081
:1078B00084BA0460022873B50E46114609D02E28FA
:1078C0002BD10022301D2FF0B3F9B0B9144802B00B
:1078D00070BD9307FAD11268124B9A42F6D17368C1
:1078E0004A68534033F00F03F0D10C1D019301A9F6
:1078F0003046FFF70CFF054608B90B48E7E70022C2
:10790000296820462FF094F90028DFD04168686884
:10791000FEF73AFC0028EAD1D8E70020D7E700BFFD
:10792000F0B3046084B70460F8B3046010B40C7A58
:10793000012C06D12E2804D149685DF8044BFFF7CD
:10794000B9BF00205DF8044B7047000010B500215E
:1079500004460C20F4F7A0FD024AC0E900240022EE
:10796000027210BD3CB7046010B5002104460C2023
:10797000F4F792FD024AC0E900240122027210BD10
:107980003CB7046010B5002204300C462FF050F9CB
:1079900028B92146034800F02CFAF4F759FD406855
:1079A00010BD00BF84BA0460024B40F8043BFEF7F0
:1079B0009FB900BF84B7046038B500210546102088
:1079C000F4F76AFD04462946FFF7EEFF204638BD6E
:1079D000F8B50C46064600216068FDF7C1FD022E91
:1079E000054660688CBFA6680B4EFEF7B3FD50B924
:1079F000FFF7E2FF0446071D2846FDF70BFE014690
:107A000018B92046F8BD4010F2E7012238462FF0A1
:107A10000FF94660F0E700BF74C8046038B505464A
:107A20008068FFF7C9FF04462B6803606B68C3F3E7
:107A30001B12436862F31F13436003F0FC032A79AF
:107A400002F00102134303712B790279C3F380031F
:107A500063F382020271AA68E968D200C0682FF05D
:107A60007FF8204638BD2DE9F34180460D460020C1
:107A700017461E46FFF7A0FF0446C0F8008005B970
:107A800056B10023009401930DB13B680193324637
:107A90006946681C2FF000F9204602B0BDE8F0816D
:107AA000406800097047022213B50446CDE9000181
:107AB00069461046FFF7F6FD204602B010BD0000F3
:107AC00038B50C461AB9FFF7EEFF0A480DE0042A54
:107AD0000CD1002204302FF0ABF828B9214606481B
:107AE00000F087F9F4F7B4FC406838BD2FF0A4F833
:107AF000EBE700BF74C8046084BA046004307047C8
:107B000013B504464068FDF785FD58B1A368694682
:107B10005A1C5B0043F00103A260CDE90030022053
:107B200005F0A0FB02B010BD30B585B00546084693
:107B300011461A4602AB01930A4B00930223FEF74B
:107B40006FF800210C20F4F7A7FC04460560002123
:107B50000298FDF705FD6060039B2046A36005B019
:107B600030BD00BFC0B70460F0B5164602F07F0715
:107B70008FB0054632060C461AD47B1E012B17D84F
:107B80000B68D888F6F71BF901462846F6F7B0FAD5
:107B9000022F11D124492846F6F7AAFAE3680BB15F
:107BA0005A687AB921492846F6F7A2FA0FB0F0BD13
:107BB000022FEFD0002FF1D03246E168284605F0C1
:107BC000D5FAF3E79B68DB0723D51949206806F04F
:107BD00039FBF0B1E3685A68022A1AD89868322251
:107BE00001A908F069FC034698B1E26828461149EA
:107BF00092685210F6F7FEFDE3685A68022AD5D162
:107C0000D86804F059F80C4902462846F6F7F2FD08
:107C1000CCE7E3685A68012ACED100229968284649
:107C2000FEF702FAC2E700BFD1070560F5C40560A0
:107C300028BC04600CB8046064AC04602DE9F34116
:107C400000240E460746194630464FF6FF7390460D
:107C5000134D22460094FDF7D7FF21461020F4F77C
:107C600027FCA04218BF05462F60AC602EB90D4C12
:107C70002846EC6002B0BDE8F081B71C2146BF0089
:107C80003846F4F715FC04460028F0D0064BA7F15F
:107C900008024146C0E9003608302EF061FFE7E7F0
:107CA0001804002098D60460A0D60460F8B51546E4
:107CB0000F460446D0E90123591991420FD30178A8
:107CC000D9B105F11006C068164401223146F4F717
:107CD0000CFC78B96568A268013D2070AD1A2A468F
:107CE0003946D4E9023018442EF03AFFA2682A44FB
:107CF000A260F8BD6660E060F1E7013AD51AEEE7F0
:107D0000C3685A680AB1986870470148704700BF55
:107D100074C8046070B513688EB005460E461446EC
:107D20004BB1472917D15268294B9A4213D10023EE
:107D3000C38023600FE0B1F5967F01D1C368F8E7F7
:107D40000368244A934208D140F24E32914204D152
:107D5000FFF7D6FF20600EB070BD1F49184606F031
:107D600071FA0028F7D040F2B3139E4201D12846A1
:107D7000EEE740F205339E4214D1EB685A68012ABF
:107D800001D9DB68D5E702B3322201A9986808F06F
:107D900093FB0546C8B12EF02AFF0146284603F0A2
:107DA00047F9D7E740F2BF139E4205D1EB685A6806
:107DB000022A0AD91B69BCE7B6F5E07FCBD1EB6894
:107DC0005A68042A01D99B69B3E7014BB1E700BFA8
:107DD00074C8046018BD046028BC046010B4C46892
:107DE0000023A4465DF8044B604700221146FFF7CC
:107DF000F5BF07B5019101AA0121FFF7EFFF03B01D
:107E00005DF804FB2DE9F04F87B00D4606460021D2
:107E1000102000AF9046F4F74BFBB5F800A00446E5
:107E200000210AF1010A5046F4F742FB4CB92346FF
:107E3000224621463046FFF701FF1C37BD46BDE80C
:107E4000F08F07F1080968B9C4E90200184BD4E9BA
:107E500002102360F5F7CCFE002360604A46012142
:107E6000BC60E7E70123EB46C7F80CA04FF0000A1F
:107E70003B72104BC7F800907B602B880733DB0800
:107E8000ABEBC3039D46C7E904A0694628460CF046
:107E90008DFA424669463846F6F756FBD7E9043272
:107EA00002F803A03B69A3607B69E360DD46CDE790
:107EB00018D40460AD7C01600EB403B503AA52F877
:107EC000041B0192FFF79EFF02B05DF804EB03B0C4
:107ED0007047FFF7F1BF0000830707D10268064B28
:107EE0009A4203D1C268054B9A4202D0044906F077
:107EF000A9B90120704700BFF8D904603D7C01603A
:107F0000E0B8046008B5FEF74FF8BDE80840FFF799
:107F1000E3BF38B504460D46FFF7F4FF18B120461D
:107F2000FEF742F8044629462046BDE8384006F0F0
:107F300089B9000010B50446FEF736F8044BC26854
:107F40009A424FF0000318BF2469A36010BD00BF20
:107F50003D7C01602DE9F041044617461E468846E7
:107F6000FEF722F8154BC2689A4218BF2469A06830
:107F700098B901460C20F4F79BFAA06058B103238E
:107F80006360E388A168D81C01EB8302E08041F8BC
:107F90002380C2E90176BDE8F081E388A588023339
:107FA000AB42EEDB03350122A900F4F79EFA00286C
:107FB000F1D0A388A0600333A380E2E73D7C016099
:107FC00070B5044615460E46FDF7EEFF064BC26837
:107FD0009A4218BF2469A36813B933602B6070BD3F
:107FE000E3883360A368F9E73D7C016073B504461C
:107FF0000A4EA068FDF70EFB019068B16568B542B6
:1080000005D001AB002201212846FCF7A9FF2EF084
:1080100033FE0028EDD0019802B070BD74C8046032
:10802000F7B500260746084619460223154600966E
:108030001A46FDF7E9FD31460C20F4F72DFA0760EA
:108040002B680446314643606868FDF789FAA060F2
:10805000204603B0F0BD000001F1FF4323F003030D
:1080600007EE903A072805D8DFE800F0051D040464
:1080700007041018002108467047F5EE407A0F48B3
:108080000F49F1EE10FA08BF0146F4E7FDEEE77A7A
:1080900017EE901A490041F00101ECE7F5EEC07AC5
:1080A000F1EE10FAE7D5F1EE677A17EE901A21F0AB
:1080B000030141F00201A1F1FF41DCE7F0B30460EC
:1080C000F8B3046030B501F1FF4587B000230446E2
:1080D00025F0030567221021009300EE105A0623B5
:1080E00002A8FBF79BFF02A92046F6F701F82E2114
:1080F00002A82EF065FD68B9652102A82EF060FD8A
:1081000040B96E2102A82EF05BFD18B90249204645
:10811000F5F7EEFF07B030BD5AF9046038B5D1ED80
:10812000000A054690ED000A0C4623F06BF9B5EE07
:10813000400AD5ED006AD4ED007A36EEC06AF1EE61
:1081400010FA86EE277A1DD117EE903A9FED210A9C
:108150009FED216A002B20FE060AB5EE407AF1EE73
:1081600010FA26D1C6EEA77A9FED1B7A17EE903A49
:10817000DFED187A002B67FE877AC5ED007A84ED73
:10818000000A38BDB5EEC00AF1EE10FAF5EEC07A7D
:108190004CBF01220022F1EE10FA4CBF0123002354
:1081A0009A421EBFB7EE006A30EE270A37EE467AD3
:1081B000D3E7FBFE477AF6EE006A37EE677AB4EE55
:1081C000E67AF1EE10FAC4BFB7EE007A77EE877A5E
:1081D000D3E700BF000000000000008070B50E462D
:1081E00086B0002514461946304601232A460095DC
:1081F000FDF70AFD16B3012203A92068FEF71AFA5B
:1082000040B12B462A460095DDE90301FCF7E8F969
:1082100006B070BD206800F00303022B03D1084BA9
:108220000340062BF4D1FEF7A3F810EE103A23F02A
:10823000030040F00200A0F1FF40E9E70148E7E752
:10824000070080FF0200808030B50C4687B00546ED
:1082500003A920468DED010AFEF752F8002800F030
:10826000CD802D2D00F23181DFE815F0EE00FB000E
:108270000801150122012F012F012F012F012F01CC
:108280002F012F012F012F012E003E0045004C0031
:108290005F006D009F002F012F012F012F012F0183
:1082A0002E003E0045004C005F006D009F002F0136
:1082B0002F012F012F012F012F012F012F012F013E
:1082C0002F012F012F01CD00DDED017A9DED037A05
:1082D00077EE877ACDED017A019820F0030040F027
:1082E0000200A0F1FF4089E0DDED017A9DED037A07
:1082F00077EEC77AEEE7DDED017A9DED037A67EE62
:10830000877AE7E7DDED037AF5EE407AF1EE10FAD1
:1083100006D16F480CF0B8F801466E48FCF72FFD07
:1083200003A901A8FFF7FAFED6E7DDED037AF5EE23
:10833000407AF1EE10FAECD0DDED016A86EEA77A14
:108340008DED017AC8E7DDED030AF5EE400AF1EEA6
:1083500010FADED09DED010A23F054F8B5EE400A84
:108360008DED010AF1EE10FA08D1039BDFED5A7A88
:10837000002B9FED5A7A67FE877AABE7B5EEC00A0D
:10838000DDED037AF1EE10FAF5EEC07A4CBF012272
:108390000022F1EE10FA4CBF012300239A429BD039
:1083A00030EE270A8DED010A96E79DED010ADDED1D
:1083B000030AB5EE400AF1EE10FA0DD1F5EEC00A4F
:1083C000F1EE10FA08D5F0EEE07A9FED457AF4EE82
:1083D000477AF1EE10FA9CDDB5EEC00AF1EE10FA24
:1083E0000ED5FBFE607AF4EE607AF1EE10FA07D05B
:1083F0002146DFED390A2020FFF702F807B030BD33
:1084000022F0FEF9CEE7DDED037AF5EE407AF1EEEB
:1084100010FA3FF47EAF03A901A8FFF77FFE019B8E
:1084200004A9022023F0030343F00203A3F1FF4356
:108430000493039B23F0030343F00203A3F1FF43E0
:10844000059304F00FFFD9E79DED017ADDED037A86
:10845000244BB4EEE77A2448F1EE10FA58BF1846E0
:10846000CCE79DED017ADDED037A1E4BB4EEE77AA1
:108470001D48F1EE10FAD8BF1846BFE79DED017A0E
:10848000DDED037A184BB4EE677A1648F1EE10FA78
:1084900008BF1846B2E79DED017ADDED037A114B76
:1084A000B4EEE77A1048F1EE10FA88BF1846A5E757
:1084B0009DED017ADDED037A0A4BB4EEE77A0A48C6
:1084C000F1EE10FAB8BF184698E7002096E700BF13
:1084D00037B50460BCBE04600000000000000080EE
:1084E000FFFF7F7FF0B30460F8B3046001F1FF4346
:1084F00023F0030300EE103A930710B404460AD1A8
:108500001168084B994206D11146DFED070A5DF864
:10851000044BFEF775BF204611465DF8044BFFF78C
:1085200093BE00BF60B5046000000000002313B5D7
:1085300004460093084611461A46FDF733FB63686C
:1085400002B0BDE81040184737B51C460023054669
:1085500008460093012311461A46FDF723FB6B687A
:10856000206803B0BDE83040184737B51C460023EB
:10857000054608460093022311461A46FDF712FBF2
:108580006B68D4E9000103B0BDE83040184737B547
:108590001C460023054608460093032311461A464D
:1085A000FDF700FB6B682068D4E9011203B0BDE859
:1085B0003040184770B51E46037988B00D4603F069
:1085C00001031146828804460093C2F34E02C38819
:1085D00028460391FDF7E6FA2379039913F0010F7A
:1085E0000BD006EB850205A8FDF794FBA36805AA4E
:1085F00031462846984708B070BDA36831462846E2
:108600009847F8E708B507F0DDFF008808BD08B512
:10861000806807F0D7FF07F0D5FF0430BDE80840B9
:10862000FFF7F0BF13B5044608460191FFF7EFFFCF
:10863000019B02460349204602B0BDE81040F6F710
:10864000D9B800BF70BF04602DE9F8430F469146CA
:1086500098460646F0B14568F7B1681C0430002121
:108660008000F3F719FF0D4B044603600C4BDB68E9
:10867000C0F80C80C0E901392EB1AA0006F108014A
:1086800010302EF06DFA17B1043544F825702046ED
:10869000BDE8F8830546DFE72846DFE788BF0460CA
:1086A00000040020F7B546680F46B068CDE90032F7
:1086B00007F080FF0546B06807F084FF07F07AFFF7
:1086C000002100EB4004E81D20448000F3F7E4FEA5
:1086D0000849044601607168C0E9011600210830AC
:1086E00041603946DDE9003207F072FF204603B0F1
:1086F000F0BD00BF00C2046070B50C460546886836
:10870000FFF785FF2346024602492846BDE8704030
:10871000F6F770B8F0C00460183008B550F8083C9F
:10872000834204D103480BF0AFFEFCF783FB1868CB
:10873000196008BD0EC1046008B50248FFF755FB7B
:10874000F3F786FE18BD046010B50021044608202A
:10875000F3F7A2FE014AC0E9002410BD3CC2046048
:108760002DE9F04704460F4690461E46FDF70EFAE7
:10877000E5681DB935602846BDE8F087236904F136
:108780001802DFF898A0934206D157450BD0204835
:108790000BF07AFEFCF74EFB1A6852451BBF002116
:1087A00090461F601960636823B91A480BF06CFE8D
:1087B000FCF72AFB184F4FF00009414604F108006E
:1087C000FA68FB60A261C4F804902EF05DFAFB68C1
:1087D000012805466360A369FB6007D002280CD01E
:1087E0002369C4F80C901B683360C4E723691B68D5
:1087F00033602369C3F800A0BDE7A368986807F059
:10880000D9FEC4F80C9004EB8004A369ECE700BF28
:1088100039C104606FC104600004002074C80460A2
:1088200013B501ABFFF79CFF01280DD00228104CB7
:108830000DD0019BA34218D0BBB101AA01210D4864
:10884000FFF7CCFAF3F704FE019802B010BD0198CF
:10885000FDF7AAFB074905F0F5FC08B90198F1E717
:108860000198FFF74DFA8442F8D10020EDE700BFF0
:1088700074C8046018BD0460022808B50B460CBF1C
:108880004A688A6818680349FFF7CAFF08B9FFF702
:1088900053FF08BD74C8046008B50022FFF7C0FF8D
:1088A00008B9FFF749FF08BD00220149FFF7B8BF2B
:1088B00074C8046007B5124A01AB1249FFF750FFB4
:1088C000012805D0022808D00E4803B05DF804FB4B
:1088D0000D480BF0D9FDFCF787FA0198FDF764FB12
:1088E0000A4905F0AFFC0028EED10198FDF75CFBCA
:1088F000074905F0A7FC0028E6D10198F3F7A8FD89
:108900001CB8046074C804608BC1046094B904602E
:1089100018BD046030B593B005466846F3F780FD96
:10892000014680B92A1D0120FCF77EFBEB68044656
:1089300023F00103023343F00103EB60F3F768FD1A
:10894000204613B030BD0198054A0368934204D015
:10895000044A934201D0F3F77BFD0024F0E700BF07
:1089600018BD046048BA0460044B0B6003684B6098
:10897000436808468B600123CB60704778C204606F
:10898000F0B50C4685B00122606801A9FDF764FED0
:1089900041F27613A568002002999D42019A0C4687
:1089A00007BF01F1FF334FF0FF361346012608BF22
:1089B0009B1814B900F057FB0BE0B0F5800F04F1E1
:1089C000FF3408D341F27610281A18BF012000F0B6
:1089D000ABFA05B0F0BD1F78334447EA0020E8E762
:1089E000F0EEC07A10B5F4EE677A2DED028BF1EE61
:1089F00010FAB0EE408A0FD69FED1B7AF4EE477A5C
:108A0000F1EE10FA0DDD19480BF03EFD0146184855
:108A1000FFF75FFAF3F71CFD16480BF035FDFCF786
:108A2000F3F910EE103A002B12DA33F0004204D0C2
:108A300003F1FF43B3F19C4F0DD8FDEEC87A17EE5A
:108A4000900A400040F001042046BDEC028B10BDAE
:108A5000DB0DDB05EEE700F02DFAB0EE480A044628
:108A60000430F6F7FCF8EFE7FFFF7F7FB4C2046045
:108A700064BC0460CDC2046070B50D4686B00026AB
:108A8000144619462846022332460096FDF7BCF8E4
:108A9000002D3FD0012D2ED12068C30723D410F024
:108AA000030203D101681C4B99421CD01B4B0340AD
:108AB000062B05D06AB903689A69194B9A4214D1FA
:108AC00005A903F011F9002305991A46FBF706FDE5
:108AD00009E0022A09D100F1FF4020F0030300EE73
:108AE000103AFFF77DFF06B070BDFDF7A7FB400011
:108AF00040F00100F7E705A9206803F0F5F80599B3
:108B0000054660680391FDF799FB334602460399D9
:108B10002846DBE70120E6E76CC30460070080FF1E
:108B2000F1C2016038B50A4C214411F8015CB0FB78
:108B3000F5F55BB16C1C0320B4FBF0F410460AB1F0
:108B40002EF055F803352C44204438BD1C46F5E77B
:108B50005CC3046013F0010F2DE9F74F07468B4605
:108B60009DF838409DF83CA00092DDE90C8640D08D
:108B70005D1045D44FF0000953463246414620204F
:108B8000FFF7D0FFDBF800300246834207D2002116
:108B90000190F3F781FC019A3860CBF80020D7F8F8
:108BA00000B000230BEB020101F8013C65B3013971
:108BB000A4F10A0E0846AC46441EB5FBF8F508FBC6
:108BC00015C3092B8CBF7344303300F8013CBAF154
:108BD000000F30D0C4451BD3A34519D20B1B032B68
:108BE00005D1841E00F802ACA34511D221462046CF
:108BF000E1E7CDE90E4A03B0BDE8F04F00F06AB9F5
:108C00006D424FF02D09B7E730238C1E01F8023C6E
:108C1000CEB1304601922DF0EAFF201A019A834529
:108C200011D2013E014616F8013F4BB90446B9F195
:108C3000000F0DD10FE0A345EAD2C445D7D2E7E734
:108C400001F8013BEFE7B9F1000F04D05C4502D910
:108C500004F8019C013C3868009B02442046121B2A
:108C6000013A1A6003B0BDE8F08F30B510228DB024
:108C700004460B460692002208AD06A9019205A8FB
:108C80000595CDE902220A22009207AAFFF762FFAA
:108C900001462046F5F72CFA0598A84201D0F3F7D3
:108CA00026FC0DB030BD00002DE9F34104460E4610
:108CB0001546CF00DFF8888042B3012000F0B8F9F4
:108CC0000190781E00F0B4F9019902460C202DF0B5
:108CD000BFFF21460246074600202DF0B9FF404560
:108CE000054605D015480BF0CFFB3146FCF7FEFEDC
:108CF00039460120FCF7B4F82146024604202DF045
:108D0000A7FF8542EED102B0BDE8F08100F02CF95A
:108D10000028E7DB012000F08BF90190384600F0D5
:108D200087F9019902460C202DF092FF2146024658
:108D300028462DF08DFF8045E4E700BFE6C20460C1
:108D4000F8B3046010B50C4698B13AB9002811DAAE
:108D50000B480BF099FB2146FCF7C8FE032908D805
:108D6000E3005A1E012393405A428242F0DC9842AB
:108D7000EEDA10BD0329FCD8E20001239340F6E7A8
:108D8000E6C204602DE9F0438BB00D460138043192
:108D900003AB01932A4B00930323FCF741FF039C91
:108DA000002C02DA0020FCF72FF8DDF8109041F2D9
:108DB0007616214606A8B9EB06062D689DF81480A4
:108DC00018BF0126F5F79BF8089F22460021384678
:108DD0002DF0EEFEEB0711D4424621462846FFF760
:108DE00063FF3B4622463146284600F0ADF806A90F
:108DF000144802F0E5F80BB0BDE8F0836D10424670
:108E00002146A0462846FFF79DFF042C28BF4FF0BF
:108E10000408002D05DA22464FF0FF3138462DF0C8
:108E2000C7FE41F276133146404699452B4614BFA2
:108E3000A4EB080200223A4406F048F9D7E700BF45
:108E400004C304607CD104601346144A934230B4D6
:108E50000C4603D1012230BC2DF0FABE104A9342D9
:108E600001D10322F7E71C2814D10E4A1A40062A22
:108E70000CD09A070ED11A680B499069884205D028
:108E80000A498A4202D00A498A4203D12246194637
:108E90001C20E0E7002030BC704700BFF0B3046046
:108EA000F8B30460070080FFF1C20160A0D604603F
:108EB000DCC4046010B500211020F3F7EDFA044B78
:108EC000044640F8043BF5F764FE204610BD00BFA1
:108ED0006CC304602DE9F74F05469DF83CB09868D7
:108EE0000E4690461C4600015B46DDE90C9A524650
:108EF0004946FFF717FE33680746834204D2002134
:108F0000F3F7CAFA286037602D6852469DF838306A
:108F10004946201DCDE900B5F6F704FDC8F800006C
:108F2000284603B0BDE8F08F73B50E4605460192A2
:108F3000FFF7C0FF0446019B324629460430F5F78F
:108F400038FF204602B070BD70B504460D46164687
:108F5000002118462DF02CFE324603462946201DDE
:108F6000BDE87040F6F782BCC30706D54010002864
:108F70000DDB14BF012000207047836853B10379D3
:108F800013F0010F14BF4FF0FF30012070474FF076
:108F9000FF3070471846704738B50C46072805D88B
:108FA000DFE800F005151E0407040E260024204605
:108FB00038BD8868144C1549002808BF0C46F6E7F0
:108FC000081DF6F727FC400040F00104EFE7FFF72B
:108FD00071FF211D05460430F5F74CFF2C46E6E7EE
:108FE000FFF768FF211D05460430F5F752FFF5E74E
:108FF0000B79DB07DBD5FFF75DFF211D054604304C
:10900000F5F72DFFEAE700BFF8B30460F0B30460A2
:109010001FB502910390FFF74DFF01210446043074
:109020000091DDE90232F5F7EEFD204604B010BDF7
:1090300090EA40024FEA400302D443F00100704737
:10904000C117FFF7E5BF1FB502910390FFF732FF8D
:109050000021044604300091DDE90232F5F7D3FD2A
:10906000204604B010BD10F0404F03D1400040F046
:10907000010070470021FFF7E6BF2DE9F3410446E8
:109080000E4617469846FFF715FF324605463B4603
:1090900021680430CDF80080F5F740FE23681844BD
:1090A0002060284602B0BDE8F081C30701D540101A
:1090B00070470430F6F7AEBBC30707B503D54010C1
:1090C00003B05DF804FB01A90430F6F7B6FB08B164
:1090D0000198F5E703480BF0D7F901460248FBF782
:1090E0004EFE00BFA8C3046064BC04602DE9F043D9
:1090F0000C4607461646E1072DED028B89B02AD5AE
:109100000DF108086310022201A902A8F5F76EFD0F
:10911000F20723D502AD7310022201A902A8F5F7C8
:1091200065FD1E2F01D0122F4AD16B68002B76D01F
:109130004046F6F7D7FBB0EE408A2846F6F7D2FB5A
:10914000C8EE007A17EE900A20F0030040F002000B
:10915000A0F1FF4428E004F10408D9E716F0030267
:1091600005D13268784B9A4210D1351DD9E7022AD1
:109170000BD1764B3340062B07D04046F6F7B2FBB7
:1091800031463846FFF760F80DE09AB93268704B07
:109190009A420FD14046F6F7A5FB3146DFED6D0A46
:1091A0003846FEF72DF90446204609B0BDEC028B87
:1091B000BDE8F083324621463846FFF745FEF2E728
:1091C000A7F109095FFA89F3242B00F28F80FFF7DA
:1091D00071FE0446B9F1170F75D8DFE809F0454B69
:1091E0003F51510C12181E743468454B3F51510CBD
:1091F00012181E7434682A4641460430F5F732FFCF
:10920000D2E72A4641460430F5F764FFCCE72A4608
:1092100041460430F6F700F9C6E76B6833B94E48AB
:109220000BF032F901464D48FBF7A9FD05A8F5F70B
:10923000B0FC2B46424605A9201DF6F7A4F905A867
:10924000F5F7ACFCB0E76B68002BE8D005A8F5F7A4
:10925000A0FC2B464246211D05A8EEE72A464146C2
:109260000430F5F777FF9FE72A4641460430F5F7CB
:10927000EFFF99E72A4641460430F6F763F893E793
:109280003046FFF719FF021E04DA35480BF0FCF8F0
:10929000FBF7BAFD182F04F10400414601D00C2F52
:1092A00002D1F5F72FFE7FE7F5F786FE7CE76B68C6
:1092B0001BB12B78DB073FF560AF2A464146201DE6
:1092C000F6F722F970E76B68002BA8D0FFF7F2FDE4
:1092D000211D06462B4642460430F6F754F905A9EF
:1092E0000220CDE9056403F0BDFF5CE72946404656
:1092F000F5F795FD042F24D8DFE807F0030A1D10C9
:109300001600184B184C14EA200438BF1C464BE7D3
:10931000144B154C0028D8BF1C4645E7114B124C86
:109320000028C8BF1C463FE70E4B0F4C34EA200410
:1093300028BF1C4638E70B4B0B4C002818BF1C46B7
:1093400032E7002430E700BF6CC30460070080FFF1
:1093500060B504600000000037B50460BCBE046066
:10936000ECAD0460F0B30460F8B304600430F6F7C9
:10937000B9BA0000044B0B60044BC1E90130002373
:109380000846CB60704700BF94C7046091930160AA
:10939000D0E9022391688B4237BFD268002252F88D
:1093A0002320013338BFC360104670470C4970B5A5
:1093B00004F0D4FF8368002203EBD3719B004910B3
:1093C0009142A3F1040301DC064870BDC468E6586D
:1093D00054F8225044F822600132C468E550EFE7A7
:1093E000DCC4046074C8046010B5044608460A4929
:1093F00004F0B4FF042C03D0052C08D0002010BDCD
:109400008268064B0648002A08BF1846F7E78068BE
:10941000400040F00100F2E7DCC40460F0B30460F7
:10942000F8B3046038B50D46104904F097FF0446C0
:10943000D0E901138B4211D3C900C068F3F74AF891
:109440006268A36800215200E0606260D21A0133B2
:10945000013A00EB830092002DF0AAFB0448D4E906
:109460000232591CA16042F8235038BDDCC40460AC
:1094700074C8046038B5044608460021FCF770F84B
:1094800005462846FCF7C6F80146204601B938BD16
:10949000FFF7C8FFF5E70000F8B50C46114907468D
:1094A000164604F05BFF836861100546384648BFE6
:1094B000C91821EAE1740C499C4228BF1C46FFF7F9
:1094C000B1FFAB68013BE9689C4203DB064841F809
:1094D0002460F8BD01EB830252F8042C41F82320EC
:1094E000F0E700BFDCC4046074C8046038B5002530
:1094F000084904F033FF102104468560C068F2F784
:10950000E9FF042310222946E06063602DF050FB40
:10951000014838BDDCC4046074C804602DE9F84F0C
:1095200081460F4690469A46FCF730FBB94501D379
:10953000BDE8F88FA9F1040B3D68B8F1000F04D025
:1095400029464046FBF766FD05463E460BF10404FE
:10955000A64209D92168B8F1000F18D12A46002087
:109560002DF076FB824510D0043EB44224D2B8F1EF
:10957000000F11D13268294600202DF069FB824589
:10958000F2D02368326822603360A346DEE74046AB
:10959000FBF740FD0146E1E731684046FBF73AFD45
:1095A0000246E8E731463E46534642464846FFF704
:1095B000B5FF3746D946B9E73A680BF1080B23687F
:1095C00022603C1B3B60A6EB0903A410013CB4EBFA
:1095D000A30FE7DC5846534642463946CB46FFF7D1
:1095E0009DFFE6E730B585B00C460138043102AB8B
:1095F0000193114B00930223FCF712FB0F492068E3
:1096000004F0ACFE8168012913D90D4C01F18041B1
:109610009DF80C500B4B0139C068029A002D08BF11
:109620002346094C00EB8101A24208BF0022FFF74C
:1096300075FF054805B030BD00C40460DCC404609B
:10964000F8B30460F0B3046074C8046013B50C464A
:1096500001900649206804F081FE2346019AD0E972
:10966000021002B0BDE8104005F056B8DCC404603A
:1096700070B50D4606461E49286804F06FFE8168E5
:10968000044621B91B480AF0FFFEFBF7B5FB012E8B
:109690004FF00003006814BF6A684FF0FF32FCF718
:1096A0000BFFA268E368013A53F8205003EB8001F6
:1096B000A260121A043103EB800092002DF05EFAD2
:1096C0000021D4E9022343F82210616804290CD94F
:1096D000A368B1EB430F08D94908E0688900F2F7A5
:1096E000F9FE6368E0605B086360284670BD00BFF8
:1096F000DCC40460ECC3046007B5CDE90001694631
:109700000220FFF7A3FF694601900220FFF7B0FF98
:10971000014803B05DF804FB74C8046007B501910B
:10972000054904F01BFE019AD0E9021003B05DF870
:1097300004EB05F027B800BFDCC404602DE9F0415C
:10974000032A4FF00006DFF84C800F460F491446FD
:1097500005460CBF14460124F4F7CAFCBB68B342AB
:1097600005D828460A49BDE8F041F4F7C1BC1EB14E
:1097700041462846F4F7BCFCFB682246284653F8CD
:1097800026100136FCF750FCE8E700BF8EB20460FB
:1097900028C00560CD04066073B511F003060346CA
:1097A0000D4636D109681D4A914232D1019104F02B
:1097B000D5FD04460199284604F0D0FDA1688368D0
:1097C000054619446368994213D90431E068890059
:1097D000F2F780FEA368E060AA681A44043262606F
:1097E000A9680B443146D21A00EB830092002DF099
:1097F000DFF9AA68E9689200D4E9020303EB80006C
:109800002DF0AEF9A368AA681344A360044802B01F
:1098100070BD29461846FFF72DFEF7E7DCC404604B
:1098200074C8046038B504290B4B04460D46036028
:10983000084638BF0420C4E9010100218000F2F786
:109840002BFE6268E0600021521B00EB8500920055
:10985000BDE838402DF0ACB9DCC4046038B5002157
:1098600005461020F2F718FE04462946FFF7DAFFF6
:10987000204638BD2DE9FF410C46384E054690463E
:109880003146204604F06AFD1A2D074624D005D83B
:10989000042D49D90E2D42D000243CE01C2DFBD1D3
:1098A00003A94046FCF706FD0446002833D0039B7D
:1098B000B868002BBCBF00230393039904F0F6FDA6
:1098C000FFF7CCFFC368044604210093BA68039BEA
:1098D000F86804F0FBFD1EE018F00304DCD1D8F8B2
:1098E0000030B34217D1D8F8083080681844FFF729
:1098F000B5FFBA680446F9689200C0682DF030F9E7
:10990000B868E368D8F80820D8F80C1003EB80009A
:1099100092002DF025F9204604B0BDE8F0814146C3
:109920002046FFF739FFF6E718F0030F03D1D8F808
:109930000030B34203D0022DAED1094CEBE7D8F88A
:1099400008300093D8F80C30D0E90221284604F002
:1099500095FE0028F1D0034CDDE700BFDCC40460B5
:10996000F0B30460F8B3046030B5002585B0084654
:10997000144619462A46012300950390FCF744F942
:10998000039820B905B0BDE83040FFF767BF28460F
:10999000FFF764FF216805B0BDE83040FFF76ABDFE
:1099A00038B50C460546FFF759FF4CB938BD54F899
:1099B0002310C26842F823100133AB42F7D1F5E718
:1099C0000023FAE7044908B504F0C8FCBDE80840E4
:1099D000D0E90201FFF7E4BFDCC4046038B50D46EE
:1099E0000449144604F0BAFC83682B60C368236002
:1099F00038BD00BFDCC404608160704770B50E469E
:109A00000749154604F0AAFC044600238168324643
:109A10000068FCF751FDE36843F8205070BD00BFBB
:109A2000DCC40460F0B50D46164689B0684904F000
:109A300095FC05F0030704468EBB4FBB2A68654BB7
:109A40009A4225D102AA2946806804F053FD10B934
:109A50000020FCF743F8DDE90201D4E90223451AAE
:109A6000521A03EB800003EB810192002DF086F87F
:109A7000A068E3686FF00302284439466A4303EBA9
:109A800080002DF095F8A3682B44A360524D19E097
:109A900005A90220CDE90545FFF7EAFDF6E7042E0A
:109AA0002DD180680FBB2A684A4B9A421DD105AA66
:109AB000294604F01FFD40B905AAD4E9020104F0CB
:109AC00087FD0546284609B0F0BDDDE90530C01A1E
:109AD000FFF7C4FEE3688268054605999200C068F6
:109AE00003EB81012DF03CF8ECE700232A46014608
:109AF0002068FCF7E1FCE36853F82050E2E7002F10
:109B00005FD12A68334B9A425BD101AA694630463D
:109B1000FCF79AFC05AA2946A06804F0EBFC002893
:109B200096D0059B009A06999D18E0686D1A002D45
:109B300027DDA16863682944994206D98900F2F7B4
:109B4000C9FCA368E0602B446360009A059BA16890
:109B50001344E068EA1A0A440699920000EB810176
:109B600000EB83002DF00AF8E368009A0598920054
:109B7000019903EB80002DF001F8A3681D44A56056
:109B800084E70199920000EB83002CF0E9FF06992D
:109B9000A268059B009E521AE0683344920000EBD5
:109BA000810100EB83002CF0E9FFA068E3686FF00F
:109BB0000302284439466A4303EB80002CF0F8FF87
:109BC000DBE7324629462046FFF718FF5EE700BF75
:109BD000DCC40460D0CC046074C80460F7B50446EB
:109BE000406800210026800004F10C07F2F754FCC5
:109BF00003466168B14206D80022A06803B0BDE800
:109C0000F040FBF7ADB957F8040B0193FBF702FDE9
:109C1000019B054618B143F826000136E9E71846CE
:109C2000F2F765FC284603B0F0BD2DE9F3410D467F
:109C300000248046194628464FF6FF7317460094C5
:109C40000222FBF7E1FFA81C013D21468000F2F74C
:109C500023FCC0F80080456006463B6800F10C0814
:109C60008360A54203D8304602B0BDE8F0810134DC
:109C7000002157F82400FBF773FC48F8040BF0E7C9
:109C800037B51546C900126841F0060144683AB973
:109C9000201D2CF0CDFF08B143682B6003B030BD10
:109CA00023799B071CD50022201D01912CF0C0FFB9
:109CB000019928B142686B689A4201D10023ECE710
:109CC0000F4B9C42EAD10F4CD4F88C3033B90120B1
:109CD0000191FDF771FE0199C4F88C00D4F88C4015
:109CE000686818B92046FDF7DEFEE7E70191F3F753
:109CF000C5F80199024620462CF09EFFDEE700BF22
:109D000064DF04600004002070B5054648680E4614
:109D100000224FF4AB7104302CF08AFFA8B14068E8
:109D200001F0CAFF044670680022A62104302CF01E
:109D30007FFF60B1406801F0BFFF2246034607493C
:109D40002846BDE87040F4F755BD054CEBE72246C8
:109D500028460449BDE87040F4F74CBD54C5046082
:109D6000F5C405606CC50460C000012270B540F008
:109D700006050E4829462CF05BFF4468064694B958
:109D800001210820F2F788FB094B044603600120FB
:109D9000FDF712FEF3F772F82A464FF4AB716060DC
:109DA0002CF04AFF7460204670BD00BF4C040020B8
:109DB000C4C60460406870474160704710B50C46E7
:109DC000C1000122034841F006012CF031FF44603C
:109DD00010BD00BF4C04002037B50C4605466A464E
:109DE0001E212046FBF7B0F9009B43B100216A46D3
:109DF0000846FBF719F921462846FFF7DFFF03B0B5
:109E000030BD000037B5C100054600220B4841F0C7
:109E1000060101912CF00CFF0199044648B9024655
:109E200007482CF005FF044620B141682846FFF79B
:109E3000D3FF6468204603B030BD00BF4C0400204F
:109E40007CC504600048704774C8046037B50024BE
:109E5000054608461946224623460094FBF7D4FEE1
:109E600021460420F2F718FB056003B030BD000066
:109E700007B5820707D10168084A914203D1C26839
:109E8000074B9A4204D007480AF0FEFAFAF7D2FFCD
:109E900001A903F0D3FF03B05DF804FBF8D9046017
:109EA0006DDE016000C704604368184770B5054661
:109EB0000E4610200021F2F7EFFA044695E80F0055
:109EC00084E80F002046E66070BD70B505460E467A
:109ED00010200021F2F7E0FA044695E80F0084E82C
:109EE0000F002046A66070BD70B505460E461020D6
:109EF0000021F2F7D1FA044695E80F0084E80F003C
:109F00002046666070BD000010B586B00446084665
:109F100011461A4602AB0193084B00930423FBF74A
:109F20007FFE00211020F2F7B7FA0460029A426027
:109F3000039A8260049AC26006B010BDD0C7046064
:109F400004307047032A0CBF01490249F4F7D0B826
:109F50006CC804604E80056038B50B680C46064935
:109F60000546DA88F4F746FC216822462846403147
:109F7000BDE83840FCF7CEBF9E82056000F140038B
:109F800010B5C26B0020824202D14FF0FF3010BDED
:109F900053F8044B8C42FAD00130F4E738B513681B
:109FA000054614464BB90068FFF7E8FF431C03D091
:109FB000831C55F82330236038BD02480AF064FA48
:109FC000FAF70AFFB4C804602DE9F34707460C46C8
:109FD0009146C56B98466BB11E68C6F31B1606EB1F
:109FE000040AAA4508D023480AF04EFA52462946E8
:109FF000FAF728FF1E46F2E7A4000021284603F0E6
:10A0000031F9224605460834494640F8087B2CF0D1
:10A01000A7FD28190024B20000212CF0C9FDA6429A
:10A0200003D1284602B0BDE8F087D8F808304FEADF
:10A03000C40953F8340001F039F80146019038465C
:10A04000FFF79CFF431C019905D10B480AF01CFA4D
:10A050000199FAF7F7FE05EB8002936813B1074800
:10A060000191F3E7D8F8083001344B445B68936002
:10A07000D5E700BF95AE0460C8C80460E9C80460B5
:10A08000F8B500F1100407460D460021A400204653
:10A09000403CF2F701FA06463C2200212CF088FDF4
:10A0A0002C44F76306F14007A54201D13046F8BDC4
:10A0B00055F8040B00F0FAFF47F8040BF4E7000032
:10A0C0001FB5019100F0F2FF019B0446164A1A40A9
:10A0D000062A05D09A0708D11A68144B9A4204D16F
:10A0E00001A9012002F0B6FB019003AA02A9019880
:10A0F000FCF7AAF9DDE90201FFF7C2FF0C4AC480B0
:10A1000002600C4A82600C4AC2600C4A42610C4AEE
:10A1100082610C4AC2610C4A02620C4A42620C4AD9
:10A12000426304B010BD00BF070080FF18D4046074
:10A13000F8D90460599F0160C99F016009D201608C
:10A14000A1D201609D9F016099D3016051D101604E
:10A15000A0D60460C268002A05DDD0E90113994247
:10A1600006DB00230AE0FCD0D0E901139942F8DDB8
:10A1700041684B000A4443F00103426018467047AF
:10A1800010B5D0E90142C3680348C1E90223C1E91F
:10A190000004084610BD00BF7CC904602DE9F341EE
:10A1A0000E460027194680460323154630460122F5
:10A1B0000097FBF729FD39461020F2F76DF90123CE
:10A1C00004469E42C360C0E90087286806D1FCF7B8
:10A1D00035F8A060204602B0BDE8F081FCF72EF80B
:10A1E00060606868FCF72AF8032EA060F2D1A868C6
:10A1F000FCF724F8E0600028ECD102480AF044F9AA
:10A20000FAF702FE20C9046038B50C460546D1E9CC
:10A2100001230949F4F7EEFAE268012A05D128463C
:10A220000649BDE83840F3F763BF28460449BDE856
:10A230003840F4F7DFBA00BF2AC90460E08805603F
:10A2400037C90460042A30B5044685B043D162683A
:10A25000D0E90203801A002B1844CCBF00F1FF3074
:10A26000013011F0030590FBF3F020EAE07024D1F7
:10A270000A681A4B9A4220D101AA04F03BF92946F8
:10A280001020F2F709F9164B0360019BE168626840
:10A2900001FB03234360029BE168626801FB032327
:10A2A00083600399E268002901FB02F2C26002DACE
:10A2B000E2689B1A836005B030BD0A460023014660
:10A2C0002068FCF7F9F8E268636802FB00304000A0
:10A2D00040F00100EFE70020EDE700BFD0CC0460C4
:10A2E00040C90460136810B514463BB940F2F62328
:10A2F000994204D14068FEF79BFE206010BD40F2F9
:10A300000133994201D18068F5E7B1F5407FF5D17D
:10A31000C068F0E7D1E902324968002AA3EB0103E3
:10A320001344CCBF03F1FF330133042893FBF2F352
:10A3300003D0052807D000207047064A0648002BA6
:10A34000C8BF1046704723EAE370400040F00100A8
:10A35000704700BFF8B30460F0B304600346806840
:10A3600040B1411E042258689960490041F0010142
:10A37000FCF728B970477FB5064600240846194601
:10A380000123154600941A46FBF73EFC372102AA2A
:10A390002868FAF7D9FE029941B12146204602AA5F
:10A3A000FAF742FE0446204604B070BD0C20F2F7D6
:10A3B00073F80446066028686060FCF7EFF8FBF766
:10A3C0003DFFA060EFE70000820708D10068064B60
:10A3D000984206D0054BC31A584258417047002096
:10A3E00070470120704700BFB0CA046074CA04609F
:10A3F000044B0B60044BC1E9013000230846CB60DD
:10A40000704700BF94C70460C1A6016001220430F8
:10A4100008B5FBF7F0FC014808BD00BF74C8046034
:10A420000222043008B5FBF7E6FC014808BD00BF76
:10A4300074C8046038B5044608460021FBF790F85C
:10A44000043405462846FBF7E5F8014600B938BD57
:10A4500001222046FBF7CFFCF4E7000070B506466A
:10A460000D460124B44201D3044870BD55F82410B0
:10A4700001342868FFF7DEFFF4E700BF74C804600A
:10A4800038B5044608460021FBF76AF8043405464F
:10A490002846FBF7BFF8014608B9034838BD032238
:10A4A0002046FBF7A8FCF3E774C8046030B585B01C
:10A4B0000446084669460434FBF752F80546284628
:10A4C000FBF7A8F8014610B9054805B030BD0022D9
:10A4D0002046FBF790FC0028F1D00248F5E700BFCA
:10A4E000F8B30460F0B3046038B5044600211020CE
:10A4F000F1F7D2FF2368054640F8043B6168FBF79B
:10A500006FFCA368E868AB606268E16892002CF0B9
:10A5100027FB284638BD13B50191FFF7E5FF044638
:10A520000199FFF787FF204602B010BD13B50191D6
:10A53000FFF7DAFF04460199FFF7A2FF204602B0B9
:10A5400010BD0000043008B5FBF714FD004808BD3D
:10A5500074C804602DE9F84307460E460C681AB922
:10A560002046FFF7C1FF0446012504F10409BD425E
:10A5700002D32046BDE8F88356F82500844204D172
:10A580004846FBF7F7FC0135F1E70021FAF7E8FF51
:10A5900080464046FBF73EF801460028F3D00222F1
:10A5A0004846FBF728FCF4E7012208B5FFF7D2FF85
:10A5B000004808BD74C804600022FFF7CBBF00004C
:10A5C0008A072DE9F84304460D4611D10E68214B48
:10A5D000F31A5E425E41AB6863B91EB11E49204664
:10A5E000F3F786FD1D492046BDE8F843F3F780BD2B
:10A5F0000026F0E71EB11A492046F3F779FD194904
:10A600002046F3F775FD00270123DFF864806A68B0
:10A61000BA4206D814492046F3F76AFDC6B1134979
:10A62000E1E7EA684FEA870952F8272072B1042A65
:10A630000CD01BB941462046F3F75AFDEB680122C6
:10A64000204653F80910FBF7EFFC00230137DEE743
:10A65000BDE8F88374CA04601D710460F4C9046025
:10A66000FAC90460A2B5046032FF0460E0880560A6
:10A67000CD04066010B5022204300C46FBF7BBFB8C
:10A6800028B921460348FDF7B4FBF1F7E1FE024883
:10A6900010BD00BF84BA046074C8046008B50430FB
:10A6A000FBF748FC30B9044809F0EEFE01460348C8
:10A6B000FAF765FB08BD00BF05CA046084BA0460F0
:10A6C00030B58268C3685468A34201D300200BE010
:10A6D000D1689D0051F8231001330029F4D00429DA
:10A6E000F2D0C360D368585930BD00000528F8B5D2
:10A6F0000D460AD006280DD0042825D18A681348B3
:10A70000134B002A08BF1846F8BD8868400040F087
:10A710000100F9E711F0030016D10E680D4B9E42BF
:10A72000F2D14F680446A74201D17000EFE7EB6811
:10A7300053F8241031B1042904D00620FAF790FB15
:10A7400006EB60060134EEE70020DDE7F8B30460B5
:10A75000F0B3046074CA0460F8B505460C461020D6
:10A760000021F1F799FE0B4B0746294604EB8505BE
:10A77000064647F8043B3846FBF732FBAC4201D1B2
:10A780003046F8BD012254F8041B3846FBF733FB72
:10A79000F4E700BFB0CA04602DE9F3410F46002181
:10A7A000054616460846FFF7D7FF002104463846FF
:10A7B000FAF7D6FE05F1040807463846FAF72AFFED
:10A7C000014670B94EB1E868F1F791FE63686B60BD
:10A7D000A368AB60E368094CEB60204602B0BDE8BB
:10A7E000F081002240460191FBF705FB019900280A
:10A7F000E3D02046FFF70AFEDFE700BF74C804601D
:10A80000814202D00122FFF7C7BF0148704700BF55
:10A8100074C80460814201D1FFF766BE0022FFF7D1
:10A82000BBBF01220430FBF7E6BAF7B50C460025A2
:10A830000646174619462A46012320460095FBF78F
:10A84000E3F944B921462046FFF786FF0446204637
:10A85000266003B0F0BD29462846FFF77DFF294654
:10A8600004463868FAF77CFE05462846FAF7D2FE19
:10A8700001460028EBD02046FFF7D3FFF5E70000A4
:10A880002DE9F04186B016460446CDE90010FFF7E9
:10A890009BFD0346002835D101AA0121204801274C
:10A8A000FFF7C3FF0446009D2846FFF78DFD0346D2
:10A8B00050BB6A4601211A484FF00108FFF7B5FF67
:10A8C00005461EB1A268AB689A4226D0154B2E1DD4
:10A8D0000293154BCDE903340023059302A8FFF73B
:10A8E000EFFE014698B9114E17B1201DFBF742FB50
:10A8F000B8F1000F02D0281DFBF73CFB304606B034
:10A90000BDE8F0810027CEE74FF00008D9E700222C
:10A910003046FBF770FA0028E0D1054EE4E700BFAF
:10A92000B0CA046094C70460C1A60160F8B30460B3
:10A93000F0B304600B46002201461846FFF7A0BFA3
:10A940000022FFF79DBF0000F0B585B01746064610
:10A950000C46CDE902128A0721D10D683F4BEB1A54
:10A960005D425D412E2E01956CD03846FFF72CFDDF
:10A9700000286FD01B2E6DD8019A1B2E6AD8DFE8F5
:10A9800006F0494F53575C69696969202D3469693C
:10A99000694469696969692810156969691B002535
:10A9A000E0E739462046FFF7C1FD03E0394620467F
:10A9B000FFF730FF044609E002A90220FFF7FCFD83
:10A9C000F8E735B102A90220FFF748FD204605B09F
:10A9D000F0BD39462046FFF79EFDEBE7394620469D
:10A9E000002DE0D0FFF74CFDF0E7BC4205D1002D73
:10A9F000ECD12046FFF778FDDCE720463946FFF72B
:10AA0000CBFE002D08BF0446E0E702A90220FFF7B5
:10AA1000A1FDCFE7012239462046FFF731FFC9E704
:10AA2000012221463846F8E7A268BB689A420FD156
:10AA300039462046FFF784FFBCE739462046FFF73A
:10AA400079FFB7E700223946201DFBF7D4F918B982
:10AA5000034CBBE70024B9E7024CB7E7B0CA046077
:10AA6000F0B30460F8B304604A680149F3F7C2BE6A
:10AA70009E820560CB0770B586B004D4254809F0E6
:10AA800003FDFAF7D7F94C1004D5234809F0FCFC74
:10AA9000FAF7BAF903230122059343680193836807
:10AAA000CDE9032102931D49C3688B420CD043FAC0
:10AAB00002F20593002A23DA631E5B0043F00103D0
:10AAC00003934FF0FF33049301AD002003AE55F81C
:10AAD000043B8B420DD05B1017D51B1915D5002AEE
:10AAE000CCBF002301235B425B0043F0010346F827
:10AAF000203040B103A9032002F0B4FB06B070BDC2
:10AB0000E2D10748C2E70120E1E7A342A8BF2346FC
:10AB1000EAE700BF64CC04607ACC046074C80460C7
:10AB200096CC046070B504460D46104E1049F3F7FC
:10AB3000DFFA012269682046FBF776FA31462046A3
:10AB4000F3F7D6FA0122A9682046FBF76DFA3146E1
:10AB50002046F3F7CDFAE96820460122FBF764FAB4
:10AB600020460449BDE87040F3F7C2BACD04066040
:10AB7000B0CC0460E088056010B413682BB940F2D3
:10AB8000F623994204D1436813605DF8044B704783
:10AB900040F20133994201D18368F5E7B1F5407F76
:10ABA00001D1C368F0E740F2FF139942EDD113469B
:10ABB0000168024A5DF8044BFAF746BA0CCD04600E
:10ABC00070B506460D46102000211446F1F764FCCE
:10ABD000024AC0E90254C0E9002670BDD0CC04602E
:10ABE00037B50D461946104B1446834204D00F4822
:10ABF00009F04AFCFAF772FF00232846012200936D
:10AC00000323FBF701F8012D206807D1084A01460C
:10AC1000104603B0BDE83040FFF7D2BF032D616896
:10AC20000CBFA268024AF4E7D0CC0460B7CC046041
:10AC300074C804602DE9F8432C4B8146C0680D466A
:10AC40001646984698421DD0FBF7F8FA071E04D125
:10AC5000274809F019FCFAF7D7F814DCD9F80400F2
:10AC6000404533D16C1ED9F80800404538D0FBF779
:10AC7000E5FA0028B8BF401940EAE070A84232DB8C
:10AC8000013D1CE00127D9F8040040451CD0FBF72A
:10AC9000D5FA041EB8BF641924EAE474AC42A8BF14
:10ACA0002C46D9F80800404509D0FBF7C7FA002820
:10ACB000B8BF401920EAE0708542A8BF0546B760DA
:10ACC000C6E90045BDE8F8830024EAE7FBF7B6FAD9
:10ACD0000028B8BF401940EAE074AC42C2DAC2E7CB
:10ACE0004FF0FF35EBE70546E9E700BF74C80460A5
:10ACF00096CC046010B544680C6081681160C2682D
:10AD00001A6010BD10F0030203D10168084B99428C
:10AD100009D010F0010306D13AB90068054BC31AF7
:10AD2000584258417047012070471846704700BF8D
:10AD300000B404606CC3046010B50446FFF7E2FF82
:10AD400048B904F00303022B04D10448204006381C
:10AD500018BF012010BD0120FCE700BF070080FFE5
:10AD6000044B0B60044BC1E9013000230846CB6063
:10AD7000704700BF94C7046053BB016008B5FBF780
:10AD800013F9C488084809F07FFBB4F5417F0146F8
:10AD900022460CBF4FF4AA734FF441730348FDF7EA
:10ADA0008BF8F1F755FB00BF14CD046008BE0460BA
:10ADB000884230B513D20378303B092B0FD80023DB
:10ADC0000A25136010F8014B1368303C814205FBE3
:10ADD0000343136003D00378303B092BF2D930BD15
:10ADE0002DE9F84F98468F1804460D460B46002271
:10ADF0009F4217D8002A0CBF27262226DFF89C90F6
:10AE00003246DFF89CA02046DFF898B01F49F3F7E0
:10AE1000F1FCBD4210D3324620461C49BDE8F84F34
:10AE2000F3F7E8BC13F8011B272903D02229DFD14F
:10AE30002726E3E70122DBE715F8012BB24205D113
:10AE4000324613492046F3F7D5FCE2E75C2A04D1E9
:10AE500010492046F3F74CF9DBE71F2A08D97F2A6F
:10AE600012D0B8F1000F01D013060DD40749E9E75D
:10AE70000A2A01D10849ECE70D2A01D15946E8E731
:10AE8000092A01D15146E4E74946DBE7AE86056071
:10AE90003FCD046043CD046046CD04604FCD0460D7
:10AEA0004CCD046049CD04602DE9F8430D461646AB
:10AEB000184F04462E44DFF87080DFF87090164972
:10AEC000F3F716F9AE4205D820461349BDE8F8431A
:10AED000F3F70EB915F8012B222A01D05C2A04D110
:10AEE00039462046F3F786FCECE71F2A01D90B49C7
:10AEF000F7E70A2A04D10A492046F3F7F9F8E1E70F
:10AF00000D2A01D10749F7E7092A01D14946F3E79C
:10AF10004146E6E73FCD046056CD0460AE8605604D
:10AF200046CD046049CD046058CD04604CCD04602A
:10AF300099422DE9F047DDF820A0804691461E4653
:10AF400013D3BAF1000FA1EB0304CEBF00252546B1
:10AF5000002408EB05073246494638462BF0F2FD3F
:10AF600020B1A54201D05544F3E700273846BDE89B
:10AF7000F087F8B5074615460E4610200021F1F778
:10AF80008BFA04460760856086B129463046F2F7A1
:10AF90002FFE00216060681CF1F77EFA2A463146D8
:10AFA000E06007462BF0DCFD00237B552046F8BD12
:10AFB00008B5F2F769FEC00040F0060008BD0000C9
:10AFC0001A4B984270B506460D460FD1D1E90110D3
:10AFD000F2F72AFE044648B1E4002846F2F7B2FF31
:10AFE000002344F006042B60204670BD0021102091
:10AFF000F1F752FA0660696804468160A868F2F7C2
:10B00000F7FD606069682B680131994208D1AB682F
:10B01000E3600023D4E902218B54AB602B60E3E7AB
:10B02000A868F1F757FAE060F3E700BF18D40460AE
:10B0300013B504460191F2F7F7FD019A20B1C00063
:10B0400040F0060002B010BD2146034802B0BDE842
:10B050001040FFF78EBF00BF18D404600A460146B7
:10B060000148FFF786BF00BF7CD104600346084655
:10B070001146034A9A4201D1FFF7DABFFFF7EEBF4C
:10B0800018D404607FB50146019002A8F2F737FF9B
:10B09000019A002104982BF08BFD02A90248FFF7CA
:10B0A0008FFF07B05DF804FB7CD1046008B50A4B44
:10B0B0000340062B01D1C00808BD830709D10268EF
:10B0C000064B9A4205D1D0E90210BDE80840F2F7DC
:10B0D000DBBDFFF753FE00BF070080FF18D40460FC
:10B0E000054A0240062A02D1C008F2F76DBE826806
:10B0F0000A60C068704700BF070080FFF0B50D46CA
:10B1000089B00646144619462BB11B6833F00F036D
:10B1100001D0FAF7E5FD0027032328463A460097B9
:10B12000FAF772FD002D57D0012D10D1102102AA7F
:10B130000DEB0100F2F7FAFE216802A83A46FAF791
:10B1400073FF04A93046FFF73BFF09B0F0BD20684C
:10B15000830732D10268214B9A422ED102A9FFF710
:10B16000BFFF1F4B054620680340062B12D1C008C5
:10B170002BF06AFD044624B902992846F2F738FDFF
:10B18000044602992846F3F7EAFB28B9002115483E
:10B19000F9F7F5FD4468EEE702992846F2F744FD19
:10B1A000014618B1C00040F00600CEE7029A3046D2
:10B1B000FFF7DFFEC5604460C7E704A90122FBF783
:10B1C0004BFADDE90401F3F7CAFB0028DED0DDE924
:10B1D0000401FFF72DFFB8E70E20B6E77CD104602D
:10B1E000070080FF44BE0460012807B50A4606D167
:10B1F0000B686A460220009340F2E6230193014661
:10B2000000230348FFF77AFF03B05DF804FB00BF9B
:10B2100018D404602DE9F04304468BB00191FAF78D
:10B22000C3FE02A906462046FFF75AFF019A0746C9
:10B23000314B12F0030F05D112689A4209D02F4901
:10B240008A4206D0DC6801AA002301212A48A047CF
:10B2500001900024DFF8AC8004AA03A925460198D8
:10B26000FBF7F2F8039BA3420FD8294606A8F2F792
:10B2700046FE0025089C039BAB4226D806A9304613
:10B28000FFF79EFE0BB0BDE8F083049B4FEA8409F4
:10B2900053F82400FAF788FE864204D0184809F0D3
:10B2A000F3F8F9F7C7FD0CB1029B1D44049B53F85A
:10B2B000090000EA0803062B05D1C008F2F77AFD61
:10B2C00005440134CEE78068FAE735B12046029A9A
:10B2D00039462BF045FC029B1C44049B05A953F8FE
:10B2E00025000135FFF7FCFE059A014620462BF0AC
:10B2F00037FC059B1C44BEE7DCC40460A0D6046098
:10B300005FCD0460070080FF2DE9FF4102AB0C46D2
:10B310000138043101931E4B00930123FAF780FC9E
:10B320002068FAF741FE002180460846FEF738FB08
:10B3300003A905462068FFF7D3FE039E0146064495
:10B34000B14203D3284604B0BDE8F0810B461A7819
:10B350001C4601330A2A19D00D2A12D163780A2B10
:10B360000CBF022701279DF80830621A03B13A4446
:10B370004046FFF77BFE01462846FEF753F8E119E9
:10B38000DEE79E421C46E2D10027ECE70127EAE710
:10B3900058D104602DE9F04F87B00D468246086809
:10B3A000CDE90223FAF700FE07466868FAF7FCFDCC
:10B3B000874202D06868FFF7E1FC04A92868FFF71C
:10B3C0008FFE05A904466868FFF78AFE049ABAF161
:10B3D000020F834604EB02082FD92149AB68894646
:10B3E0008B4228D0012138460091214601F0A8FC6B
:10B3F0000646BAF1030F0AD0EB684B4507D001228D
:10B40000214638460092049A01F09AFC8046B045E5
:10B410000AD3029BA8EB06015A4630460093059BCF
:10B42000FFF786FD014650B9039BB3B10D4809F003
:10B430002BF8F9F7E9FC2646DBE72646E7E70A4B57
:10B440009F4208D12046F3F708FA400040F001007F
:10B4500007B0BDE8F08F001BF7E74FF0FF30F7E7CC
:10B4600074C80460A4CD046018D4046000230122D1
:10B47000FFF790BF00234FF0FF32FFF78BBF012390
:10B480001A46FFF787BF01234FF0FF32FFF782BF55
:10B490002DE9F04F8BB00C46164603901068FAF772
:10B4A00083FD012C074633D07068FAF77DFD874293
:10B4B00002D07068FFF762FC09A97068FFF710FE00
:10B4C000099B0490059309A93068FFF709FE039BC7
:10B4D000DDF824900024012B0790CB46A2460BBF39
:10B4E0004FF0FF33012309F1FF350025A0460CBFC3
:10B4F00006930693BBF1000F0FD1BAF1000F1DD1D7
:10B500001D4B1E489F4208BF0E200BB0BDE8F08FB8
:10B51000062305931A4B0493D5E70123079ADDE927
:10B5200004012A440093FFF703FDA8B9BAF1000F04
:10B5300017D1039B4BB909F1FF34A846621CA2EB5B
:10B540000802914511D13068DFE7039B2C46012B9F
:10B5500009D0A8464FF0010A069B0BF1FF3B1D44A2
:10B56000C8E72C46F8E7D046E8E7079B384643444F
:10B570001946FFF77BFDC8E718D404606CD104605E
:10B58000C8D304600A4601460220FFF781BF0A467D
:10B5900001460020FFF77CBF0A4601460120FFF765
:10B5A00077BF70B586B00C46054601A9FFF798FD38
:10B5B00006462046FAF742FE019B0446834217D214
:10B5C000014602A8F2F79BFC2246202104982BF0AA
:10B5D000EFFA019A04983146A41A00EB54002BF0BC
:10B5E000BFFA2846FAF7E0FC02A9FFF7E9FC054696
:10B5F000284606B070BD04282DE9F04F0C462DED0D
:10B60000028B8FB01AD1C868FAF718FE28B92068E3
:10B610000FB0BDEC028BBDE8F08F40EAE07320680C
:10B620000293FAF7C1FC03906068FAF7BDFC039B34
:10B630000546984205D06068FFF7A0FB4FF0FF3346
:10B64000EDE7A068FAF7B0FC854201D0A068F3E707
:10B6500007A92068FFF744FD08A904906068FFF778
:10B660003FFD09A908EE100AA068FFF739FD8346DF
:10B67000DDE907329A42CAD80026DDE907535BBBF1
:10B6800026B1099A594630462BF06AFA099F4FF0C5
:10B69000010ADDF81080029B53450DD065B10122EF
:10B6A000089B29464046009218EE102A0593FFF7A2
:10B6B0003FFC059B814698B926B12A464146F019C0
:10B6C0002BF04EFAE91956BBBAF1000F9FD00AA829
:10B6D000F2F715FC0C9ED0E74FF0000A5746D8E76A
:10B6E0000BB909F10109A9EB080526B12A46414623
:10B6F000F0192BF035FA2F4426B1099A5946F01962
:10B700002BF02EFA089B0AF1010A079D09EB0308AA
:10B71000049B09991D440F44A5EB0805BBE70AA942
:10B720000398FFF74DFC73E72DE9F04F0C4685B009
:10B7300083460868FAF738FC81466068FAF734FCFB
:10B74000814502D06068FFF719FB02A92068FFF766
:10B75000C7FC03A906466068FFF7C2FC029ABBF16A
:10B76000020F804606EB020728D91F49A3688A46C4
:10B770008B4221D0012148460091314601F0E0FA88
:10B780000546BBF1030F0AD0E368534507D00122F9
:10B79000314648460092029A01F0D2FA0746039BCE
:10B7A00003BB791B2846F3F765F80130400040F0F1
:10B7B000010005B0BDE8F08F3546E2E73546EEE71B
:10B7C000414628462BF0BEF938B901343546039A74
:10B7D000AE18BE42F4D96000E9E72846F3F734F822
:10B7E0000646F3E70024F2E774C804602DE9F0414F
:10B7F0000F4688B090460446FAF7D6FB0546384611
:10B80000FAF7D2FB854202D03846FFF7B7FA03A910
:10B810002046FFF765FC04A906463846FFF760FCA2
:10B82000049B024623B9194808F02EFEF9F7ECFAFA
:10B8300017493046CDF800808D420CBF0E211549C6
:10B84000B8F1010F079118BF0794CDE905110399CD
:10B8500008BF0594FFF76CFB88B1841B314628466E
:10B860002246FFF703FCDDE90321CDE90507521A63
:10B8700021442846121B3144FFF7F8FB079005A925
:10B88000032001F0EFFC08B0BDE8F081B8CD046002
:10B8900018D404606CD104600122FFF7A7BF4FF0F9
:10B8A000FF32FFF7A3BF2DE9F0410D4686B00746F2
:10B8B000002401A92846FFF713FC0199064602A8B7
:10B8C000F2F71DFBDDF81080019BA34208D8284643
:10B8D000FAF76AFB02A9FFF773FB06B0BDE8F08137
:10B8E000305DB84708F804000134EDE7014601482F
:10B8F000FFF7D9BF31E9006001460148FFF7D3BF28
:10B9000041E90060F7B50646084601A9FFF7E8FBE4
:10B91000019B074603B3124B9E421FD0114B0024DC
:10B920009E4205D1254612E0385DB047A0B10134F2
:10B93000019BA342F8D80C4803B0F0BD385DF2F784
:10B94000B3FF18B1385DB047054628B10134019BFB
:10B95000A342F3D8002DEED10448EDE70024E1E73F
:10B9600009E900601DE90060F8B30460F0B3046009
:10B9700001460148FFF7C6BF95E80060014601484F
:10B98000FFF7C0BFA9E8006001460148FFF7BABF52
:10B99000BDE8006001460148FFF7B4BF09E9006057
:10B9A00001460148FFF7AEBF1DE9006070B50346D0
:10B9B000424D08680C4690B000EA0501062905D002
:10B9C000820724D101683E4A914220D1023B012BDB
:10B9D0006FD80CA9FFF784FB0646206800EA050231
:10B9E000062A12D1C0082BF02FF9044624B90C996D
:10B9F0003046F2F7FDF804460C9A00213148FFF773
:10BA0000B8FAC660446010B070BD4468EEE710F04C
:10BA1000010513D0421002D50020F9F7F5F91146BF
:10BA20000CA80192F2F76BFA0021019A0E982BF004
:10BA3000BFF80CA92348FFF7C3FAE4E7012B38D875
:10BA400003AA0821F9F780FB039B2BB103AA29461F
:10BA50002846F9F7E9FAD6E7012205A92068FAF79E
:10BA6000E9FD20B1DDE90501FFF7F8FACBE7206831
:10BA7000FAF770FD70B9102108A8F2F72EFA2068C5
:10BA80000CA9F9F76DFD04462046F9F7C3FD18B976
:10BA900008A9CFE74110EFE7FAF7D0FBFF2803D959
:10BAA000094808F0F1FCB8E7C1B208A8F2F7A2FA19
:10BAB000EAE7064808F0E8FCF9F7BCF9070080FF60
:10BAC00018D404607CD10460C8CD0460E1CD04606A
:10BAD0000846114608B52BB11B6833F00F0301D09F
:10BAE000FAF7FEF818B1BDE80840FFF75FBF01485C
:10BAF00008BD00BF6CD10460012807B50BD10B68ED
:10BB000002206946009340F2E6230193FFF74EFFBF
:10BB100003B05DF804FB0028F8D10148F8E700BF46
:10BB20006CD10460012A13B50C460AD101A9FFF7B4
:10BB3000D7FA019B2060002063604223A36002B01B
:10BB400010BD00230120C1E900334FF0FF338B60AB
:10BB5000F5E713B5044601A98068FFF7C1FAE2686A
:10BB6000019B9A4237BF835C002001325B003CBFDF
:10BB7000E26043F0010002B010BD0000F0B50546E0
:10BB800085B017460C46FAF70FFA6946064628466E
:10BB9000FFF7A6FA042F054624D1A307009816D173
:10BBA0002268114B9A4212D101AA214602F0A2FC4E
:10BBB00020B90E4808F068FCF9F790FFDDE90112A2
:10BBC0003046521A2944FFF751FA05B0F0BD01463C
:10BBD000002322463046FAF76FFC285C400040F014
:10BBE0000100F2E70020F0E7D0CC046000B204606E
:10BBF00073B516460446084601A9FFF771FA032EED
:10BC0000054606D10146019A2046FFF74DF902B0DC
:10BC100070BD042E06D10346019A08492046F2F76A
:10BC2000E9FDF4E706492046F2F762FA0123019A9A
:10BC300029462046FFF7D4F8E9E700BFFBCD0460B2
:10BC40007FB204601B4B01EA03020340062B73B56D
:10BC500004460D460CD1062A04D1431A58425841D5
:10BC600002B070BDC0082AF0EFFF0646686805E024
:10BC7000062A4668FAD1C8082AF0E6FF26B118B1AC
:10BC8000B04201D00020EBE769462046FFF728FAD2
:10BC900001A904462846FFF723FA0146DDE90023FF
:10BCA0009A42EFD120462AF04DFFB0FA80F04009C9
:10BCB000D6E700BF070080FF094B0340062B07B5FE
:10BCC00006D083070AD103689A69064B9A4205D1C8
:10BCD00001A9FFF705FA03B05DF804FBFFF74EF882
:10BCE000070080FFF1C201600A4B0340062B13B529
:10BCF0000C4606D083070BD103689A69064B9A421B
:10BD000006D101A9FFF7ECF9019B236002B010BD39
:10BD1000FFF734F8070080FFF1C201602DE9F04F12
:10BD20002DED028B95B09FEDB08A0F4691460490A1
:10BD300008AA10210CA89A46F2F7F8F84F450AD342
:10BD40000CAB049C0FCB84E80F00204615B0BDEC73
:10BD5000028BBDE8F08F3E4616F8011B7D290ED1FF
:10BD6000B14507D979787D2904D10CA83746F2F777
:10BD700041F909E09D4808F087FBF9F745F87B2970
:10BD800004D00CA8F2F736F90137D7E7B14519D935
:10BD900079787B29E9D07D2900F08C82212900F077
:10BDA00089823A2900F0868231460A780B460131B1
:10BDB0007D2A03D0212A01D03A2A01D11D467CE2F6
:10BDC0008945F2D18A48D6E75A1C91451AD95C7840
:10BDD000A4F17202012A15D802339945F2D91A78D2
:10BDE0003A2A40F065825F1C5B787D2B13D0394680
:10BDF000012249450B46E5D211F8010B7B2803D1FE
:10BE00000132F6E77B48B6E77D28F2D1013AF0D15E
:10BE1000B8461F4603E0B945D4D94FF000083B7837
:10BE20007D2B01D07448A6E7002E48D0002330783F
:10BE30001093F2F743FDD8B93346AB429B4605D287
:10BE400013F8012B2E2A01D05B2AF6D1ABEB0601A9
:10BE50003046FFF7ADF800220146059022982AF0FF
:10BE6000E7FE059948BB6548FBF7C3FFF0F7F0FA1A
:10BE7000DAF80030002B01DD61487CE710AA294682
:10BE80003046FEF795FF209A109B8346013A9A426E
:10BE900004D85C4808F0F8FAF8F7AEFF0133219AAD
:10BEA00052F823604FF0FF33CAF80030AB4516D28A
:10BEB000554808F0E9FAF9F711FE4668F6E7DAF8AE
:10BEC0000030002B01DA514855E7209A013A93429D
:10BED000DFD20133219A52F82360CAF80030B8F15A
:10BEE000000F13D114B1733C18BF01240AAA10210A
:10BEF00010A8F2F71BF8314622460AA8FAF794F880
:10BF000010A94348FFF75CF8064601E0002CEAD18F
:10BF10004FF0FF3307930A93B8F1000F00F0AF80A2
:10BF2000F9F734FE229B3A464146029310A8219B22
:10BF30000193209B00935346FFF7F0FE10A8F2F701
:10BF40004AF8119A90F80080034600EB020BB8F112
:10BF5000000F72D0059041462E482AF031FE059B15
:10BF6000002800F09F81013300251A782B2A66D023
:10BF70002D2A66D0202A66D1042401331A78232A78
:10BF800004BF013344F010041A78302A07D1B8F105
:10BF9000000F08BF4FF03D08002D08BF302507AA4D
:10BFA00018465946FEF704FF027803462C2A04BFC0
:10BFB000013344F020041A782E2A04D1581C0AAA0E
:10BFC000FEF7F6FE034693F800B00593BBF1000FB1
:10BFD0003BD0594610482AF0F3FD10B1059B5B7821
:10BFE0009BB30E48C7E600BF0000C84200CE046005
:10BFF00041CE046028CE046059CE046084BA046047
:10C000007DCE0460C7CE0460E0CE0460FDCE046047
:10C0100018D4046047CF04604CCF04605CCF046048
:10C020002946A94805932AF0CBFD059B20B12A4655
:10C0300002334546904698E78046454695E70224F8
:10C040009BE7002499E7002498E710A8F1F77AFF0E
:10C05000B8F1000F08D13046FEF76EFE002814BF7D
:10C060004FF03E084FF03C08002D08BF202514F08B
:10C07000060F0DD0BBF1730F05D194487BE6444603
:10C08000C3464546E7E7BBF1630F01D1904872E62E
:10C09000B8F13D0F2DD0B8F15E0F2DD0B8F13C0FA7
:10C0A00001D144F001043046FEF72CFE002800F0D8
:10C0B0009C80BBF1780F10D8BBF1610F1FD8BBF18A
:10C0C000470F51D8BBF1440F00F28F80BBF1000F36
:10C0D00073D0BBF1250F00F088807E4808F0D4F9BA
:10C0E00004463046F9F797FF594602462046F8F7CE
:10C0F00093FE44F04004D6E744F08004D3E7ABF16C
:10C100006203162BE9D801A252F823F083C1016023
:10C110009DC10160BBC10160EBC10160EBC1016069
:10C12000EBC10160DBC00160DBC00160DBC001600E
:10C13000DBC00160DBC00160DBC00160BBC101602E
:10C14000CDC10160DBC00160DBC00160DBC001600C
:10C15000DBC00160DBC00160DBC00160DBC00160EF
:10C16000DBC001606FC10160BBF1580FB5D1002386
:10C17000102200940393079BCDE90153ABF1170301
:10C1800007E00023022200940393079BCDE90153AB
:10C190006123314608A8F2F77BF8F5E53046FAF757
:10C1A0004DF8079B012210A98DF84000CDE90053FE
:10C1B000234608A8F1F7ACFFE6E500230A22009425
:10C1C0000393079BCDE901536123E2E7E3064FF0B8
:10C1D00000034FF0080248BF44F400740393079B28
:10C1E0000094CDE901536123D3E73046FEF7A4FD67
:10C1F000002837D0BBF1000F23D0BBF16E0F20D049
:10C20000BBF1250F20D0BBF1240F7FF666AFBBF149
:10C21000470F11D8BBF1440F7FF65FAF3046FAF7F6
:10C22000A7F80A9B224659460193079B00932B4689
:10C2300008A8F2F739F9A7E5ABF16503022BEDD9B0
:10C240004BE74FF0670BE9E73046FAF791F80A9BA6
:10C2500020EE080A44F4807201936621079B009344
:10C260002B46E5E7B8F13D0F01D11B4883E5BBF153
:10C27000000F03D0BBF1730F7FF42FAF10A930462E
:10C28000FFF732FD0A9B109A0146002BB8BF0A92B5
:10C290000A9B9A4288BF1093079B109ACDE90053DE
:10C2A000234686E75D78002D7FF4BAAEA8465CE6AB
:10C2B0000027ADE53346002635461A78212A3FF49B
:10C2C00083AD00248BE500BF47CF046075CF0460C9
:10C2D000A1CF0460D4CF046005D0046007B501A9E4
:10C2E000FFF702FD0199FEF763FE03B05DF804FB62
:10C2F0002DE9F04F1F289DB005460C46099240F0ED
:10C300000D8209AB12F0030591460B934FF0010328
:10C310000C9308D11368B44A934207D10BAA0CA915
:10C32000484601F0C3F84FF0000904E0AF4A9342D9
:10C3300018BF4FF000090C9B0DA9204604930B9BDE
:10C340000593FEF7CDFE0690A00718D1A84B2268F2
:10C35000D11A4B424B4110AA102114A80793F1F7B0
:10C36000E5FD069A0D9B0027144602EB0308A04545
:10C3700007D8049BBB4200F0C7819E481FE0002302
:10C38000E9E72178252904D014A8F1F733FE013418
:10C39000EDE7661C464504D3974808F075F8F8F7B2
:10C3A00033FD6178252904D114A83446F1F722FE23
:10C3B000EDE7282932D1B9F1000F04D18F4808F0F8
:10C3C00063F8F8F737FDA01C01460E4616F8013B4E
:10C3D000292B1DD1091A0127FEF7EAFD014648461F
:10C3E000FBF7D0FA05464FF0000B33464FF0200A1A
:10C3F0005E4698451C4613D80023A0450E9336D9B7
:10C4000023782A2B6DD1049BBB4225D87C48D6E7E4
:10C41000884501D17B48C0E73146D6E70025E2E7F1
:10C4200013F8012B2D2A02D146F00106E1E72B2A51
:10C4300002D146F00206DCE7202A02D146F00406CB
:10C44000D7E7232A05D0302AD6D146F040069246B7
:10C45000CFE74FF0100BCCE77B1C01340893059B12
:10C4600053F82700F9F7EAFE089B0E901F464FF09D
:10C47000FF33A0450F938FD923782E2B16D1601C44
:10C48000804589D963782A2B32D1049BBB42BDD920
:10C490007B1C02340893059B53F82700F9F7CEFE66
:10C4A000089B0F901F46A0457FF676AF35B9049BD9
:10C4B000BB42ABD9059B53F8275001372378472B54
:10C4C00066D8442B69D92846F9F752FF0F9B21788B
:10C4D0003246019310A80E9B00935346F1F7E4FFF8
:10C4E00055E720460EAA4146FEF762FC0446BEE729
:10C4F00000230FAA41460F93FEF75AFC0446D2E7E9
:10C50000202A4AD801A151F822F000BFF3C60160E9
:10C510009BC501609BC501609BC501609BC5016017
:10C520009BC501609BC501609BC501609BC5016007
:10C530009BC501609BC50160ADC501603FC6016040
:10C54000C7C40160C7C40160C7C401609BC5016066
:10C550003FC601609BC501609BC501609BC5016032
:10C560009BC501609BC501607BC601609BC50160E6
:10C570009BC5016097C6016097C601609BC50160BD
:10C580003FC601609BC501609BC50160F3C60160A9
:10C59000A3F15802D1B22029B2D91B4807F074FF89
:10C5A0002278069B1146E31AF8F736FC174B2B400E
:10C5B000062B05D0AA072FD12B68154A93422BD101
:10C5C00018A92846FFF790FB189A0146012A01D0C6
:10C5D0001048F4E60E9B019320230093334610A8E5
:10C5E000F1F796FDD3E600BFA0D6046084B70460DF
:10C5F0007CD10460FFD004603AD004604CD0046069
:10C6000079D0046063D00460CAD00460070080FF62
:10C6100018D40460A0D004602846FEF773FB60B114
:10C620002846F9F70BFE0E9B012218A9019320233F
:10C630008DF8600000933346D1E77F48BFE605F0F0
:10C640000303022B0CD17D4B2B40062B08D005F1A8
:10C65000FF4525F0030300EE103AFCF7C1F905464B
:10C660000F9B0A22009603930E9BCDE901A3612341
:10C67000294610A8F1F70CFE89E6BBF1000F01D0A6
:10C6800046F404760F9B0822009603930E9BCDE997
:10C6900001A36123ECE712AA102118A8F1F746FCC8
:10C6A0002378722B0CBF0122002208D0079B33B1E4
:10C6B000AB0704D12B6862498B4208BF042229468C
:10C6C00012A8F9F7B1FC0F9B199A10A8002B0E9B2A
:10C6D000B8BF0F920F99019320238A4200933346EB
:10C6E00028BF0A461A99F1F713FD18A8F1F72AFC9A
:10C6F0004DE60F9A46EA0B06173B03920E9A0096F8
:10C70000CDE901A21022B3E74D4814A94D4B079A79
:10C71000002A08BF1846FEF753FC18E00846F9F750
:10C7200043FC12A906462046FEF7DAFC1C2D0746FC
:10C7300022D114A90998F9F7BDFD40B11499002937
:10C7400008DC4048404B864214BF18460E201DB0FE
:10C75000BDE8F08F129801F0A9FE014618A8F1F784
:10C76000CEFB1A9B012138460093129A149B01F0CC
:10C77000ADFE18A93046CEE70998F9F715FC8642B8
:10C780000FD118A90998FEF7ABFCDDF86090804640
:10C790001A2D22D014D8042D45D90E2D1DD00020DD
:10C7A000D5E7274B09989E4208D1012218A9F9F72D
:10C7B00041FF0028CBD0DDE91889E9E7FEF7DEFA72
:10C7C0002E2DECD1012342461299384600934B4658
:10C7D000FEF7AEFB28BB1D48B9E7129B3BB9099891
:10C7E000F9F7E2FB864202D1099C2046AFE7B9F196
:10C7F000000FFAD0129918A84944F1F780FB129A59
:10C8000039461A982AF0ACF9129B1A984A464146C2
:10C8100018442AF0A5F918A93046FEF7D1FB0446C2
:10C82000E3E70B4893E74346129A39462846CDF88A
:10C83000009001F0EFFECDE7B9D00460070080FF63
:10C840007CD1046018D404606CD10460F0B304603F
:10C85000F8B304602DE9F74F054608680C46F9F770
:10C86000A3FB012D8146DFF828A120D9022D67689E
:10C870001ED0A068F9F7E2FC054600210846FDF746
:10C880008FF8694680462068FEF72AFC009E5745CF
:10C890000446064443D1B442274629D238780134AD
:10C8A000F1F7F8FF0028F6D17DB3BA4606E0574607
:10C8B0004FF0FF35E1E75645544607D954460AF193
:10C8C000010A2078F1F7E6FF0028F4D0E21B394690
:10C8D0004846FEF7CBFB01464046FCF7A3FDA642C7
:10C8E00006D9A642274607D1002D0CDCB742DBD380
:10C8F000404603B0BDE8F08F38780134F1F7CAFF45
:10C900000028EED1F0E7013DF0E73946F21B48463A
:10C91000FEF7ACFB01464046FCF784FDE8E73846ED
:10C92000F9F742FB814502D03846FEF727FA01A904
:10C930003846FFF7D9F9019B8246ABB9134807F097
:10C94000A3FDF8F761FA37463A1B21464846FEF741
:10C950008DFB01464046FCF765FDB742C8D2019CFD
:10C96000002D3C4400DD013DDDF804B02746002DDC
:10C97000E9D007EB0B039E42E5D35A4651463846B1
:10C980002AF0E0F80028DFD00137F0E7B8CD0460E6
:10C9900074C8046002282DE9F04F064685B00C46A5
:10C9A00006D8FFF757FF0446204605B0BDE8F08FD4
:10C9B0000868F9F7F9FA02A9824620686768FEF765
:10C9C0008FFB8146A068F9F739FC051E02DA214683
:10C9D0003046E6E705F1010800214046FCF7E0FF9C
:10C9E000294B04469F4204D1284807F04DFDF9F732
:10C9F00075F803A93846FFF777F9039B834623B9F7
:10CA0000234807F041FDF8F7FFF9029E4E44039BCF
:10CA1000F71A5DB1B94509D81A4659463846019307
:10CA20002AF090F8019B00B3013FF2E7D4F80CB074
:10CA3000A6EB090249465046FEF718FB4BF82500C5
:10CA4000AF00002DB0D0A8EB0505E068AE00C1191D
:10CA500032462AF093F86268E0680021521B3044A5
:10CA600092002AF0A5F8A5609EE7E268F918504602
:10CA70000192F21B3E46D21AFEF7F8FA019B43F8E8
:10CA80002500013DC3E700BF74C8046034D10460D1
:10CA9000B8CD04602DE9FF410D4680460868F9F7DE
:10CAA00083FA02A907462868FEF71AFB03A9044681
:10CAB0006868FFF719F9B8F1020F064619D9012382
:10CAC000029A214638460093AB6800F039F9039A80
:10CAD000041B029B14449C420DD831462AF032F8C4
:10CAE000064B074A002814BF1846104604B0BDE89C
:10CAF000F0812046EBE70148F8E700BFF0B304609F
:10CB0000F8B3046073B50C46064669462068FEF724
:10CB1000E7FA01A905466068FFF7E6F8022E01462C
:10CB200004D90B4807F0B0FCF8F7D8FFDDE9003274
:10CB30009A420BD89B1AE8182AF004F8054B064ACB
:10CB4000002814BF1846104602B070BD0148FBE72C
:10CB500043D10460F0B30460F8B3046070B50C46D0
:10CB60008AB00546164604A92068FEF7B9FA049A69
:10CB7000002301460244009506A8059305ABCDE9C4
:10CB80000146FFF7CBF806A90248FEF719FA0AB0EA
:10CB900070BD00BF18D40460044B0B60044BC1E9A6
:10CBA000013000230846CB60704700BF94C7046083
:10CBB000B5CB016073B5054601A98068FEF790FA10
:10CBC000019B0446E86898420DD204442046F1F7E0
:10CBD0003BFE061B20463146FEF7EAF9E968314480
:10CBE000E96002B070BD0020FBE7000013B5044609
:10CBF000084601A9FEF774FA042C04D0052C09D0CC
:10CC0000002002B010BD019A0648074B002A08BF59
:10CC10001846F6E70199F1F72DFE400040F00100BB
:10CC2000EFE700BFF8B30460F0B304602DE9F74FFD
:10CC300015460446084601A9FEF752FA032D06469A
:10CC4000019A06D101462046FEF72EF903B0BDE851
:10CC5000F08F2DB9034630492046F1F7CBFDF5E7BB
:10CC600000EB020803460022984516D8002A0CBFA4
:10CC700027272227DFF8BC903A46DFF8BCA02046E1
:10CC8000DFF8B8B02549F1F7B5FDB0450FD83A4601
:10CC900022492046F1F7AEFDD8E713F8011B2729FA
:10CCA00003D02229E0D12727E4E70122DCE7304640
:10CCB000F1F7ADFD05463046F1F7C6FDAF42064639
:10CCC00005D13A4616492046F1F794FDDDE75C2D83
:10CCD00004D114492046F1F70BFAD6E7A5F1200359
:10CCE0005E2B02D82A460D49EDE70A2D01D10E49E7
:10CCF000F0E70D2D01D10D49ECE7092D01D10C49CB
:10CD0000E8E7FF2D2A4601D85946DCE7B5F5803F14
:10CD100034BF51464946D6E7FBCD0460AE86056078
:10CD20003FCD046043CD046046CD046049CD04602E
:10CD30004CCD0460CFD3046058CD04604FCD046067
:10CD4000F7B51E462B4B0D46144683429DF82070C6
:10CD500008D13B4632462146F9F7AEFB054428464A
:10CD600003B0F0BDF3070BD57610019601992A198F
:10CD700000292ADA013A0020134691B9551CEEE742
:10CD800001A93046F9F796FA0028EFD11A4807F0C2
:10CD90007BFB04463046F9F73EF901462046F8F79A
:10CDA00051F8AA4208D200B10191002FD7D11348FF
:10CDB00007F06AFBF8F720F81B78013A03F0C0038C
:10CDC000802B1CBF01310120D6E70024954205D3FA
:10CDD00004B10191002FEAD01546C0E70139BED356
:10CDE000681C0124054601302B7803F0C003802B1A
:10CDF000F8D0EBE77CD10460D6D30460FED30460A6
:10CE0000F0B5044687B017460E46F9F7CDF802A9EB
:10CE100005462046FEF764F9042F044653D1B307B4
:10CE200038D13268294B9A4234D105AB04AA03A900
:10CE30003046FDF75FFF264F059BBB4206D0032B14
:10CE400004D0244807F020FBF8F748FE039BBB42C0
:10CE50001AD00122214628460092029AFFF770FF5D
:10CE60000646049B029ABB4210D00121284600913D
:10CE70002146FFF765FF86420AD8821B31462846C5
:10CE8000FEF7F4F807B0F0BD2646EAE7A018F2E78F
:10CE90000E20F7E70023029A2146284600933346E6
:10CEA000FFF74EFF90F900300278002B08DB0121DC
:10CEB000FEF77EF8E6E701315B081A42FBD1F7E79F
:10CEC00040230121F9E70020DCE700BFD0CC04605B
:10CED00074C8046000B20460086801F06DBC000012
:10CEE00030B40A460D68054C0549064B8D420CBF0F
:10CEF0002146194630BCF1F77DBC00BF3CD504602B
:10CF0000D0D504604FD5046008B5024807F0BCFADC
:10CF1000F7F77AFF61D504602DE9F84345680446C8
:10CF20000F46164698460DB9FFF7EEFF2B7BDB0741
:10CF300013D500216868D5F80890EFF7ADFAA8601E
:10CF4000636849465A68986829F00AFE63681A7B44
:10CF50006FF300021A730023E360A568AD1924D2B1
:10CF60006368D3E90028AA4205D25A606068016864
:10CF7000691AF1F725F8A268424507D96368A2EB60
:10CF8000080200219868404429F012FE6368324686
:10CF900039469868A368184429F0E2FD6368A560E3
:10CFA0005A68AA4238BF5D6004E01B234FF0FF3689
:10CFB000C8F800303046BDE8F8830000F0B50746F9
:10CFC00085B00D46102000211646EFF765FA0023C4
:10CFD00004460760C0E90233002D3CD03068C50725
:10CFE00005D4810713D102681C4B9A420FD100254A
:10CFF000F9F724F9F0F7B1FF606035B3002320465C
:10D00000DDE90112FFF788FF0023A3601DE0012284
:10D0100001A9F9F721FB3368114A1A40062A06D004
:10D020009A0715D11B689A690E4B9A4210D10021BC
:10D030001020EFF731FA6060DDE90121F0F76CFFB5
:10D040006368029A5A603368E360204605B0F0BD19
:10D0500002980125CEE71020CCE700BF6CC3046026
:10D06000070080FFF1C201600229F8B5044605D02F
:10D07000042923D001291CD1002024E05668012E68
:10D0800010D0022E10D00020156829182CBF0127BF
:10D09000002766B1002D0ADA884238BF0021A1605E
:10D0A0001160E9E78068EFE741684868ECE7002F26
:10D0B000F5D016224FF0FF301A6004E04068F0F718
:10D0C00058FF00206060F8BD38B543680BB9FFF722
:10D0D0001BFF0568064C0748D3E90121064B854232
:10D0E0000CBF20461846BDE83840FDF7BFBF00BF63
:10D0F00018D40460D0D504607CD1046070B50546B6
:10D1000008466E680EB9FFF7FFFE7468A9688C4286
:10D110000DD9641AB3689442194428BF14462246B4
:10D1200029F01EFDAB682344AB60204670BD00248F
:10D13000FBE7D0E9022351688B4237BF991C0022DC
:10D14000013352F8212038BFC360104670470000F9
:10D15000044B0B60044BC1E9013000230846CB604F
:10D16000704700BF94C7046033D10160032A2DE9E2
:10D17000F84304460F46154612D11649F0F7B8FF9A
:10D1800007F108080026DFF860907B68B3420CD8EE
:10D19000032D17D110492046BDE8F843F0F7A8BF8A
:10D1A0000E490125F0F7A4FFEAE71EB149462046E3
:10D1B000F0F79EFF2A4658F8041B20460136F8F780
:10D1C00033FFE2E7012B03D105492046F0F790FF3A
:10D1D0000449E0E78EB2046028C00560B5CC046065
:10D1E00094D60460E0880560CD04066002460868B5
:10D1F0000B46083050F8041C01F08EBA0A4608307D
:10D2000050F8041C01F0BEBA052870B50D461ED0BA
:10D21000062808D004281DD14A680F480F4B002A61
:10D2200008BF184670BD0E4C01235E1C6A68013BA6
:10D230009A4203D8600040F00100F3E755F8261049
:10D240000620F7F70DFE334604EB6004EDE748686F
:10D250004000F0E70020E5E7F8B30460F0B30460B5
:10D2600098D6046038B50D46044698B102300021C6
:10D270008000EFF711F9084BC0E900344DB100F11F
:10D280000802002355F8231001339C4242F8041B86
:10D29000F8D138BD0148FCE7A0D6046098D60460F8
:10D2A00010287FB504460E4615460AD005D8042836
:10D2B00049D90E2820D0002440E01A281CD01C2870
:10D2C000F9D103A92846F8F7F5FF0028F3D0039910
:10D2D000002936DD706801F0E9F80021FFF7C2FF90
:10D2E00000F108030446726800930421039B06F1D1
:10D2F000080001F0EBF821E02846F8F755FE214937
:10D3000000F0A0FF0028D6D06B6800217068184498
:10D31000FFF7A8FF726800F1080306F10801920008
:10D320000446184629F01CFC6A680346706892009F
:10D3300005F1080103EB800029F012FC204604B03F
:10D3400070BD114CFAE71046F8F72EFE0F4B426AFB
:10D350009A4209D028460B4901F000F8054618B951
:10D36000022CA8D10A4CE9E76B6806F10801726843
:10D370002046009305F1080301F080F90028F1D060
:10D38000044CDBE7A0D6046098D6046051D101605C
:10D39000F0B30460F8B30460042A7FB504460D4678
:10D3A00037D103681A6A1C4B9A4203D01B4900F01C
:10D3B000D5FF044615F00306606820D12A68184B93
:10D3C0009A421CD101AA294601F094F820B91548C7
:10D3D00007F05AF8F8F782FBDDE9013031460834EE
:10D3E000C01AFFF73FFF01994268054604EB81012F
:10D3F0000830920029F0B4FB284604B070BD2A46DC
:10D40000014600232068F9F757F8023054F82050FD
:10D41000F2E70025F0E700BF99D30160A0D60460D1
:10D42000D0CC046000B204602DE9F3410C461646EE
:10D4300000221946204601230092F8F7E5FB7CB351
:10D440003568AB0703D12A68164B9A4218D00021E1
:10D450001020EFF721F8002104463068F8F780F833
:10D460000025804604274046F8F7D4F8064658B908
:10D4700028462146FFF7F6FE05462046EFF737F827
:10D48000284602B0BDE8F081AF4205D8F900204639
:10D49000EFF720F804467F0044F825600135E2E705
:10D4A000014DEDE7A0D6046098D6046043680830CB
:10D4B0000B6010607047EFF71AB80000F8B50E4621
:10D4C000114C1249124B88421AD0C268A24203D0B2
:10D4D000012430602046F8BD406B98B102689A4242
:10D4E000F1D100F108054768002405EB8707BD422C
:10D4F000F0D2314655F8040BFFF7E0FF0444F6E79D
:10D500000024E7E70446E5E76DDE016020C704601C
:10D51000A0D60460F0B50C4685B0054654F8046BFF
:10D5200003A90192002203923068FFF7C7FF039816
:10D53000019B2246C768691EB8473061014805B0A3
:10D54000F0BD00BF74C804602DE9F04705460C46E5
:10D55000DFF8C8802F4FDFF8C890AB684BB1E268A6
:10D56000424506D0E35823B1EB6804221A60BDE8B7
:10D57000F087A06BD8B1696800220430C90041F07F
:10D58000060129F055FB90B1297C4268EB6829B16E
:10D5900029680020BDE8F047F7F756BD910703D191
:10D5A00010681D498842E1D021462868F2E72B68BF
:10D5B00093B9646B002CDAD023684B4509D1A2469D
:10D5C0005AF8046F04EB8604261D5AF8044FB2453E
:10D5D00014D3BC42C1D1CAE72A7C002AE9D1E2684F
:10D5E0004245E6D0BC42E4D01869EA686968F7F7BA
:10D5F000ABFDEB681B68002BDBD0B8E7BC42E4D086
:10D6000021462846FFF7A0FFEB681B68002BDCD003
:10D61000ADE700BF20C70460F0C704606DDE0160A5
:10D62000A0D6046073B504460026084619460123B7
:10D63000154600961A46F8F7E7FA31460820EEF745
:10D640002BFF2A68C0E9004202B070BDCA880149B8
:10D65000F1F7D0B810D70460F0B58BB00F460021B9
:10D660000646154606A81022CDE9001129F0A0FAB9
:10D670002023316805960793CDF820D0B5B90E2345
:10D6800005A80693FFF760FF0221009C042C18D127
:10D690003069F8F789FC2A46036A394630469847CC
:10D6A000044606F01FFE20460BB0F0BD042D01D14C
:10D6B0001923E5E7442305A80693FFF745FF032157
:10D6C000E3E7002CEFD02046054C02AB0022049586
:10D6D000CDE90267F7F744FC042D08BF0446E2E7F2
:10D6E00074C804602DE9F0438DB0136814460190AE
:10D6F000002B30D11E290646D0E90120CDE909349E
:10D70000CDE907018DF82C3008BF0C23516B08BF01
:10D710000993B9B10A682F4B9A421FD10D460027D1
:10D72000DFF8B89055F8048F47450BD055F8041F23
:10D73000494501D10137F7E707A8FFF705FF23683F
:10D74000002BF7D02568002D3DD0042D0DD1224BA4
:10D750002360B36863600DB0BDE8F0831F4B99424E
:10D76000F0D007A8FFF7F0FEECE715F0030216D1A2
:10D7700029681B4B994212D128460092FCF7E0FB26
:10D78000184B0068009A984204D1174806F07CFEB6
:10D79000F7F722FB01AB0121F7F7E2FB206003AAB8
:10D7A00017212846F7F7D0FC039B002BD3D0019814
:10D7B0000590F8F7F9FB03AA069000210220F7F77D
:10D7C00033FC2060C7E7054907A80995FFF7BCFEB1
:10D7D000C1E700BFA0D6046040DA046020C704603F
:10D7E000F0C7046074C8046087AC04602DE9F041A0
:10D7F000044688B00F461546DFF85880002618F812
:10D80000043003A8396804931823CDF818D0059381
:10D810008DF81C60CDE90066CDE90267FFF794FE44
:10D820000098042807D12A463969204629F010FAC1
:10D8300008B0BDE8F08130B16A46002101200295B0
:10D84000F7F7F2FBF4E7A4F109030B2BF0D80C3443
:10D85000E4B2D4E704D904601E4B70B50D4688B01D
:10D86000195C002301AA064603A88DF81C30CDE9F7
:10D8700003511421CDE905122968CDE90133FFF7E1
:10D8800063FE019C042C07D129693046F7F7E8FABA
:10D890000446204608B070BD64B120462946F7F71B
:10D8A000B9FB062E0446F4D1F8F7F6FC400040F030
:10D8B0000104EEE7062EECD11223296803A8049395
:10D8C000FFF742FE019B002BE3D16C0044F0010402
:10D8D000DFE700BF34DA046070B5151E88B00C466F
:10D8E0004FF000030CBF4521362101AA064603A8CC
:10D8F0008DF81C30CDE903410821CDE905122168DE
:10D90000CDE90133FFF720FE019B3BB935B9362342
:10D91000216803A8CDE90435FFF716FE0198042815
:10D9200019D12069F8F740FB134BC2689A4210D115
:10D930003DB12368D888F0F742FA01463046F0F747
:10D94000D7FB45F0800221693046F8F76DFB08B03F
:10D9500070BD2A46F7E728B12146F7F75BFB0022A6
:10D960000146F1E72046F8F756FB234602460349F5
:10D970003046F0F73FFFEAE73D7C01601DD70460C9
:10D9800038B504460D460B49F0F7B2FB0022696832
:10D990002046F8F749FB08492046F0F7A9FBA9689B
:10D9A00020460022F8F740FB20460449BDE83840F5
:10D9B000F0F79EBB2FD70460CD0406601BD7046030
:10D9C0002DE9F041174612688EB004460D46002A34
:10D9D00079D14FEAC1080390043048F00608414667
:10D9E00029F026F9064610B143683B600BE00F2D85
:10D9F0001AD160680009F9F7DFFF8046A3689E42EC
:10DA000004D3C7F800800EB0BDE8F081E36853F896
:10DA1000361003EBC60229B1042903D052684046F0
:10DA200029F00AF90136E9E7CDE90B078DF8340052
:10DA300009A82168CDE90945FFF786FD3E68002E5B
:10DA400031D023689B889A07DDD516F0030217D1E1
:10DA500031684F4B994213D130460192FCF770FA6E
:10DA60004C4B0068019A984204D14B4806F00CFDDB
:10DA7000F7F7B2F903AB0121F7F772FA3860C2E7A2
:10DA800005AA17213046F7F75FFB059B002BBAD09C
:10DA900003980790F8F788FA05AA08900021022059
:10DAA000F7F7C2FAEAE7182DADD005AA18210398B6
:10DAB000F7F74AFB059B002BA5D005AA31460120AC
:10DAC000CDF81C80ECE701687E688B889B0749D500
:10DAD000002303AACDE9090509A88DF83430CDE962
:10DAE0000333CDE90B32FFF72FFD0398002839D01F
:10DAF00010F003021DD10168254B994219D1019202
:10DB0000FCF71EFA234B019ACDE9054656B9806809
:10DB100098423FF478AF05AB32460121F7F720FA7F
:10DB2000002362E7406898423FF46DAF05AB0221E5
:10DB3000F4E705AA5EB90D21F7F706FB059B93B143
:10DB400005AA314601200794F7F76EFAE8E743216A
:10DB5000F7F7FAFA059B8BB105AA00210220CDE95F
:10DB60000746F1E756B9E9000222201D41F00601FF
:10DB700029F05EF800283FF446AFD1E7E900012222
:10DB8000201D41F0060129F053F84660C8E700BFA8
:10DB9000F0C7046074C8046087AC0460F0B589B055
:10DBA0000E4601242C210023174601AA03900546A6
:10DBB0008DF81C300692CDE90441016803A8CDE937
:10DBC0000133FFF7C1FC019B042B09D12869F8F749
:10DBD000EBF93A46C36A31462869984709B0F0BD67
:10DBE0002046FBE7F0B589B000252122242301AEB1
:10DBF000039004460F46016803A8019506968DF828
:10DC00001C507560CDE90423FFF79EFC019840B1DC
:10DC1000042808D12069F8F7C7F93946436A206912
